:020000040800F2
:10000000406C0324AD020008918B00086B4F000880
:100010008D8B00089908000883C0000800000000CC
:100020000000000000000000000000001F94000815
:100030002D0A000800000000318D000821950008FD
:10004000C7020008C7020008C7020008C70200086C
:10005000C7020008C7020008C7020008C70200085C
:10006000C7020008C7020008C7020008C70200084C
:10007000C7020008C7020008C7020008C70200083C
:10008000C7020008C7020008C7020008C70200082C
:10009000C7020008C7020008C7020008C70200081C
:1000A000C7020008C7020008C7020008C70200080C
:1000B000C7020008C7020008BD950008C702000873
:1000C000C7020008C7020008C7020008C7020008EC
:1000D000C7020008FDA30008C7020008C702000805
:1000E000C7020008C702000800000000C70200089D
:1000F000C7020008C7020008C7020008C7020008BC
:10010000C7020008C7020008C7020008C7020008AB
:10011000C7020008C7020008C7020008C70200089B
:10012000C7020008C7020008C7020008C70200088B
:10013000C7020008C7020008C7020008C70200087B
:1001400000000000000000000000000000000000AF
:10015000C7020008C7020008C7020008C70200085B
:10016000C7020008C7020008C7020008C70200084B
:10017000C7020008C7020008C7020008C70200083B
:10018000C7020008C7020008C7020008C70200082B
:10019000C7020008C7020008C7020008C70200081B
:1001A000C7020008C7020008C7020008C70200080B
:1001B000C7020008C7020008C7020008C7020008FB
:1001C000C7020008C7020008C7020008C7020008EB
:1001D000C7020008958B0008C7020008C702000884
:1001E000C7020008C7020008C7020008C7020008CB
:1001F000C7020008C7020008C7020008C7020008BB
:10020000C7020008C7020008C7020008C7020008AA
:10021000C7020008C7020008C7020008C70200089A
:10022000C7020008C7020008C7020008000000005B
:10023000C7020008C702000800000000C70200084B
:10024000C7020008C7020008C7020008C70200086A
:10025000C7020008C7020008C7020008C70200085A
:10026000C7020008C7020008C7020008C70200084A
:10027000C7020008C7020008C7020008000000000B
:10028000C702000800000000C702000800000000CC
:1002900000000000C7020008DFF80CD000F050FAA0
:1002A0000048004755CC0008406C032406488047AE
:1002B00006480047FEE7FEE7FEE7FEE7FEE7FEE74B
:1002C000FEE7FEE7FEE7FEE7299500089902000831
:1002D0002DE9F05F0546002092469B46884606467B
:1002E000814640241BE0284641464746224600F00E
:1002F0005EF853465A46C01A914110D3114618462B
:10030000224600F045F82D1A67EB01084F462246B9
:100310000120002100F03CF817EB00094E41201E9F
:10032000A4F10104DFDC484631462A464346BDE8D5
:10033000F09F40EA01039B0703D009E008C9121FA0
:1003400008C0042AFAD203E011F8013B00F8013B8F
:10035000521EF9D27047421C10F8011B0029FBD134
:10036000801A704730B50B46014600202022012438
:1003700009E021FA02F59D4205D303FA02F5491B73
:1003800004FA02F52844151EA2F10102F1DC30BD89
:10039000202A04DB203A00FA02F100207047914045
:1003A000C2F1200320FA03F3194390407047202A3A
:1003B00004DB203A21FA02F00021704721FA02F30F
:1003C000D040C2F1200291400843194670472DE900
:1003D000FE4F804681EA0300C00F0C46009021F0DA
:1003E000004123F00045B8EB0200A94105D2404688
:1003F000214690461C460B46024623F0004010431F
:1004000047D0270DC7F30A00C3F30A510290401AE0
:10041000019040286BDAC3F3130040F4801B00986E
:10042000924620B10023D2EB030A63EB0B0B019839
:100430005946C0F140025046FFF7AAFF06460D4656
:1004400050465946019A00F08DF910EB08006141C1
:10045000002487EA115284EAE7731A4340D0009AD5
:1004600062B3019A012A4FEA075215DC001B61EBC7
:1004700002014FF0004202EA0752CDE90042001C9F
:1004800041F5801132462B4600F08DF903B0BDE8EE
:10049000F08F40462146F9E7001B61EB0201001C8A
:1004A00041F5801300185B412018A2F5001747EBB7
:1004B000030140EAD570B6196D4111E06D084FEAAD
:1004C000360645EAC0754FEA0752001B61EB020190
:1004D000001C41F5801149084FEA300000195141D4
:1004E00032462B4603B0BDE8F04F00F04DB90098FE
:1004F000012240000023D0EB020263EBE07300987E
:1005000021464FEAE074B8EB000061EB0401E9E733
:1005100083F000435BE781F0004158E72DE9FE4F8F
:1005200081EA030404F0004421F0004100944FF0FC
:10053000000B23F0004350EA01045ED052EA0304AA
:100540005BD0C3F30A54C1F30A552C44A4F2F3342C
:100550000194A0FB0254C1F3130141F48011C3F3D1
:10056000130343F4801301FB024400FB034E840A8F
:10057000970A44EA815447EA8357A4FB0768029527
:100580008D0A05FB07854FEA932C04FB0C542705C5
:10059000029D4FEA065847EA1637B5EB08056EEBA1
:1005A000070C870E920E47EA811742EA8312A7FBD7
:1005B0000201B6EB0B0164EB00042B0D43EA0C3394
:1005C0005E1844EB1C50DA465146E7FB0201C5F3C6
:1005D00013044FEA0B3343EA14534FEA0432019CED
:1005E00043EA0603A4F10C040294009CCDE900B494
:1005F00000F0D9F803B0BDE8F08F00200146F9E71C
:100600002DE9F04D81EA030404F0004B21F0004590
:1006100014464FF0000A23F0004150EA050220D0B2
:1006200054EA01021DD0C5F30A570246C5F313036D
:10063000C1F31300C1F30A5640F4801543F480134C
:10064000A7EB0608101BD64608F2FD3873EB050031
:1006500002D308F1010801E092185B41B8F1000FE4
:1006600003DA00200146BDE8F08D00204FF4801130
:10067000064684460EE0171B73EB050705D3121BD5
:1006800063EB050306434CEA010C49084FEA3000CE
:1006900092185B4150EA0107EDD152EA030012D0F3
:1006A00082EA040083EA0501084305D0101BAB4130
:1006B00006D20122002306E000224FF0004302E0B0
:1006C0006FF0010253101AEB06004CEB085110EBCF
:1006D0000A0041EB0B01BDE8F04D00F055B8C1F345
:1006E0000A52C1F3130140F2FF3341F480119A42E0
:1006F00002DA00200146704740F233439A42A2F2E8
:10070000334202DC5242FFF752BEFFF741BE000007
:1007100030B5041E71F1000404DB4FF00044404288
:1007200064EB0101141E73F1000405DB1C464FF05D
:100730000043524263EB0403994208BF904230BD2C
:10074000064C074D06E0E06840F0010394E807001E
:1007500098471034AC42F6D3FFF7A2FD442B0108B2
:10076000642B0108202A06DBCB17203A41FA02F05D
:1007700043EAE07306E041FA02F3D040C2F12002FE
:10078000914008431946704710B5141E73F10004D8
:1007900008DA401C41F1000192185B411A4301D173
:1007A00020F0010010BD2DE9F04D92469B4611B19D
:1007B000B1FA81F202E0B0FA80F220329046FFF7FF
:1007C000E7FD04460F4640EA0A0041EA0B015346A2
:1007D0005A46084313D0114653EA010019D0C8F114
:1007E00040025046FFF7E3FD05460E465046594687
:1007F0004246FFF7CDFD084305D0012004E0204626
:100800003946BDE8F08D0020054346EAE0762C43EA
:1008100037430A986305E40AA0EB08000022FD0AAA
:1008200044EA47540A3002D500200146E9E70105B1
:1008300010196941DDE9084500196941BDE8F04D2D
:10084000A2E770B58C1810F8015B15F0070301D111
:1008500010F8013B2A1106D110F8012B03E010F823
:10086000016B01F8016B5B1EF9D12B0705D4002346
:10087000521E0DD401F8013BFAE710F8013BCB1AE8
:10088000921C03E013F8015B01F8015B521EF9D5DD
:10089000A142D8D3002070BD00BFFEE770B5054669
:1008A0000C461646042D15D007DC7DB1012D0ED067
:1008B000022D0DD0032D50D10BE0202D0BD0212D7A
:1008C00030D0222D47D0232D47D145E046E045E0EA
:1008D00044E043E042E02078617840EA0120A178DA
:1008E00040EA0140E17840EA01601E490860207951
:1008F000087160794871A0798871084601791AA059
:100900000BF0B4FC174841791DA00BF0AFFC154863
:10091000817922A00BF0AAFC1248016826A00BF0F6
:10092000A5FC1BE00F48007820700E480088000AE4
:1009300060700C480068000CA0700A480068000E47
:10094000E0700848007920710648407960710548D8
:100950008079A07102E001E000E000BF00BF00204C
:1009600070BD0000B80200246C696E65636F646935
:100970006E672E666F726D61743A25640D0A000011
:100980006C696E65636F64696E672E7061726974FD
:1009900079747970653A25640D0A00006C696E659A
:1009A000636F64696E672E64617461747970653A0F
:1009B00025640D0A000000006C696E65636F646950
:1009C0006E672E626974726174653A25640D0A005F
:1009D0000020704710B50349034809F031FE00209C
:1009E00010BD0000740F0024F802002470B5054605
:1009F0000C462846216808F0CDFA044809F0FCFDB1
:100A0000284621680BF040FB002070BDF80200244E
:100A100010B508F033FB08F0E3FA0348006840F033
:100A200004000149086010BD9CEF00E07047000021
:100A300070B504461D460023B5F5804F13D154F818
:100A400022300C480340D1E9000640EA06108E68C7
:100A500040EA06208E8940EA06408E69304303430F
:100A600044F8223003E06FF0704044F82200002088
:100A700070BD00000000F0CF10B5024600230868EA
:100A800052F820301B480340D1E901042043CC68D0
:100A900020430C6920434C6920438C692043CC6976
:100AA00020430C6A20434C6A20438C6A2043CC6A62
:100AB00020430C6B20438C6B20434C6B204303433F
:100AC0008868082801D143F04003086842F82030C4
:100AD000086BB0F5801F05D1086818B110680C6B61
:100AE00020431060086818B110684C6B20431060F8
:100AF000002010BD8004C0FF30B50346144600221C
:100B0000601C53F8202002F04042D1E9000540EA81
:100B100005108D6840EA05208D8940EA0545088A60
:100B2000401E45EA0055087D801E45EA00608D693B
:100B300028430243601C43F82020186800F480100A
:100B400038B1586820F47002088A401E42EA005208
:100B50005A60002030BD30B50246002300240868EA
:100B6000012816D013686FF30E03D1E9010528435D
:100B7000CD6828430D6928434D6928438D69284372
:100B8000CD6928430D6A28434D6A28430343136007
:100B900019E0136823F4F843D1E9070528434D6AA7
:100BA0002843034354686FF30E04D1E90105284339
:100BB000CD6828430D6928434D6928438D69284332
:100BC000044313605460002030BD0246506940EA7F
:100BD000410050610020704718B503460020009086
:100BE000D1E9000420438C68641E40EA4410CC68BC
:100BF00040EA4420009000981861002018BD0000D1
:100C000070B50346154600220024012D1FD09A68B6
:100C100002F070420868401E4E68761E40EA0616D2
:100C20008868401E46EA0026C868401E46EA00362C
:100C3000088A401E46EA0046888A401E46EA005658
:100C4000087E401E46EA006002439A6022E09A68ED
:100C500011480240C868401E0603888A401E46EAC2
:100C600000500243DC6804F070440868401E4E687F
:100C7000761E40EA06168868401E46EA0026088A64
:100C8000401E46EA0046087E401E46EA00600443D5
:100C90009A60DC60002070BDFF0F0FFF70B5052467
:100CA00006250726344454B108220549204604F09D
:100CB000DBFA042202491031284604F0D5FA70BD4F
:100CC0009E02002410B504460CB9012010BD94F812
:100CD0003500022803D0802060650120F6E7344902
:100CE0002068884205D333492068884201D8012012
:100CF00000E00020C0B1042084F835002C492068B1
:100D000088420AD32B492068884206D820680068A8
:100D100020F001002168086048E02068006820F0A9
:100D200001002168086041E02068006820F00E00A2
:100D3000216808601E49206888420AD31D4920683E
:100D4000884206D82068006820F001002168086009
:100D500005E02068006820F0010021680860206E2E
:100D6000006820F48070216E086094F85C10012007
:100D7000884011490860D4E919104860E06E40B11C
:100D8000E06E006820F48070E16E0860D4E91C1009
:100D9000486000BF002084F8340000BF012084F8C0
:100DA0003500206D10B12046216D884700208DE769
:100DB00010000240B80402400454025870B50446C2
:100DC00000F052F906462546681C10B10448007828
:100DD000054400BF00F048F9801BA842FAD370BD5B
:100DE0001C0000240348006840F00100014908602D
:100DF0007047000020040058F8B502460B46002159
:100E0000002600240020824D00BFFCE0012707FAE5
:100E100001F61F6807EA0604B4427CD15F68022F1E
:100E200002D05F68122F1AD14FEAD10C02F12007CD
:100E300057F82C004F074FEAD76C0F2707FA0CF72B
:100E4000B8434FEA417C4FEADC6C1F6907FA0CF7A4
:100E500038434FEAD10C02F1200747F82C00106804
:100E60004FEA410C032707FA0CF7B8431F7907F044
:100E700003074FEA410C07FA0CF7384310605F682C
:100E8000012F08D05F68022F05D05F68112F02D0B4
:100E90005F68122F17D190684FEA410C032707FAB9
:100EA0000CF7B8434FEA410CDF6807FA0CF73843F8
:100EB0009060506801278F40B8431F79C7F300172F
:100EC0008F4038435060D0684FEA410C032707FA3F
:100ED0000CF7B8434FEA410C9F6807FA0CF7384308
:100EE000D0605F6807F08057B7F1805F95D100BF91
:100EF000484F3F6847F00207DFF818C1CCF8007090
:100F000067463F6807F00207009700BF00BF424FE7
:100F10004FEA910C00E075E057F82C008F074FEA7C
:100F2000177C0F2707FA0CF7B8433C4FBA4201D1A0
:100F300000272DE03A4FBA4201D1012728E0394F6E
:100F4000BA4201D1022723E0374FBA4201D1032729
:100F50001EE0364FBA4201D1042719E0344FBA429D
:100F600001D1052714E0334FBA4201D106270FE023
:100F7000314FBA4201D107270AE0304FBA4201D1BE
:100F8000082705E02E4FBA4201D1092700E00A27C1
:100F90004FEA817C4FEA1C7C07FA0CF738431E4F5E
:100FA0004FEA910C47F82C002868A0435F6807F4CB
:100FB0008037B7F5803F00D1204328606868A043A0
:100FC0005F6807F40037B7F5003F00D12043686041
:100FD0004FF0B0473868A0435F6807F48017B7F553
:100FE000801F00D120434FF0B04738607868A0439D
:100FF0005F6807F40017B7F5001F00D120434FF0DA
:10100000B0477860491C1029FFF400AFF8BD00001C
:1010100080000058F44402580804005800000258A8
:101020000004025800080258000C02580010025830
:101030000014025800180258001C025800200258E0
:1010400000240258024613690B400BB1012000E056
:101050000020704742694A40426170470AB10183EB
:1010600000E04183704700000148006870470000BD
:101070001400002403480068034909780844014922
:1010800008607047140000241C00002410B50320E1
:1010900000F08AFA002000F007F808B1012010BD26
:1010A00000F034FA0020FAE770B504460E480078E4
:1010B0004FF47A71B1FBF0F00C490968B1FBF0F51F
:1010C000284603F0E7FC08B1012070BD102C07D2C0
:1010D00000222146501E00F02AFA0548046001E073
:1010E0000120F2E70020F0E71C00002400000024AB
:1010F0001800002470B504460E46154600BF94F84B
:10110000A000012801D1022070BD012084F8A000B8
:1011100000BF022084F8A10005EB850101EBC502A8
:1011200004F1380101EB820034223146FFF701F966
:101130002A463146204607F0D9FB01202168486243
:1011400084F8A10000BF002084F8A00000BF00BF09
:10115000DAE7000070B50446002500260CB901202E
:1011600070BD94F8A10028B9002084F8A0002046A2
:1011700000F07EF8022084F8A1002068806920F049
:10118000704021688861D4E901010843E16808439F
:1011900021690843216889690843216888612068BA
:1011A00080683249084021688860A08A0504206868
:1011B0008068A16929430843216888602068C06865
:1011C0002A4908402168C860A08B05042068C068CF
:1011D000216A294308432168C860206800692349BF
:1011E000084021680861A08C050420680069A16A94
:1011F0002943084321680861206840691B49084069
:1012000021684861A08D050420684069216B29434D
:1012100008432168486194F83500050294F83600C7
:1012200006042068C06A00F07F402168C86246EA70
:10123000050094F8341008432168C96A08432168FE
:10124000C8622068406B40F006002168486320684F
:10125000806940F00100216888610020C4F8A40082
:10126000012084F8A10000207AE7000000F800F0D7
:1012700010B586B0044600BF3748006840F008004B
:10128000354908600846006800F00800009000BF7B
:1012900000BF00BF30481038006840F010002E49F1
:1012A000103908600846006800F01000009000BF88
:1012B00000BF00BF2848001F006840F48070264926
:1012C000091F08600846006800F48070009000BFA5
:1012D00000BF00BF0846006840F400700860084680
:1012E000006800F40070009000BF00BF00BF084617
:1012F000006840F4806008600846006800F4806080
:10130000009000BF00BF20200190012002900390B8
:101310000320049001A91148FFF76EFD4FF4E0404F
:1013200001900220029000200390032004900E20E0
:10133000059001A90A48FFF75FFD48F67C6001901F
:1013400001A90848FFF758FDFF20019001A90648B0
:10135000FFF752FD06B010BDE444025800040258E5
:101360000020025800240258002802582DE9F041BC
:1013700004460E461746984600BF94F8A000012880
:1013800002D10220BDE8F081012084F8A00000BF56
:10139000022084F8A10008EB880000EBC80104F1EA
:1013A000380000EB81052E60A86A30446860AF60A9
:1013B000E86A3844E86042462946204607F096FA33
:1013C00001202168486284F8A10000BF002084F851
:1013D000A00000BF00BFD5E72DE9F04104460E464E
:1013E0001746984600BF94F8A000012802D10220B9
:1013F000BDE8F081012084F8A00000BF022084F83D
:10140000A10008EB880000EBC80104F1380000EBF4
:101410008105286830446860A8683844E860AE6296
:10142000EF6242462946204607F060FA0120216813
:10143000486284F8A10000BF002084F8A00000BF2B
:1014400000BFD5E74178154A11600178F9B1121D46
:1014500041681160017B0907C27A41EA0261827A20
:1014600041EAC241427B41EA8241827B41EA4241F8
:10147000C27B41EA0241427A41EA0221027A41EA10
:10148000420102781143054A0832116005E000214B
:10149000024A121D1160121D1160704798ED00E0A4
:1014A00000BF00BF00BFBFF35F8F00BF00BF00BF22
:1014B0000548006820F48030034908600020024994
:1014C000703108607047000024ED00E040F0010139
:1014D0000D4A11600C497039096841F480310A4A9B
:1014E000703A116000BF00BF00BFBFF34F8F00BF55
:1014F00000BF00BF00BF00BF00BFBFF36F8F00BFC2
:1015000000BF00BF7047000094ED00E07047014647
:101510000846002809DB00F01F0301229A40430916
:101520009B0003F1E023C3F8002100BF70472DE9C1
:10153000F05F80460D4616460AF0BAFE0746394669
:101540002A46334601F00700C0F1070ABAF1040F3A
:1015500002D94FF0040A01E0C0F1070AD14600F1B8
:10156000040ABAF1070F02D24FF0000A01E0A0F11D
:10157000030AD4464FF0010A0AFA09FAAAF1010A4D
:101580000AEA020A0AFA0CFA4FF0010B0BFA0CFBFA
:10159000ABF1010B0BEA030B4AEA0B042146404670
:1015A0000AF08EFEBDE8F09F00BF00F00702064B78
:1015B00019684FF6FF031940044B0B4343EA02211D
:1015C000014B196000BF70470CED00E00000FA0508
:1015D000024611680120C2F8F803886B40F400301D
:1015E0008863886B40F48020886300207047000087
:1015F00001460A680120C1F8F403002081F8EC03D9
:10160000906940F000609061506D024B1843506546
:1016100000207047030000107047024610684162C6
:1016200000207047F0B503461446002500221868D4
:10163000426A21B942EA04401E68B06219E01868A3
:10164000806A02EB1042002508E0186800F58270FD
:1016500050F8250002EB1042681CC5B2481EA84293
:10166000F3DC42EA0447186800F582704E1E40F829
:1016700026700020F0BD000010B50446012003498B
:101680000870D4F8FC0309F0FBFA10BD65020024D1
:1016900070B504460D46C5EBC50304F1380101EBF6
:1016A0008301CA682946D4F8FC0309F039FA70BDF1
:1016B00070B504460D46C5EBC50304F5FC7101EB9E
:1016C0008301CA682946D4F8FC0309F096FA70BD74
:1016D00010B5044600200549087005A00AF0C6FDB3
:1016E000D4F8FC0309F0CFFA10BD00006502002415
:1016F0005553422044657669636520446973636F7E
:101700006E6E65637465642E0D0A000070B5044644
:101710000D46002605F08000802808D105F07F00E6
:10172000C0EBC00104F1380000EB810607E005F0D2
:101730007F00C0EBC00104F5FC7000EB810605F0F2
:101740007F00307005F08000C009707000BF94F811
:10175000B803012801D1022070BD012084F8B8032C
:1017600000BF3146206809F057FF00BF002084F811
:10177000B80300BF00BFEFE770B504460D46002672
:1017800005F08000802808D105F07F00C0EBC00183
:1017900004F1380000EB810605E0C5EBC50104F556
:1017A000FC7000EB81060020B07005F07F00307007
:1017B000C5F3C010707000BF94F8B803012801D1C0
:1017C000022070BD012084F8B80300BF31462068B4
:1017D0000AF06CF900BF002084F8B80300BF00BF16
:1017E000EFE7024601F00F00C0EBC00302F5FC700A
:1017F00000EB8300008B80B270472DE9F04705466F
:101800000E4690461F464FF00009002406F0800067
:10181000802808D106F07F00C0EBC00105F1380038
:1018200000EB810407E006F07F00C0EBC00105F586
:10183000FC7000EB810406F07F00207006F0800051
:10184000C0096070C4F80880E770607808B120783B
:10185000E080022F01D10020207100BF95F8B8036D
:10186000012802D10220BDE8F087012085F8B803E5
:1018700000BF2146286809F0EDFD00BF002085F873
:10188000B80300BF4846EEE72DE9F04104460E4696
:1018900017469846002506F07F00C0EBC00104F50E
:1018A000FC7000EB8105EF60C5F814800020A86192
:1018B000687006F07F0028702069012800D12F6130
:1018C00006F07F0028B9227C2946206809F0F4FF41
:1018D00004E0227C294620680AF072F90020BDE865
:1018E000F08170B504460D46002605F08000802882
:1018F00008D105F07F00C0EBC00104F1380000EB17
:10190000810605E0C5EBC50104F5FC7000EB81061E
:101910000120B07005F07F003070C5F3C01070700A
:1019200000BF94F8B803012801D1022070BD012046
:1019300084F8B80300BF314620680AF0FBF805F0D0
:101940007F0028B9217C04F56F7220680AF08CF8BA
:1019500000BF002084F8B80300BF00BFE6E72DE910
:10196000F04104460E4617469846002506F07F00D3
:10197000C0EBC00104F1380000EB8105EF60C5F851
:1019800014800020A8610120687006F07F00287094
:101990002069012800D12F6106F07F0028B9227C40
:1019A0002946206809F088FF04E0227C2946206847
:1019B0000AF006F90020BDE8F08100002DE9FC5F87
:1019C000044626684FF0000B002001908046002559
:1019D000009081468246FE4F20680AF0B1FA002846
:1019E0007DD120680AF0E4FA08B9BDE8FC9F2068C0
:1019F0000AF0DEFA00F00200022801D121684861F5
:101A000020680AF0D5FA00F40020B0F5002F67D165
:101A1000002520680AF0A2FA0190A8E0019800F0E1
:101A2000010000287ED0E9B220680AF0B6FA8046AC
:101A300008F00100002860D0012106F5306000EBBD
:101A400045108160306CE34988420ED3206901283B
:101A50000BD1D6F8080B00F4004030B14FF4004130
:101A600006F5306000EB45108160206901282BD11C
:101A7000C5EBC50104F5FC7000EB8100816806F53B
:101A8000306000EB45100069C0F31200091AC5EB85
:101A9000C50204F5FC7000EB82008161C5EBC50155
:101AA00004F5FC7000EB8100C5EBC502C16804F5CC
:101AB000FC7000EB820080680144C5EBC50204F5B0
:101AC000FC7000EB8200C160E9B22046FFF7F0FD38
:101AD0002069012811D185B9C5EBC50101E0EEE20D
:101AE00049E004F5FC7000EB8100406928B904F579
:101AF0006F720121206809F0B7FF08F0080008287C
:101B00001DD1306CB349884210D3206901280DD112
:101B1000D6F8080B00F4004040B14FF4004106F540
:101B2000306000E01FE000EB45108160204600F0CF
:101B300071FC082106F5306000EB4510816008F06B
:101B40001000102805D1102106F5306000EB45107B
:101B5000816008F02000202805D1202106F53060A2
:101B600000EB451081606D1C0198400801900198C0
:101B700000287FF453AF20680AF01AFA00F480209E
:101B8000B0F5802F7DD120680AF0DFF901900025A3
:101B900085E0019800F0010000287CD0E9B22068BF
:101BA0000AF0E5F9804608F00100E8B30120A840FA
:101BB000009040F6340080590099884340F6340183
:101BC0008851012106F5106000EB45108160206905
:101BD000012815D1C5EBC50104F1380000EB8100E7
:101BE000C5EBC502C16804F1380000EB82008068D3
:101BF0000144C5EBC50204F1380000EB8200C1606E
:101C0000E9B22046FFF744FD2069012810D15DB9F3
:101C1000C5EBC50104F1380000EB8100406918B93B
:101C200004F56F72012100E002E0206809F01CFF5A
:101C300008F00800082805D1082106F5106000EB1F
:101C40004510816008F01000102805D1102106F51C
:101C5000106000EB4510816008F04000402805D17D
:101C6000402106F5106000EB4510816008F002008D
:101C7000022805D1022106F5106000EB45108160B5
:101C800001E010E007E008F08000802803D1294639
:101C9000204606F087FF6D1C0198400801900198CE
:101CA00000287FF476AF20680AF082F900F0004047
:101CB000B0F1004F1AD140F60400805920F0010124
:101CC00040F60400815194F8EC03012807D100206C
:101CD00084F8EC0300212046FFF79EFC02E020463A
:101CE00000F064FB4FF000402168486120680AF072
:101CF0005FF900F40060B0F5006F0CD140F6080009
:101D0000805900F0010010B1204600F097FB4FF41D
:101D100000602168486120680AF04AF900F000601C
:101D2000B0F1006F17D14FF000602168486194F85E
:101D3000EC0368B9012084F8EC032068406DC0F31F
:101D40008300C4F8F00301212046FFF765FC02E0A0
:101D5000204600F073FB20680AF02AF900F4805056
:101D6000B0F5805F60D140F60400805920F0010199
:101D700040F604008151102120680AF0A7F84FF0C6
:101D8000000B0CE0FF2106F5106000EB4B108160AA
:101D900006F5306000EB4B1081600BF1010B6068C1
:101DA0005845EFD84FF0FF3140F618008151001D23
:101DB000805940F0011140F61C008151206BA0B108
:101DC000D6F8840840F00B01C6F8841804E000003F
:101DD0000084D7170A31544F40F64400805940F030
:101DE0000B0140F6440081510EE040F6140080598A
:101DF00040F00B0140F614008151001F805940F063
:101E00000B014FF401608151D6F8000820F4FE6008
:101E1000C6F80008217C04F56F72206809F024FEE2
:101E20004FF480502168486120680AF0C1F800F43E
:101E30000050B0F5005F7AD1206809F06DFB206892
:101E4000C06820F470502168C86020680AF056F815
:101E500058B90021E1604FF4007161612068C068E9
:101E600040F410502168C86082E00321E160402105
:101E7000616101F02DFC07469248874209D39248E0
:101E8000874206D22068C06840F470502168C8605C
:101E90006EE08D48874209D38C48874206D220687D
:101EA000C06840F460502168C86061E0874887429C
:101EB00009D38748874206D22068C06840F4505052
:101EC0002168C86054E08248874209D3814887422C
:101ED00006D22068C06840F440502168C86047E0DE
:101EE0007C48874209D37C48874206D22068C06874
:101EF00040F430502168C8603AE07748874209D3FF
:101F00007648874206D22068C06840F42050216895
:101F1000C8602DE0714887420AD37148874207D2D2
:101F20002068C06840F410502168C86020E026E0B6
:101F30006B48874209D36B48874206D22068C06845
:101F400040F400502168C86012E06648874209D317
:101F50006548874206D22068C06840F4E050216896
:101F6000C86005E02068C06840F4C0502168C860BF
:101F7000204600F0CFF94FF40050216848612068F6
:101F80000AF016F800F01000102845D1206880698A
:101F900020F0100021688861D6F8209009F00F0029
:101FA000C0EBC00104F5FC7000EB810AC9F34340AB
:101FB00002281AD147F6F07009EA000030B3C9F3DD
:101FC0000A123046DAF80C1009F0F8FFC9F30A11CA
:101FD000DAF80C000844CAF80C00C9F30A11DAF860
:101FE00018000844CAF8180010E0C9F34340062856
:101FF0000CD1082204F56F71304609F0DFFFC9F3F8
:102000000A11DAF818000844CAF818002068806934
:1020100040F0100021688861206809F0C9FF00F0D5
:102020000800082805D1204600F0D4F908202168CE
:102030004861206809F0BCFF00F48010B0F5801FF3
:1020400007D1E9B2204600F051F84FF48010216822
:102050004861206809F0ACFF00F40010B0F5001FE3
:1020600007D1E9B2204600F04AF84FF40010216889
:102070004861206809F09CFF00F08040B0F1804F7B
:1020800006D12046FFF7F8FA4FF0804021684861FA
:10209000206809F08DFF00F0040004280FD12068AB
:1020A000D0F8049009F00400042802D12046FFF77C
:1020B0000FFB2068406840EA09002168486000BFC3
:1020C00093E40000C0ACD800C0E1E4000024F400B8
:1020D00080730601A0491A01002D310140A44C0172
:1020E00000366E0120ABA6010048E80170B5044639
:1020F0000D462946D4F8FC0308F02AFE70BD70B5E1
:1021000004460D462946D4F8FC0308F024FE70BDB1
:1021100030B58BB00446002514B901200BB030BD9A
:10212000032084F8B903204600F0A0F8206809F0E5
:10213000BBFB282204F110016846FEF7FAF894E888
:102140000F0009F00BFA0021206809F04BFF002571
:1021500030E00121C5EBC50204F1380000EB82003C
:102160004170C5EBC50204F1380000F82250C5EB00
:10217000C50200EB8200C5800021C5EBC50204F159
:10218000380000EB8200C170C5EBC50204F13800D5
:1021900000EB82008160C5EBC50204F1380000EB62
:1021A0008200C160C5EBC50204F1380000EB82007B
:1021B00041616D1C0F2DCCD3002536E00021C5EB0D
:1021C000C50204F5FC7000EB82004170C5EBC5024E
:1021D00004F5FC7000F82250C5EBC50204F138008C
:1021E00000EB8200C580C5EBC50204F5FC7000EB76
:1021F0008200C170C5EBC50204F5FC7000EB8200E3
:102200008160C5EBC50204F5FC7000EB8200C16083
:10221000C5EBC50204F5FC7000EB8200416120684B
:1022200000F5827040F825106D1C0F2DC6D32822B2
:1022300004F110016846FEF77CF894E80F0009F0FD
:102240005DFA012084F8B903A06A012802D1204672
:10225000FFF7CEF9606A012802D12046FFF7B8F9EE
:10226000206809F03CFA002058E7000010B5B6B02D
:1022700004464FF4802002904FF44010239002A8AF
:1022800000F062FB20492068884239D100BF1F4816
:10229000006840F001001D4908600846006800F031
:1022A0000100019000BF00BF4FF4C05031900220E8
:1022B000329000203390032034900A20359031A9C9
:1022C0001348FEF799FD0121032006F00AFD00BF27
:1022D0000E480838006840F000600C490839086072
:1022E0000846006800F00060019000BF00BF0022B7
:1022F00001216520FFF71BF96520FFF708F900E0D1
:1023000000BF36B010BD000000000840E044025895
:102310000000025870B504460125E06810B102289B
:102320000AD104E00CA009F0A1FF002509E011A0EA
:1023300009F09CFF012504E015A009F097FF012595
:1023400000BF00BFD4F8FC0308F028FD2946D4F8EC
:10235000FC0308F05DFD70BD55534220446576696D
:102360006365204C69627261727920205B48535D1D
:102370000D0A000055534220446576696365204C80
:1023800069627261727920205B46535D0D0A00001C
:1023900055534220446576696365204C69627261D9
:1023A000727920205B46533F5D0D0A0010B504464C
:1023B00003A009F05BFFD4F8FC0308F011FD10BD89
:1023C00044657669636520526573756D65640D0AB1
:1023D0000000000010B50446D4F8FC0308F007FD27
:1023E00010BD70B504460D4600BF94F8B80301282F
:1023F00001D1022070BD012084F8B80300BF294636
:10240000206809F007FE00BF002084F8B80300BF71
:1024100000BFEFE710B5044604F56F71D4F8FC0374
:1024200008F00AFD10BD10B50446206809F048F90F
:10243000206809F02DFD002010BD000010B50446F5
:1024400000200549087005A009F010FFD4F8FC032E
:1024500008F03BFD10BD000065020024446576696C
:10246000636520496E2073757370656E64206D6FAF
:1024700064652E0D0A0000000348006840F080707B
:1024800001490860704700000C48025810B501F07F
:1024900067F90949096801F470614FF4807292FA92
:1024A000A2F2B2FA82F2D140044A515CC840044917
:1024B00008600846006810BD1844025824E300086C
:1024C0000000002410B501F003F90749096801F084
:1024D0007001102292FAA2F2B2FA82F2D140034ABB
:1024E000515CC84010BD00002044025824E300089D
:1024F00070B5014600220120002300249FED811ABF
:10250000B0EE410A9FED7F1AF0EE410A7E4D2D6834
:1025100005F003027C4D2D68C5F305307A4D2D1D65
:102520002D6805F01003784D14352D68C5F3CC05E2
:1025300015FB03F501EE105AB8EE411AB0EE410A50
:1025400022B1012A4DD0022A7DD169E06E4D283D8D
:102550002D68C5F340152DB36B4D283D2D68C5F38F
:10256000C1066A4D25FA06F4B4FBF0F501EE105AE7
:10257000F8EE411A9FED661A80EE012A624D103581
:102580002D68C5F3080501EE105AB8EE411A32EE77
:10259000011AB7EE002A31EE021A21EE811AF0EE8E
:1025A000410A1DE0594DB5FBF0F501EE105AF8EE69
:1025B000411A9FED571A80EE012A534D10352D68B0
:1025C000C5F3080501EE105AB8EE411A32EE011AB1
:1025D000B7EE002A31EE021A21EE811AF0EE410A1E
:1025E0005EE04C4DB5FBF0F501EE105AB8EE412A15
:1025F0009FED471AC0EE011A434D10352D68C5F303
:10260000080501EE105AB8EE411A31EE811AF7EEC4
:10261000001A31EE211A22EE011AF0EE410A3FE0D3
:102620003D4DB5FBF0F501EE105AF8EE411A9FED65
:10263000381A80EE012A344D10352D68C5F308058F
:1026400001EE105A00E00CE0B8EE411A32EE011A29
:10265000B7EE002A31EE021A21EE811AF0EE410A9D
:102660001EE02C4DB5FBF0F501EE105AB8EE412AF4
:102670009FED271AC0EE011A234D10352D68C5F3C2
:10268000080501EE105AB8EE411A31EE811AF7EE44
:10269000001A31EE211A22EE011AF0EE410A00BFB3
:1026A00000BF194D10352D68C5F346256D1C01EE90
:1026B000105AB8EE411AC0EE811ABCEEE11A81ED53
:1026C000001A114D10352D68C5F306456D1C01EE3D
:1026D000105AB8EE411AC0EE811ABCEEE11A81ED33
:1026E000011A094D10352D68C5F306656D1C01EE04
:1026F000105AB8EE411AC0EE811ABCEEE11A81ED13
:10270000021A70BD00000000284402580090D00357
:102710000000004600093D0040787D0170B501468B
:1027200000220120002300249FED811AB0EE410A0F
:102730009FED7F1AF0EE410A7E4D2D6805F00302F1
:102740007C4D2D68C5F305507A4D2D1D2D6805F47F
:102750008073784D1C352D68C5F3CC0515FB03F54A
:1027600001EE105AB8EE411AB0EE410A22B1012A28
:102770004DD0022A7DD169E06E4D283D2D68C5F30C
:1027800040152DB36B4D283D2D68C5F3C1066A4D2C
:1027900025FA06F4B4FBF0F501EE105AF8EE411AF2
:1027A0009FED661A80EE012A624D18352D68C5F33B
:1027B000080501EE105AB8EE411A32EE011AB7EED2
:1027C000002A31EE021A21EE811AF0EE410A1DE0D4
:1027D000594DB5FBF0F501EE105AF8EE411A9FED98
:1027E000571A80EE012A534D18352D68C5F3080598
:1027F00001EE105AB8EE411A32EE011AB7EE002A75
:1028000031EE021A21EE811AF0EE410A5EE04C4DE3
:10281000B5FBF0F501EE105AB8EE412A9FED471ACC
:10282000C0EE011A434D18352D68C5F3080501EEB9
:10283000105AB8EE411A31EE811AF7EE001A31EE55
:10284000211A22EE011AF0EE410A3FE03D4DB5FBA0
:10285000F0F501EE105AF8EE411A9FED381A80EEAD
:10286000012A344D18352D68C5F3080501EE105ABC
:1028700000E00CE0B8EE411A32EE011AB7EE002A81
:1028800031EE021A21EE811AF0EE410A1EE02C4DC3
:10289000B5FBF0F501EE105AB8EE412A9FED271A6C
:1028A000C0EE011A234D18352D68C5F3080501EE59
:1028B000105AB8EE411A31EE811AF7EE001A31EED5
:1028C000211A22EE011AF0EE410A00BF00BF194D95
:1028D00018352D68C5F346256D1C01EE105AB8EE6B
:1028E000411AC0EE811ABCEEE11A81ED001A114DB9
:1028F00018352D68C5F306456D1C01EE105AB8EE6B
:10290000411AC0EE811ABCEEE11A81ED011A094D9F
:1029100018352D68C5F306656D1C01EE105AB8EE2A
:10292000411AC0EE811ABCEEE11A81ED021A70BDA7
:1029300000000000284402580090D0030000004628
:1029400000093D0040787D012DE9F0410446002555
:102950000026206800F00060B0F1006F30D1606E9A
:1029600048B1B0F5801F0DD0B0F5001F10D0B0F504
:10297000401F15D113E0F948006840F40030F749D2
:1029800008600FE00221201D06F0D4F9054609E099
:10299000022104F1240006F065FA054602E001E098
:1029A000012500BF00BF55B9EC482430006820F471
:1029B0004010616E0843E9492431086000E02E436D
:1029C000208800F48070B0F5807F2DD1606D0528DF
:1029D0001AD2DFE800F0030A10171800DF48006879
:1029E00040F40030DD49086010E00021201D06F0B1
:1029F000A1F905460AE0002104F1240006F032FAAC
:102A0000054603E002E001E0012500BF00BF55B923
:102A1000D2482430006820F00700616D0843CF4998
:102A20002431086000E02E43208800F40070B0F5E7
:102A3000007F33D1A06D802817D003DC40B140283F
:102A40001CD10CE0C02817D0B0F5807F16D114E05F
:102A5000C248006840F40030C049086010E000211E
:102A6000201D06F067F905460AE0002104F1240064
:102A700006F0F8F9054603E002E001E0012500BF99
:102A800000BF55B9B5482430006820F4E070A16D4E
:102A90000843B2492431086000E02E43208800F446
:102AA0008060B0F5806F38D1D4F8A400B0F5800F05
:102AB00019D004DC50B1B0F5001F1DD10DE0B0F508
:102AC000C00F17D0B0F5000F16D114E0A34800686E
:102AD00040F40030A149086010E00021201D06F0FC
:102AE00029F905460AE0002104F1240006F0BAF9AC
:102AF000054603E002E001E0012500BF00BF5DB92B
:102B000096482C30006820F46000D4F8A4100843E4
:102B100092492C31086000E02E43208800F40060C8
:102B2000B0F5006F38D1D4F8A800B0F1007F19D00B
:102B300004DC50B1B0F1807F1DD10DE0B0F1407FD9
:102B400017D0B0F1806F16D114E08448006840F4CB
:102B500000308249086010E00021201D06F0EAF8EC
:102B600005460AE0002104F1240006F07BF9054641
:102B700003E002E001E0012500BF00BF5DB9774836
:102B80002C30006820F0E060D4F8A81008437349A6
:102B90002C31086000E02E43206800F00070B0F196
:102BA000007F27D1A06CA0B1102804D0202809D024
:102BB00030280FD10CE06948006840F400306749C4
:102BC000086009E00221201D06F0B4F8054603E084
:102BD00002E001E0012500BF00BF55B95F48203089
:102BE000006820F03000A16C08435C492031086087
:102BF00000E02E43208800F48050B0F5805F36D18D
:102C0000E06DB0F5005F19D004DC50B1B0F5805F25
:102C10001DD10DE0B0F5405F17D0B0F5804F16D153
:102C200014E04E48006840F400304C49086010E061
:102C30000021201D06F07EF805460AE0002104F17F
:102C4000240006F00FF9054603E002E001E001254B
:102C500000BF00BF55B941482430006820F4E0406F
:102C6000E16D08433D492431086000E02E4320888F
:102C700000F40050B0F5005F34D1206EB0F5403F55
:102C80001DD007DC68B1B0F5803F0BD0B0F5003F38
:102C900018D10DE0B0F5802F12D0B0F5A02F11D1D2
:102CA0000FE011E00121201D06F044F805460BE07D
:102CB000012104F1240006F0D5F8054604E003E004
:102CC00002E001E0012500BF00BF55B923482430D0
:102CD000006820F4E020216E084320492431086078
:102CE00000E02E43208800F48040B0F5804F38D1BA
:102CF000D4F8AC00B0F1405F1DD007DC68B1B0F192
:102D0000805F0BD0B0F1005F18D10DE0B0F1804FC3
:102D100012D0B0F1A04F11D10FE011E00121201D20
:102D200006F008F805460BE0012104F1240006F046
:102D300099F8054604E003E002E001E0012500BF48
:102D400000BF6DB905482C30006820F0E040D4F891
:102D5000AC10084301492C31086002E02C440258B1
:102D60002E43208800F40040B0F5004F26D1E06EDD
:102D700098B1B0F1805F03D0B0F1005F0ED106E0F2
:102D8000FA48006840F40030F849086008E0012182
:102D9000201D05F0CFFF054602E001E0012500BF40
:102DA00000BF55B9F1482430006820F04050E16E72
:102DB0000843EE492431086000E02E43206800F00B
:102DC0008070B0F1807F27D1606CA0B1012804D061
:102DD000022809D003280FD10CE0E448006840F431
:102DE0000030E249086009E00221201D05F0A2FF41
:102DF000054603E002E001E0012500BF00BF55B930
:102E0000DA482030006820F00300616C0843D7499D
:102E10002031086000E02E43206800F48000B0F507
:102E2000800F7DD1D248006840F48070D04908609E
:102E3000FEF71AF9074606E0FEF716F9C01B6428EC
:102E400001D9032505E0CA48006800F48070002815
:102E5000F2D000BF8DBBC5484430006800F440701C
:102E6000B4F8B01001F44071884214D0BF48443027
:102E7000006820F44078BD484430006840F4803059
:102E8000BA49443108600846006820F48030086080
:102E90000846C0F80080D4F8B000B0F5807F15D1A6
:102EA000FEF7E2F8074609E0FEF7DEF8C01B41F244
:102EB0008831884202D9032507E038E0AB48443026
:102EC0000068C0F340000028EED000BF4DBB00BF3B
:102ED000B4F8B00000F44070B0F5407F0ED1A348C4
:102EE0001C38006820F47C51A24AD4F8B00010408D
:102EF00041EA10109D491C39086007E09B481C38C6
:102F0000006820F47C5099491C3908609748443087
:102F10000068B4F8B010C1F30B010843934901E015
:102F200006E002E04431086002E02E4300E02E4358
:102F3000207800F0010068B3A06F182819D005DCD4
:102F400048B1082808D0102816D10BE0202811D04D
:102F5000282811D10FE011E00121201D05F0EAFE23
:102F600005460BE0012104F1240005F07BFF054636
:102F700004E003E002E001E0012500BF00BF55B915
:102F80007A482830006820F03800A16F084377495C
:102F90002831086000E02E43207800F0020002286B
:102FA00028D1606F062815D2DFE800F003040A116B
:102FB000121311E00121201D05F0BCFE05460BE0B7
:102FC000012104F1240005F04DFF054604E003E073
:102FD00002E001E0012500BF00BF55B96348283079
:102FE000006820F00700616F0843604928310860DD
:102FF00000E02E43207800F0040004282AD1D4F801
:103000009000062815D2DFE800F003040A1112131D
:1030100011E00121201D05F08DFE05460BE0012188
:1030200004F1240005F01EFF054604E003E002E081
:1030300001E0012500BF00BF5DB94C482C3000689D
:1030400020F00700D4F89010084348492C3108605C
:1030500000E02E43207800F02000202836D1D4F85C
:103060008C00B0F1405F1DD007DC68B1B0F1805F2B
:103070000BD0B0F1005F18D10DE0B0F1804F12D04D
:10308000B0F1A04F11D10FE011E00021201D05F09B
:1030900051FE05460BE0022104F1240005F0E2FE9A
:1030A000054604E003E002E001E0012500BF00BFA7
:1030B0005DB92E482830006820F0E040D4F88C102C
:1030C00008432A492831086000E02E43207800F0A8
:1030D0004000402836D1D4F89800B0F5406F1DD09C
:1030E00007DC68B1B0F5806F0BD0B0F5006F18D178
:1030F0000DE0B0F5805F12D0B0F5A05F11D10FE008
:1031000011E00021201D05F015FE05460BE002210F
:1031100004F1240005F0A6FE054604E003E002E009
:1031200001E0012500BF00BF5DB910482C300068E8
:1031300020F4E050D4F8981008430C492C31086072
:1031400000E02E43207800F0800080283BD1D4F8A6
:103150009C00B0F5C04F24D00EDCA0B1B0F5005FEC
:1031600012D0B0F5804F1FD114E000002C4402585B
:1031700000480258FFFCFF0FB0F5004F12D0B0F529
:10318000204F11D10FE011E00021201D05F0D2FDEC
:1031900005460BE0022104F1240005F063FE05461C
:1031A00004E003E002E001E0012500BF00BF4DB9EB
:1031B000B248006820F46040D4F89C100843AF493E
:1031C000086000E02E43207800F00800082816D19F
:1031D000D4F88000B0F5805F06D1022104F124000C
:1031E00005F040FE06430AE0A448001F006820F4F2
:1031F0004050D4F880100843A049091F0860207887
:1032000000F01000102814D1D4F89400B0F5807F9D
:1032100006D1022104F1240005F024FE064308E053
:103220009648006820F44070D4F8941008439349FD
:103230000860206800F40020B0F5002F26D1D4F8F3
:10324000A00030B1B0F5803F09D0B0F5003F0ED1FD
:103250000CE00021201D05F06DFD054609E002216E
:1032600004F1240005F0FEFD054602E001E0012521
:1032700000BF00BF4DB98148006820F44030D4F849
:10328000A01008437D49086000E02E43206800F448
:103290008020B0F5802F2DD1D4F88400B0F5801FA8
:1032A00006D0B0F5001F0CD0B0F5401F11D10FE0D3
:1032B00072482C38006840F4003070492C3908609E
:1032C00009E0012104F1240005F0CCFD054602E0EF
:1032D00001E0012500BF00BF5DB96848001F00681C
:1032E00020F44010D4F8841008436449091F086092
:1032F00000E02E43206800F48030B0F5803F24D1F8
:10330000E06C18B1B0F5803F0FD108E05B482C3875
:10331000006840F4003059492C39086007E0022168
:10332000201D05F007FD054601E0012500BF00BF97
:1033300055B952480C38006820F48030E16C0843DD
:103340004E490C39086000E02E43206800F0005020
:10335000B0F1005F05D1022104F1240005F082FDE7
:103360000643206800F40030B0F5003F27D1E06F3D
:10337000A0B1B0F5807F06D0B0F5007F0CD0B0F5DD
:10338000407F0CD109E03D482C38006840F4003003
:103390003A492C39086004E003E002E001E001252D
:1033A00000BF00BF55B93548001F006820F44070C9
:1033B000E16F08433149091F086000E02E4320688F
:1033C00000F48010B0F5801F09D12C48083800683F
:1033D00020F00040216F0843284908390860206820
:1033E00000F08050B0F1805F0AD12448483800686E
:1033F00020F48040D4F8B4100843204948390860CC
:10340000206800F40010B0F5001F09D11B480838EF
:10341000006820F08070A16E0843184908390860E0
:10342000206800F08040B0F1804F11D100BF1348F8
:103430004838006820F400401049483908600846C0
:103440000068D4F8B81008430C494839086000BF38
:10345000206800F00040B0F1004F09D107480C3857
:10346000006820F04050216D084304490C39086081
:1034700016B90020BDE8F0810120FBE7584402584E
:1034800070B504460D4600268D48006800F0070020
:10349000A8420ED28A48006820F0070028438849D5
:1034A00008600846006800F00700A84201D001202B
:1034B00070BD207800F00200022807D18148006822
:1034C00020F00F00E16808437E490860207800F092
:1034D0000100002851D07B48006820F47060A1688A
:1034E0000843784908606068022807D17548183891
:1034F0000068C0F34040F8B90120D9E760680328AC
:1035000007D1704818380068C0F34060A0B90120A6
:10351000CEE76068012807D16A4818380068C0F310
:10352000002048B90120C3E7664818380068C0F396
:10353000800008B90120BBE762480838006820F025
:103540000700616808435F4908390860FDF78CFD92
:1035500006466068022811D108E0FDF785FD801B52
:1035600041F28831884201D90320A1E75548083843
:10357000006800F038001028EFD13AE060680328B6
:1035800011D108E0FDF770FD801B41F288318842BF
:1035900001D903208CE74B480838006800F0380058
:1035A0001828EFD125E06068012811D108E0FDF767
:1035B0005BFD801B41F28831884201D9032077E707
:1035C00040480838006800F038000828EFD110E0C3
:1035D00008E0FDF749FD801B41F28831884201D99E
:1035E000032065E737480838006800F038000028F5
:1035F000EFD13348006800F00700A8420ED93048E8
:10360000006820F0070028432D490860084600683C
:1036100000F00700A84201D0012049E7207800F01F
:103620000400042807D12748006820F070002169B1
:10363000084324490860207800F00800082809D1D0
:103640002048001D006820F07000616908431D4992
:10365000091D0860207800F01000102809D11948D1
:10366000001D006820F4E060A16908431549091DA8
:103670000860207800F02000202809D11148083087
:10368000006820F07000E16908430E4908310860C5
:1036900000F066F80B49096801F470614FF480721C
:1036A00092FAA2F2B2FA82F2D140074A515CC840C3
:1036B000064908600020FDF7F7FC0020F8E600004E
:1036C000002000521844025824E30008000000249F
:1036D00010B5FEF7DBFE0949096801F00F01012270
:1036E00092FAA2F2B2FA82F2D140054A515CC84085
:1036F000044908600846006810BD000018440258DC
:1037000024E300080400002410B5FFF7E1FF074997
:10371000096801F07001102292FAA2F2B2FA82F264
:10372000D140034A515CC84010BD00001C440258FF
:1037300024E3000810B5FFF7CBFF0749096801F43F
:10374000E0614FF4807292FAA2F2B2FA82F2D140B2
:10375000024A515CC84010BD1C44025824E30008D2
:1037600070B5012500EE905A0022012100230024AB
:10377000DFED861AB0EE610ADFED841AB0EE611A51
:103780000020834D2D6805F0380535B1082D15D082
:10379000102D15D0182D7CD114E07D4D103D2D68D5
:1037A000C5F3401545B17A4D103D2D68C5F3C106EE
:1037B000784D25FA06F000E07648E5E07648E3E04B
:1037C0007648E1E0724D18352D6805F00302704D22
:1037D00018352D68C5F305116D4D1C352D6805F0A4
:1037E00001036B4D24352D68C5F3CC0515FB03F59E
:1037F00001EE905AF8EE611AB0EE610A22B1012A88
:103800004FD0022A7DD16BE0614D103D2D68C5F38C
:1038100040152DB35E4D103D2D68C5F3C1065D4DBD
:1038200025FA06F4B4FBF1F501EE905AB8EE612AE0
:10383000DFED5B1AC0EE212A554D20352D68C5F30A
:10384000080501EE905AF8EE611A72EEA11AF7EE31
:10385000002A71EEA21A62EE211AB0EE611A1FE080
:103860004C4DB5FBF1F501EE905AB8EE612ADFED53
:103870004C1AC0EE212A464D20352D68C5F30805A7
:1038800001EE905AF8EE611A72EEA11AF7EE002AD4
:1038900000E077E071EEA21A62EE211AB0EE611A32
:1038A0005EE03D4DB5FBF1F501EE905AB8EE612AB0
:1038B000DFED3B1AC0EE212A354D20352D68C5F3CA
:1038C000080501EE905AF8EE611A72EEA11AF7EEB1
:1038D000002A71EEA21A62EE211AB0EE611A3FE0E0
:1038E0002E4DB5FBF1F501EE905AB8EE612ADFEDF1
:1038F0002C1AC0EE212A264D20352D68C5F3080567
:1039000000E00EE001EE905AF8EE611A72EEA11A94
:10391000F7EE002A71EEA21A62EE211AB0EE611AD9
:103920001EE01D4DB5FBF1F501EE905AF8EE612A4F
:10393000DFED1B1A80EE212A154D20352D68C5F3C9
:10394000080501EE905AF8EE611A72EE211AB7EEF0
:10395000002A71EE821A62EEA11AB0EE611A00BF5F
:1039600000BF0B4D20352D68C5F346256D1C00EEBC
:10397000905AF8EE601A81EE212AFCEEC21A11EE7E
:10398000900A01E0044800BF00BF70BD00000000C5
:10399000104402580090D00300093D0040787D019A
:1039A0000000004670B504460025207800F00100B4
:1039B000002872D0F948006800F0380010280CD0B8
:1039C000F648006800F03800182812D1F348183083
:1039D000006800F0030002280BD1F048103800689E
:1039E000C0F3404000286DD0606800286AD10120F3
:1039F00070BD00BF6068B0F5803F08D1E74810385F
:103A0000006840F48030E549103908602EE06068B5
:103A100068B9E2481038006820F48030DF49103976
:103A200008600846006820F4802008601EE0606896
:103A3000B0F5A02F0DD1D9481038006840F480208F
:103A4000D649103908600846006840F480300860A4
:103A50000CE0D2481038006820F48030CF4910398B
:103A600008600846006820F48020086000BF606895
:103A7000A0B1FDF7F9FA054608E0FDF7F5FA401B9D
:103A800041F28831884201D90320B1E7C348103898
:103A90000068C0F340400028EFD013E0FDF7E4FADF
:103AA000054608E0FDF7E0FA401B41F28831884204
:103AB00001D903209CE7B94810380068C0F34040A2
:103AC0000028EFD1207800F00200022847D1B34847
:103AD000006800F0380058B1B048006800F03800C5
:103AE00018283ED1AD481830006800F00300B8BB7C
:103AF000AA4810380068C0F3800018B1E06808B91F
:103B0000012075E7A5481038006820F01900E16829
:103B10000843A24910390860FDF7A6FA054606E0F9
:103B2000FDF7A2FA401B022801D9032060E79B4859
:103B300010380068C0F380000028F1D097480C3896
:103B4000006820F47C304FF47C3292FAA2F2B2FA90
:103B500082F221699140084390490C3908604AE09B
:103B6000FFE7E06868B38D481038006820F019005E
:103B7000E1680843894910390860FDF775FA054680
:103B800006E0FDF771FA401B022801D903202FE758
:103B9000824810380068C0F380000028F1D07F48C8
:103BA0000C38006820F47C304FF47C3292FAA2F298
:103BB000B2FA82F221699140084378490C390860D1
:103BC00019E076481038006820F001007349103978
:103BD0000860FDF749FA054606E0FDF745FA401B87
:103BE000022801D9032003E76C4810380068C0F3AD
:103BF00080000028F1D1207800F01000102877D143
:103C00006648006800F0380008280CD06348006857
:103C100000F03800182823D160481830006800F000
:103C2000030001281CD15D4810380068C0F3002053
:103C300020B1E069802801D00120D9E657480C382E
:103C4000006820F0F8404FF0F84292FAA2F2B2FA7F
:103C500082F2216A9140084350490C39086047E0DC
:103C6000E06958B34D481038006840F080004B4977
:103C700010390860FDF7F8F9054606E0FDF7F4F99C
:103C8000401B022801D90320B2E6444810380068DE
:103C9000C0F300200028F1D040480C38006820F024
:103CA000F8404FF0F84292FAA2F2B2FA82F2216A98
:103CB0009140084339490C39086019E037481038F9
:103CC000006820F08000354910390860FDF7CCF914
:103CD000054606E0FDF7C8F9401B022801D903207C
:103CE00086E62E4810380068C0F300200028F1D185
:103CF000207800F00800082836D16069D0B1274844
:103D00006430006840F00100244964310860FDF728
:103D1000ABF9054606E0FDF7A7F9401B022801D9DB
:103D2000032065E61D4864300068C0F340000028A9
:103D3000F1D019E019486430006820F001001749FB
:103D400064310860FDF790F9054606E0FDF78CF94F
:103D5000401B022801D903204AE61048643000685D
:103D6000C0F340000028F1D1207800F02000202886
:103D700034D1A069D8B109481038006840F48050A7
:103D8000064910390860FDF76FF9054608E0FDF7B0
:103D90006BF9401B022803D9032029E6104402587E
:103DA000AF480068C0F340300028F0D016E0AC48BF
:103DB000006820F48050AA490860FDF755F90546CF
:103DC00006E0FDF751F9401B022801D903200FE658
:103DD000A3480068C0F340300028F2D1207800F0FA
:103DE000040004287DD19F48006840F480709D49FC
:103DF0000860FDF739F9054606E0FDF735F9401B87
:103E0000642801D90320F3E59648006800F4807027
:103E10000028F2D000BFA068012808D19048703077
:103E2000006840F001008E49703108602DE0A06804
:103E300068B98B487030006820F001008849703103
:103E400008600846006820F0040008601DE0A068D3
:103E500005280DD182487030006840F00400804988
:103E6000703108600846006840F0010008600CE00E
:103E70007B487030006820F001007949703108609B
:103E80000846006820F00400086000BFA068A0B1E8
:103E9000FDF7EAF8054608E0FDF7E6F8401B41F2B9
:103EA0008831884201D90320A2E56D48703000684E
:103EB000C0F340000028EFD013E0FDF7D5F8054629
:103EC00008E0FDF7D1F8401B41F28831884201D962
:103ED00003208DE5624870300068C0F34000002880
:103EE000EFD1606A00287CD05D481030006800F097
:103EF0003800182876D0606A022874D158480068C3
:103F000020F0807056490860FDF7AEF8054606E0DF
:103F1000FDF7AAF8401B022801D9032068E55048A4
:103F20000068C0F340600028F2D100BFD4E90A1055
:103F300041EA00104A492831096840F2F3329143BE
:103F40000843474928310860208E401EC0F308000E
:103F5000616B491E4FF47E4202EA41210843218FE2
:103F6000491ED20102EA014108433C21095D491E74
:103F7000120202EA0161084339493031086000BF8A
:103F8000081D00684FF6F87188434FF6F87292FAF0
:103F9000A2F2B2FA82F2A16C914008433049343166
:103FA00008602F482C30006820F00C00216C08437A
:103FB0002B492C3108600846006820F00200616C33
:103FC000084327492C3108600846006840F48030D7
:103FD00008600846006840F4003008600846006841
:103FE00002E03BE038E01FE040F480200860084633
:103FF000006840F0010008601948006840F08070D7
:1040000017490860FDF730F8054606E0FDF72CF883
:10401000401B022801D90320EAE411480068C0F3DC
:1040200040600028F2D019E00D48006820F0807050
:104030000B490860FDF718F8054606E0FDF714F88F
:10404000401B022801D90320D2E405480068C0F3D0
:1040500040600028F2D101E00120C9E40020C7E45B
:10406000004402580048025870B504460D460CB989
:10407000012070BD94F82C0028B9002084F82D0090
:10408000204600F019F8022084F82C00211D206839
:10409000FCF761FD2946D4E90002FCF7B1FD0548B3
:1040A000006840F0004003490860012084F82C00BB
:1040B0000020DEE70040005210B586B0044600BF85
:1040C0005A48006840F002005849086008460068F5
:1040D00000F00200009000BF00BF00BF534820382E
:1040E000006840F480505149203908600846006853
:1040F00000F48050009000BF00BF00BF4B48143850
:10410000006840F004004949143908600846006816
:1041100000F00400009000BF00BF00BF0846006828
:1041200040F0080008600846006800F008000090B1
:1041300000BF00BF00BF0846006840F010000860E4
:104140000846006800F01000009000BF00BF00BFEC
:104150000846006840F0200008600846006800F04B
:104160002000009000BF00BF00BF0846006840F07C
:10417000400008600846006800F04000009000BF62
:1041800000BF00BF0846006840F080000860084695
:10419000006800F08000009000BF00BF00BF08462C
:1041A000006840F4807008600846006800F4807081
:1041B000009000BF00BF0D2001900220029001205E
:1041C0000390032004900C20059001A91848FCF7E7
:1041D00013FE4CF20370019001A91648FCF70CFE87
:1041E0004FF68370019001A91348FCF705FE4FF6C6
:1041F0003F00019001A91148FCF7FEFD48F237107D
:10420000019001A90E48FCF7F7FD4FF47F400190A3
:1042100001A90C48FCF7F0FD40F2FF60019001A9F4
:104220000948FCF7E9FD06B010BD0000F44402584F
:1042300000080258000C02580010025800140258DE
:1042400000180258001C02580020025870B504469D
:104250000D4694F82C00022800D170BD022084F88D
:104260002C0029462068FCF7B0FC012084F82C00C3
:104270000020F2E770B504460D46164694F82C006F
:10428000022800D170BD022084F82C003246294655
:104290002068FCF7A1FC2868022803D1052084F8D7
:1042A0002C0002E0012084F82C000020EAE7000046
:1042B00070B50446002500260CB9012070BD606A67
:1042C00000B900BFA06AB0F5800F00D100BF8E49D1
:1042D000206888420CD08D492068884208D08C49DB
:1042E0002068884204D0E0680F2801D90120E5E762
:1042F000204605F067F8064683492068884209D0C1
:1043000082492068884205D081492068884201D0CE
:10431000082E0DD87C492068884207D07B49206848
:10432000884203D07A492068884203D1102E01D9EF
:104330000120C3E7A06AB0F5800F1DD17249206843
:1043400088420DD071492068884209D070492068A0
:10435000884205D0206BB0F5702F01D90120ADE760
:10436000206B10B9A089050400E0256BE068B0EB74
:10437000154F01D90120A1E794F8810028B9002048
:1043800084F88000204600F0C5F8022084F88100FF
:104390002068006820F0010021680860A069B0F181
:1043A000806F0BD16068B0F5800F07D1A06B28B982
:1043B0002068006840F4805021680860A16AE069C4
:1043C00008432843E16B0843E1680843216888609B
:1043D000616A606B0843A16B0843A16908432169C6
:1043E000084361690843216A084361680843E16C36
:1043F0000843A1680843A16C0843A16D08432168E4
:10440000C860A06AB0F5800F4DD1206C012806D19C
:104410002068006840F400402168086005E02068DA
:10442000006820F4004021680860606C012806D113
:104430002068006840F480402168086005E020683A
:10444000006820F48040216808602F492068884275
:104450000AD02E492068884206D02D49206888421B
:1044600002D0B5F5702F0ED027492068884207D0BA
:1044700026492068884203D025492068884209D10E
:10448000B5F5F81F06D12068006840F40050216897
:10449000086005E02068006820F40050216808608A
:1044A0002168E06A0864606888B9A06A38B9206841
:1044B000806820F4C05040F4006021688860206863
:1044C000806820F4C06040F48060216888602068C3
:1044D000006D20F0010021680865606800F480002C
:1044E000B0F5800F07D12068C06820F00040616DF2
:1044F00008432168C8600020C4F88400012084F8C3
:1045000081000020DAE60000003001400038004061
:10451000003C004010B5B6B0044600BF1A48006821
:1045200040F00200184908600846006800F00200E8
:10453000019000BF00BF00BF13480830006840F47E
:1045400080401149083108600846006800F4804046
:10455000019000BF00BF4FF48050029000201990DE
:1045600002A8FEF7F1F94FF460403190022032903A
:1045700001203390032034900520359031A9034861
:10458000FCF73AFC36B010BDE04402580004025873
:104590002DE9F84F0446884691461D460A9E00279D
:1045A000BA4600BF94F88000012802D10220BDE87D
:1045B000F88F012084F8800000BFFCF755FD074606
:1045C00094F88100012812D06068B0F5800F05D101
:1045D000A06818B994F88100042808D04FF0020AA6
:1045E00000BF002084F8800000BF5046DFE7B8F12C
:1045F000000F03D0B9F1000F00D045B94FF0010A08
:1046000000BF002084F8800000BF5046CFE794F838
:104610008100042802D0052084F881000020C4F81D
:104620008400C4F86490A4F86A50A4F86850C4F8F0
:104630005C80A4F86250A4F860502067606720682E
:1046400040686FF30F0028432168486020680068C5
:1046500040F00100216808606068B0F5800F05D166
:104660002068006840F4007021680860E0680F2846
:104670004CD942E0B4F8620088B12068406900F08B
:10468000020002280BD1E06D006821680862E06D2D
:10469000001DE065B4F86200401EA4F86200B4F8A2
:1046A0006A0088B12068406948F20801084058B1A2
:1046B0002068006B616E0860606E001D6066B4F873
:1046C0006A00401EA4F86A00701CB0B1FCF7CCFC74
:1046D000C01BB04211D3204604F0F6FD00BF0020FD
:1046E00084F8800000BFD4F8840040F48070C4F8DF
:1046F0008400012084F8810059E7B4F862000028A2
:10470000B8D1B4F86A000028B4D10FE1E0680728F6
:1047100071D966E0B4F8620020B32068406900F007
:10472000020002281ED1B4F8620001280ED9E06B05
:1047300060B1E06D006821680862E06D001DE06511
:10474000B4F86200801EA4F862000BE0E06D0088FF
:1047500021680884E06D801CE065B4F86200401EAA
:10476000A4F86200B4F86A0010B32068406900F44D
:104770006040E8B12068406900F4004060B1206802
:10478000006B616E0860606E001D6066B4F86A00C0
:10479000801EA4F86A000BE02068008E616E08801D
:1047A000606E801C6066B4F86A00401EA4F86A005F
:1047B000701CB0B1FCF758FCC01BB04211D32046AE
:1047C00004F082FD00BF002084F8800000BFD4F810
:1047D000840040F48070C4F88400012084F88100D3
:1047E000E5E6B4F86200002894D1B4F86A00002825
:1047F00090D19BE0FFE790E0B4F8620058B32068E6
:10480000406900F00200022833D1B4F862000328A6
:104810000FD9E06B40280CD9E06D00682168086270
:10482000E06D001DE065B4F86200001FA4F86200AE
:104830001FE0B4F8620001280ED9E06B60B1E06DB2
:10484000008821680884E06D801CE065B4F862008F
:10485000801EA4F862000CE0E06D0078216881F809
:104860002000E06D401CE065B4F86200401EA4F832
:104870006200B4F86A0048B32068406900F4604000
:1048800020B32068406900F4004060B12068006BEC
:10489000616E0860606E001D6066B4F86A00001FFB
:1048A000A4F86A0020E02068406900F4C040B0F538
:1048B000005F0CD92068008E616E0880606E801CDD
:1048C0006066B4F86A00801EA4F86A000CE02068F4
:1048D00090F83000616E0870606E401C6066B4F83D
:1048E0006A00401EA4F86A00701CB0B1FCF7BCFB63
:1048F000C01BB04211D3204604F0E6FC00BF0020EC
:1049000084F8800000BFD4F8840040F48070C4F8BC
:104910008400012084F8810049E6B4F86200002890
:104920007FF46AAFB4F86A000028F9D13B46002250
:1049300008212046009604F052FD28B1D4F88400E6
:1049400040F02000C4F88400204604F0BDFC00BF05
:10495000002084F8800000BF012084F88100D4F892
:10496000840008B1012022E6002020E670B504464C
:104970000E4615460CB9012070BD94F8450028B9C3
:10498000002084F84400204600F024F804F10801D7
:104990002068FCF771F83146A2682068FCF7ACF893
:1049A0002946E36AD4E90102FCF742F8A1682068CD
:1049B00050F8210040F00100A268216841F822006F
:1049C0000348006840F00040014908600020D3E738
:1049D0000040005210B586B0044600BF2048006871
:1049E00040F480501E4908600846006800F480507A
:1049F000009000BF00BF00BF19480C30006840F0B5
:104A0000080017490C3108600846006800F00800EB
:104A1000009000BF00BF00BF0846006840F01000D3
:104A200008600846006800F01000009000BF00BF5A
:104A30004EF2B370019002200290012003900320F7
:104A400004900C20059001A90648FCF7D5F94FF613
:104A50008070019001A90448FCF7CEF906B010BDA2
:104A6000D4440258000C025800100258042808D1FF
:104A70004FF0E021096941F004014FF0E02211619B
:104A800007E04FF0E021096921F004014FF0E02236
:104A90001161704770B504462546681EB0F1807FED
:104AA00001D301200FE0681E4FF0E02148610F2183
:104AB0004FF0FF3007F004FC00204FF0E021886148
:104AC00007200861002070BD10B504460CB9012014
:104AD00010BD94F83D0028B9002084F83C00204621
:104AE00000F00CF8022084F83D00211D206804F03D
:104AF00087FD012084F83D000020E9E7704701466A
:104B00000868C06840F001000A68D0600868008842
:104B100040F001000A68108000207047704770471D
:104B200001460022002391F8792091F87A3042EA78
:104B3000030070472DE9F04104462068C5692068EC
:104B400007682068866805F00F08B8F1000F0DD1DE
:104B500005F0200050B107F0200010B906F0805099
:104B600020B1204604F0BBFEBDE8F081B8F1000F93
:104B700072D05D48304018B907F4907000287AD0A0
:104B800005F0010048B107F4807030B101202168C0
:104B90000862E06F40F00100E06705F0020048B1F4
:104BA00006F0010030B1022021680862E06F40F099
:104BB0000400E06705F0040048B106F0010030B1E0
:104BC000042021680862E06F40F00200E06705F011
:104BD000080078B107F0200028B906F0805010B91D
:104BE00006F0010030B1082021680862E06F40F053
:104BF0000800E067E06F70B305F0200040B107F0F7
:104C0000200010B906F0805010B1204604F067FE75
:104C1000E06F00F0080020B92068806800F04000D4
:104C200018B3204604F03BFE2068806800F0400086
:104C3000B8B12068806820F0400021688860606F0B
:104C400058B12A48616F0865606FFCF73BF810B1F6
:104C5000606F016D88470DE00DE02046FFF75FFFB4
:104C600008E02046FFF75BFF04E02046FFF757FF10
:104C70000020E06778E705F4801078B106F4800042
:104C800060B14FF4801021680862202084F8790018
:104C900084F87A002046FFF741FF65E705F08000C1
:104CA00048B107F0800010B906F4000018B12046A2
:104CB00005F02CFB58E705F0400030B107F040004C
:104CC00018B1204604F0FBFD4EE705F4000040B1AA
:104CD00007F0804028B12068006820F080402168FB
:104CE000086000BF40E7000001000010879800083E
:104CF00010B504460CB9012010BDA06900B100E058
:104D000000BF94F8790028B9002084F87800204684
:104D100000F02AF8242084F879002068006820F048
:104D2000010021680860204604F01EFE012800D121
:104D3000E2E7606B10B1204604F0F6FC20684068A2
:104D400020F49040216848602068806820F02A00A4
:104D5000216888602068006840F0010021680860D0
:104D6000204604F056FDC7E710B586B00446214939
:104D7000206888423BD100BF1F48006840F0010016
:104D80001D4908600846006800F00100009000BF5F
:104D900000BF00BF18481030006840F010001649EE
:104DA000103108600846006800F01000009000BF55
:104DB00000BF4FF400700190022002900120039088
:104DC000022004900720059001A90C48FCF714F874
:104DD0004FF48060019001A90848FCF70DF82520E8
:104DE000FCF795FB032211462520FCF7A0FB06B03B
:104DF00010BD000000100140E044025800000258BD
:104E000010B5034693F87A00202867D101B10AB99A
:104E1000012010BD00BF93F87800012801D10220C5
:104E2000F7E7012083F8780000BF5966A3F86820EF
:104E3000A3F86A2000BF9868B0F5805F0AD11869AE
:104E400020B940F2FF10A3F86C001CE0FF20A3F88B
:104E50006C0018E0986848B9186918B9FF20A3F8E1
:104E60006C0010E07F20A3F86C000CE09868B0F1B3
:104E7000805F08D1186918B97F20A3F86C0002E0A0
:104E80003F20A3F86C0000BF0020D867222083F8E1
:104E90007A0000BF002083F8780000BF186880689F
:104EA00040F001001C68A0601868006800F0005025
:104EB00060B11868006840F480701C682060186851
:104EC000806840F080501C68A06005E018680068A9
:104ED00040F490701C68206000209AE7022098E758
:104EE0001D4A0168914236D11C49098801F40041EC
:104EF00089BB1A49098801F4804171B118490978C0
:104F00000A2903D00021154A118024E01349098899
:104F100041F40041114A11801DE0114909780D2921
:104F200006D10E49098841F480410C4A118012E0F3
:104F30000B490978094A1288C2F30D02094B9954AA
:104F400006490988491C054A118011460988C72964
:104F500001DD002111807047001001401000002485
:104F6000120000241C050024704700BFFEE700006B
:104F700010B5002210211248FCF770F810480068A4
:104F800020F440600E4908600846006840F48060E4
:104F90000860002220210A48FCF760F8022007F090
:104FA00027FE012210210648FCF758F8022007F0DE
:104FB0001FFE002210210248FCF750F810BD00002F
:104FC000001C025800B587B000BF1248006840F0CE
:104FD0008000104908600846006800F080000190D9
:104FE00000BF00BF302002900120039004900320F6
:104FF000059002A90848FBF7FFFE01222021064880
:10500000FCF72CF8012210210348FCF727F807B021
:1050100000BD0000E0440258001C025810B50022F8
:1050200010211248FCF71AF81048006820F440607C
:105030000E4908600846006840F48060086001225C
:1050400020210A48FCF70AF8022007F0D1FD0122CE
:1050500010210648FCF702F8022007F0C9FD0022E3
:1050600010210248FBF7FAFF10BD0000001C025897
:1050700070B5054600241848006820F440601649C1
:10508000086008460068086000261AE00022102127
:105090001148FBF7E3FF022007F0AAFD01221021CF
:1050A0000D48FBF7DBFF6006040E20210A48FBF7E2
:1050B000C9FF08B1601CC4B2012007F099FD701C43
:1050C000C6B2082EE2DB15B9FFF7A8FF01E0FFF733
:1050D0004FFF204670BD0000001C025870B504460A
:1050E0001C48006820F440601A49086008460068BF
:1050F00040F480600860002210211648FBF7AEFFE4
:10510000002523E0E00928B1012220211148FBF706
:10511000A5FF04E0002220210E48FBF79FFF600658
:10512000040E022007F064FD012210210948FBF75C
:1051300095FF022007F05CFD002210210548FBF7D7
:105140008DFF022007F054FD681CC5B2082DD9DB85
:1051500070BD0000001C025810B51348006820F410
:105160004060114908600846006840F480600860AB
:10517000012220210C48FBF771FF012210210A486F
:10518000FBF76CFF042007F033FD002220210648C6
:10519000FBF764FF042007F02BFD002210210248DA
:1051A000FBF75CFF10BD0000001C025810B513484F
:1051B000006820F44060114908600846006840F427
:1051C00080600860002210210C48FBF747FF002296
:1051D00020210A48FBF742FF042007F009FD0122C5
:1051E00010210648FBF73AFF012220210348FBF774
:1051F00035FF042007F0FCFC10BD0000001C025825
:1052000010B500241748006820F440601549086074
:10521000084600680860012220211248FBF71EFFA3
:10522000012007F0E5FC012210210E48FBF716FFD4
:10523000012007F0DDFC07E0601CC4B2FA2C03DD9E
:10524000FFF7B4FF012010BD20210648FBF7FAFE4E
:105250000028F1D1002210210248FBF7FFFE0020B8
:10526000F1E70000001C025830B50B46002100BFDA
:1052700016E00A24B4EB107F05D9302404EB107437
:1052800003F8114005E0412404EB10740A3C03F8D4
:105290001140000100254C00641C1D554C1CE1B25E
:1052A0009142E6DB30BD000000B587B000BF244866
:1052B000006840F00100224908600846006800F0DC
:1052C0000100019000BF00BF00BF0846006840F029
:1052D000040008600846006800F00400019000BF68
:1052E00000BF00BF0846006840F080000860084624
:1052F000006800F08000019000BF00BF0120029014
:1053000000200390022004900320059002A90D487C
:10531000FBF772FD4FF40050029000200390012033
:1053200004900320059002A90748FBF765FD0C20B7
:10533000029002A90548FBF75FFD07B000BD000021
:10534000E04402580000025800080258001C0258AD
:1053500070B5044600260D4805880D48006818B150
:10536000204602F0F5FE0FE0084840884543002142
:10537000084602F029FD02F0ADFE002602E00549D4
:105380000C80761CAE42FAD370BD0000E406002407
:10539000FC0700240000086010B504465C488471D6
:1053A0005C48006850B1204602F0FCFE5948C08AB3
:1053B000574908805748008B488010BD002C51D1B8
:1053C000F020534908804FF4A07048800846808838
:1053D00049F24131884205D04D48808845F210316C
:1053E000884214D12C204A4908812A2048812B2048
:1053F00088810846808845F21031884206D14FF4F2
:10540000A070434908804FF4F07048807BE040482A
:10541000808845F21051884210D14FF430503C49F9
:1054200008814FF4285048814FF42C5088814FF464
:10543000F07008804FF44870488064E034488088F9
:1054400041F6631188425ED12C20314908812B201E
:1054500048812A2088814FF4F07008804FF448700A
:10546000488050E04FF4A07029490880F02048801F
:105470000846808849F24131884205D02448808816
:1054800045F21031884207D12C20214908812A2079
:1054900048812B20888129E01D48808845F21051E1
:1054A000884210D14FF43050194908814FF42850E8
:1054B00048814FF42C5088814FF4487008804FF495
:1054C000F070488012E01248808841F663118842EB
:1054D0000CD12C200E4908812A2048812B2088815C
:1054E0004FF4487008804FF4F07048800848808876
:1054F00045F21031884206D14FF4F070044908801B
:105500004FF4A0704880002002F024FB00BF54E755
:10551000E4060024FC07002470B504460D46164638
:105520004348006828B132462946204602F050FE22
:1055300070BD4048808849F24131884205D03D48DD
:10554000808845F21031884214D13A49488902F0E6
:10555000B5FD201202F0A6FDE0B202F0A3FD354930
:10556000888902F0ABFD281202F09CFDE8B202F03F
:1055700099FD54E02F48808845F21051884220D18F
:105580002C49488902F09AFD201202F08BFD29492E
:105590004989491C88B202F091FDE0B202F082FD17
:1055A0002449888902F08AFD281202F07BFD2149F6
:1055B0008989491C88B202F081FDE8B202F072FDCF
:1055C0002DE01C48808841F66311884227D1194894
:1055D000807920B917480088401E001B84B2154905
:1055E000488902F06BFD201202F05CFDE0B202F08F
:1055F00059FD201202F056FDE0B202F053FD0D49B4
:10560000888902F05BFD281202F04CFDE8B202F03E
:1056100049FD281202F046FDE8B202F043FD0548BC
:10562000008905490880891C0E8000BF80E70000C2
:10563000FC070024E4060024FEFF076000B595B0D7
:1056400003F0E6F8FE4988800846808818B102F029
:105650008BFE02F0E4B900BFFA48006840F0020097
:10566000F84908600846006800F00200019000BF99
:1056700000BF202010900120119012900320139061
:1056800010A9F148FBF7B8FB02F00AFAEF48F0491D
:105690000860F0484860002088600021EC48C16044
:1056A00001611021416100218161C16101624FF4FA
:1056B00080514162002181624FF48041C16200212A
:1056C000016341634FF48011816311200990002030
:1056D0000A9055200B9000200F901520029000207A
:1056E0000390152004900020089002AA09A9D84828
:1056F000FFF73CF9322007F06FFAD32002F0DEFC0E
:1057000002F0F6F9CE49888002F0F2F9CC4988809F
:1057100002F0EEF9CA498880084680884FF6FF718A
:1057200001EA0020C649888002F0E2F9C44989886C
:105730000843C34988800846808849F2413188423D
:1057400078D0D42002F0BAFC02F0D2F9BC498880AB
:1057500002F0CEF9BA49888002F0CAF9B8498880C7
:10576000084680884FF6FF7101EA0020B44988801E
:1057700002F0BEF9B24989880843B14988800846D9
:10578000808845F21031884254D04FF45A4002F0DC
:1057900095FC02F0ADF9AA4988804FF45B4002F015
:1057A0008DFC02F0A5F9A6498880084680884FF64E
:1057B000FF7101EA0020A24988804FF45C4002F0AA
:1057C0007DFC02F095F99E49898808439C498880B0
:1057D00008468088B0F5004F02D145F2105088800D
:1057E0009748808845F21051884223D0A12002F0CA
:1057F00065FC02F07DF99249888002F079F99049C0
:105800008880084680884FF6FF7101EA00208C49A5
:10581000888002F06DF98A49898808438849888020
:105820000846808845F26171884203D141F66310D1
:10583000834988808248808849F2413188427CD1FE
:10584000CF2002F03BFC002002F02CFCC12002F033
:1058500029FC302002F026FCED2002F02FFC642011
:1058600002F020FC032002F01DFC122002F01AFCC2
:10587000812002F017FCE82002F020FC852002F0D5
:1058800011FC102002F00EFC7A2002F00BFCCB2061
:1058900002F014FC392002F005FC2C2002F002FC7E
:1058A000002002F0FFFB342002F0FCFB022002F09B
:1058B000F9FBF72002F002FC202002F0F3FBEA20C3
:1058C00002F0FCFB002002F0EDFB002002F0EAFBFE
:1058D000C02002F0F3FB1B2002F0E4FBC12002F029
:1058E000EDFB012002F0DEFBC52002F0E7FB3020DB
:1058F00002F0D8FB302002F0D5FBC72002F0DEFB1F
:10590000B72002F0CFFB362002F0D8FB482002F08F
:10591000C9FB3A2002F0D2FB552002F0C3FBB120B4
:1059200002F0CCFB002002F0BDFB1A2002F0BAFB13
:10593000B62002F0C3FB0A2000E0A5E002F0B2FBB3
:10594000A22002F0AFFBF22002F0B8FB002002F030
:10595000A9FB262002F0B2FB012002F0A3FBE0200D
:1059600002F0ACFB0F2002F09DFB2A2002F09AFB14
:10597000282002F097FB082002F094FB0E2002F092
:1059800091FB082002F08EFB542002F08BFBA92033
:1059900002F088FB432002F085FB0A2002F082FB24
:1059A0000F2002F07FFB002002F07CFB002002F0C1
:1059B00079FB002002F076FB002002F073FBE1206F
:1059C00002F07CFB002002F06DFB152002F06AFB68
:1059D000172002F067FB072002F064FB112002F0A1
:1059E00061FB062002F05EFB2B2002F05BFB5620E1
:1059F00002F058FB3C2002F055FB052002F052FB60
:105A0000102002F04FFB0F2002F04CFB3F2002F071
:105A100049FB3F2002F046FB0F2002F043FB2B2006
:105A200002F04CFB002002F03DFB002002F03AFBAC
:105A3000012002F037FB3F2002F034FB2A200BE06C
:105A4000E4060024E04402580004025800400052DA
:105A5000980600240441005202F030FB002002F0BE
:105A600021FB002002F01EFB002002F01BFBEF20B8
:105A700002F018FB112002F021FB782007F0ACF8AF
:105A8000292002F01BFBE4E5FE48808845F2103136
:105A9000884240F07C87ED2002F010FB012002F0EC
:105AA00001FBFE2002F0FEFAEE2002F007FBDE20F2
:105AB00002F0F8FA212002F0F5FAF12002F0FEFAE5
:105AC000012002F0EFFADF2002F0F8FA102002F0D5
:105AD000E9FAC42002F0F2FA8F2002F0E3FAC620BD
:105AE00002F0ECFA002002F0DDFAE22002F0DAFA2D
:105AF000E22002F0D7FAE22002F0D4FABF2002F04E
:105B0000DDFAAA2002F0CEFAB02002F0D7FA0D207A
:105B100002F0C8FA002002F0C5FA0D2002F0C2FA25
:105B2000002002F0BFFA112002F0BCFA002002F0BF
:105B3000B9FA192002F0B6FA002002F0B3FA2120D7
:105B400002F0B0FA002002F0ADFA2D2002F0AAFA1D
:105B5000002002F0A7FA3D2002F0A4FA002002F093
:105B6000A1FA5D2002F09EFA002002F09BFA5D206F
:105B700002F098FA002002F095FAB12002F09EFAA5
:105B8000802002F08FFA002002F08CFA8B2002F0C5
:105B900089FA002002F086FA962002F083FA0020AB
:105BA00002F080FAB22002F089FA002002F07AFABC
:105BB000002002F077FA022002F074FA002002F0CE
:105BC00071FA032002F06EFA002002F06BFAB320A3
:105BD00002F074FA002002F065FA002002F062FA86
:105BE000002002F05FFA002002F05CFA002002F0D0
:105BF00059FA002002F056FA002002F053FA002071
:105C000002F050FA002002F04DFA002002F04AFAA9
:105C1000002002F047FA002002F044FA002002F0CF
:105C200041FA002002F03EFA002002F03BFA002088
:105C300002F038FA002002F035FA002002F032FAC1
:105C4000002002F02FFA002002F02CFA002002F0CF
:105C500029FA002002F026FA002002F023FA0020A0
:105C600002F020FAB42002F029FA8B2002F01AFA8E
:105C7000002002F017FA962002F014FA002002F039
:105C800011FAA12002F00EFA002002F00BFAB52062
:105C900002F014FA022002F005FA002002F002FAE3
:105CA000032002F0FFF9002002F0FCF9042002F0CA
:105CB000F9F9002002F0F6F9B62002F0FFF9002011
:105CC00002F0F0F9002002F0EDF9B72002F0F6F949
:105CD000002002F0E7F9002002F0E4F93F2002F092
:105CE000E1F9002002F0DEF95E2002F0DBF900208D
:105CF00002F0D8F9642002F0D5F9002002F0D2F9C0
:105D00008C2002F0CFF9002002F0CCF9AC2002F098
:105D1000C9F9002002F0C6F9DC2002F0C3F9002026
:105D200002F0C0F9702002F0BDF9002002F0BAF9CB
:105D3000902002F0B7F9002002F0B4F9EB2002F055
:105D4000B1F9002002F0AEF9DC2002F0ABF900203E
:105D500002F0A8F9B82002F0B1F9002002F0A2F98F
:105D6000002002F09FF9002002F09CF9002002F0D0
:105D700099F9002002F096F9002002F093F9002032
:105D800002F090F9002002F08DF9BA2002F096F9A5
:105D9000242002F087F9002002F084F9002002F0AC
:105DA00081F9002002F07EF9C12002F087F920205D
:105DB00002F078F9002002F075F9542002F072F92F
:105DC000002002F06FF9FF2002F06CF9002002F0D1
:105DD00069F9C22002F072F90A2002F063F900208A
:105DE00002F060F9042002F05DF9002002F05AF997
:105DF000C32002F063F93C2002F054F9002002F0C5
:105E000051F93A2002F04EF9002002F04BF9392006
:105E100002F048F9002002F045F9372002F042F97B
:105E2000002002F03FF93C2002F03CF9002002F093
:105E300039F9362002F036F9002002F033F9322029
:105E400002F030F9002002F02DF92F2002F02AF99B
:105E5000002002F027F92C2002F024F9002002F0A3
:105E600021F9292002F01EF9002002F01BF926205A
:105E700002F018F9002002F015F9242002F012F9BE
:105E8000002001E0E406002402F00CF9242002F0D6
:105E900009F9002002F006F9232002F003F900209E
:105EA00002F000F93C2002F0FDF8002002F0FAF8C0
:105EB000362002F0F7F8002002F0F4F8322002F069
:105EC000F1F8002002F0EEF82F2002F0EBF80020AD
:105ED00002F0E8F82C2002F0E5F8002002F0E2F8E9
:105EE000292002F0DFF8002002F0DCF8262002F082
:105EF000D9F8002002F0D6F8242002F0D3F80020D0
:105F000002F0D0F8242002F0CDF8002002F0CAF808
:105F1000232002F0C7F8002002F0C4F8C42002F0E9
:105F2000CDF8622002F0BEF8002002F0BBF8052098
:105F300002F0B8F8002002F0B5F8842002F0B2F8C0
:105F4000002002F0AFF8F02002F0ACF8002002F0E0
:105F5000A9F8182002F0A6F8002002F0A3F8A42067
:105F600002F0A0F8002002F09DF8182002F09AF844
:105F7000002002F097F8502002F094F8002002F080
:105F800091F80C2002F08EF8002002F08BF8172018
:105F900002F088F8002002F085F8952002F082F8DF
:105FA000002002F07FF8F32002F07CF8002002F0DD
:105FB00079F8E62002F076F8002002F073F8C520A8
:105FC00002F07CF8322002F06DF8002002F06AF84E
:105FD000442002F067F8002002F064F8652002F027
:105FE00061F8002002F05EF8762002F05BF80020F5
:105FF00002F058F8882002F055F8002002F052F81C
:10600000C62002F05BF8202002F04CF8002002F0DD
:1060100049F8172002F046F8002002F043F801206A
:1060200002F040F8002002F03DF8C72002F046F8E8
:10603000002002F037F8002002F034F8002002F0CF
:1060400031F8002002F02EF8C82002F037F80020C6
:1060500002F028F8002002F025F8002002F022F8D3
:10606000002002F01FF8C92002F028F8002002F0FA
:1060700019F8002002F016F8002002F013F80020B2
:1060800002F010F8002002F00DF8002002F00AF8EB
:10609000002002F007F8002002F004F8002002F0CF
:1060A00001F8002001F0FEFF002001F0FBFF0020BE
:1060B00001F0F8FF002001F0F5FF002001F0F2FFF1
:1060C000002001F0EFFF002001F0ECFFE02001F0E4
:1060D000F5FF162001F0E6FF002001F0E3FF1C2091
:1060E00001F0E0FF002001F0DDFF212001F0DAFFE8
:1060F000002001F0D7FF362001F0D4FF002001F08E
:10610000D1FF462001F0CEFF002001F0CBFF52204E
:1061100001F0C8FF002001F0C5FF642001F0C2FFBC
:10612000002001F0BFFF7A2001F0BCFF002001F049
:10613000B9FF8B2001F0B6FF002001F0B3FF9920DA
:1061400001F0B0FF002001F0ADFFA82001F0AAFF90
:10615000002001F0A7FFB92001F0A4FF002001F00A
:10616000A1FFC42001F09EFF002001F09BFFCA2088
:1061700001F098FF002001F095FFD22001F092FF7E
:10618000002001F08FFFD92001F08CFF002001F0EA
:1061900089FFE02001F086FF002001F083FFF3205B
:1061A00001F080FF002001F07DFFE12001F086FF7B
:1061B000162001F077FF002001F074FF1C2001F091
:1061C00071FF002001F06EFF222001F06BFF002024
:1061D00001F068FF362001F065FF002001F062FF4A
:1061E000452001F05FFF002001F05CFF522001F02C
:1061F00059FF002001F056FF642001F053FF0020FA
:1062000001F050FF7A2001F04DFF002001F04AFF1D
:106210008B2001F047FF002001F044FF992001F09E
:1062200041FF002001F03EFFA82001F03BFF0020CD
:1062300001F038FFB92001F035FF002001F032FFF6
:10624000C42001F02FFF002001F02CFFCA2001F034
:1062500029FF002001F026FFD22001F023FF0020BB
:1062600001F020FFD82001F01DFF002001F01AFFEF
:10627000E02001F017FF002001F014FFF32001F0EF
:1062800011FF002001F00EFFE22001F017FF0520B2
:1062900001F008FF002001F005FF0B2001F002FFD4
:1062A000002001F0FFFE1B2001F0FCFE002001F0A9
:1062B000F9FE342001F0F6FE002001F0F3FE442048
:1062C00001F0F0FE002001F0EDFE4F2001F0EAFEAB
:1062D000002001F0E7FE612001F0E4FE002001F063
:1062E000E1FE792001F0DEFE002001F0DBFE8820D7
:1062F00001F0D8FE002001F0D5FE972001F0D2FE7B
:10630000002001F0CFFEA62001F0CCFE002001F01D
:10631000C9FEB72001F0C6FE002001F0C3FEC22076
:1063200001F0C0FE002001F0BDFEC72001F0BAFE62
:10633000002001F0B7FED12001F0B4FE002001F0F2
:10634000B1FED62001F0AEFE002001F0ABFEDD2054
:1063500001F0A8FE002001F0A5FEF32001F0A2FE4E
:10636000002001F09FFEE32001F0A8FE052001F0CF
:1063700099FE002001F096FE0A2001F093FE002015
:1063800001F090FE1C2001F08DFE002001F08AFE3D
:10639000332001F087FE002001F084FE442001F04C
:1063A00081FE002001F07EFE502001F07BFE0020E7
:1063B00001F078FE622001F075FE002001F072FE0F
:1063C000782001F06FFE002001F06CFE882001F0C3
:1063D00069FE002001F066FE972001F063FE0020B8
:1063E00001F060FEA62001F05DFE002001F05AFEE3
:1063F000B72001F057FE002001F054FEC22001F04A
:1064000051FE002001F04EFEC72001F04BFE00209F
:1064100001F048FED12001F045FE002001F042FECF
:10642000D52001F03FFE002001F03CFEDD2001F010
:1064300039FE002001F036FEF32001F033FE00208B
:1064400001F030FEE42001F039FE012001F02AFEC7
:10645000002001F027FE012001F024FE002001F0C1
:1064600021FE022001F01EFE002001F01BFE2A206A
:1064700001F018FE002001F015FE3C2001F012FE94
:10648000002001F00FFE4B2001F00CFE002001F077
:1064900009FE5D2001F006FE002001F003FE7420DD
:1064A00001F000FE002001F0FDFD842001F0FAFD66
:1064B000002001F0F7FD932001F0F4FD002001F031
:1064C000F1FDA22001F0EEFD002001F0EBFDB32074
:1064D00001F0E8FD002001F0E5FDBE2001F0E2FD45
:1064E000002001F0DFFDC42001F0DCFD002001F000
:1064F000D9FDCD2001F0D6FD002001F0D3FDD32041
:1065000001F0D0FD002001F0CDFDDD2001F0CAFD3D
:10651000002001F0C7FDF32001F0C4FD002001F0D0
:10652000C1FDE52001F0CAFD002001F0BBFD002007
:1065300001F0B8FD002001F0B5FD002001F0B2FD32
:10654000022001F0AFFD002001F0ACFD292001F098
:10655000A9FD002001F0A6FD3C2001F0A3FD0020D4
:1065600001F0A0FD4B2001F09DFD002001F09AFDFF
:106570005D2001F097FD002001F094FD742001F0F2
:1065800091FD002001F08EFD842001F08BFD0020A4
:1065900001F088FD932001F085FD002001F082FDCF
:1065A000A22001F07FFD002001F07CFDB32001F06E
:1065B00079FD002001F076FDBE2001F073FD002082
:1065C00001F070FDC42001F06DFD002001F06AFDB6
:1065D000CD2001F067FD002001F064FDD32001F023
:1065E00061FD002001F05EFDDC2001F05BFD00207C
:1065F00001F058FDF32001F055FD002001F052FD9F
:10660000E62001F05BFD112001F04CFD002001F0BF
:1066100049FD342001F046FD002001F043FD5620E5
:1066200001F040FD002001F03DFD762001F03AFD33
:10663000002001F037FD772001F034FD002001F04B
:1066400031FD662001F02EFD002001F02BFD882099
:1066500001F028FD002001F025FD992001F022FD28
:10666000002001F01FFDBB2001F01CFD002001F007
:1066700019FD992001F016FD002001F013FD6620A0
:1066800001F010FD002001F00DFD552001F00AFD84
:10669000002001F007FD552001F004FD002001F06D
:1066A00001FD452001F0FEFC002001F0FBFC432031
:1066B00001F0F8FC002001F0F5FC442001F0F2FCB0
:1066C000002001F0EFFCE72001F0F8FC322001F09F
:1066D000E9FC002001F0E6FC552001F0E3FC00207D
:1066E00001F0E0FC762001F0DDFC002001F0DAFC96
:1066F000662001F0D7FC002001F0D4FC672001F0F7
:10670000D1FC002001F0CEFC672001F0CBFC002082
:1067100001F0C8FC872001F0C5FC002001F0C2FC9C
:10672000992001F0BFFC002001F0BCFCBB2001F06F
:10673000B9FC002001F0B6FC992001F0B3FC002068
:1067400001F0B0FC772001F0ADFC002001F0AAFCC4
:10675000442001F0A7FC002001F0A4FC562001F029
:10676000A1FC002001F09EFC232001F09BFC0020F6
:1067700001F098FC332001F095FC002001F092FC20
:10678000452001F08FFC002001F08CFCE82001F096
:1067900095FC002001F086FC002001F083FC99208C
:1067A00001F080FC002001F07DFC872001F07AFCE4
:1067B000002001F077FC882001F074FC002001F03B
:1067C00071FC772001F06EFC002001F06BFC66206C
:1067D00001F068FC002001F065FC882001F062FCFB
:1067E000002001F05FFCAA2001F05CFC002001F019
:1067F00059FCBB2001F056FC002001F053FC99200D
:1068000001F050FC002001F04DFC662001F04AFC34
:10681000002001F047FC552001F044FC002001F06D
:1068200041FC552001F03EFC002001F03BFC4420DF
:1068300001F038FC002001F035FC442001F032FC6E
:10684000002001F02FFC552001F02CFC002001F06D
:1068500029FCE92001F032FCAA2001F023FC0020F1
:1068600001F020FC002001F01DFC002001F01AFCCA
:10687000002001F023FCAA2001F014FCCF2001F03D
:106880001DFC002001F00EFC002001F00BFC00209C
:1068900001F008FC002001F005FC002001F002FCE2
:1068A000002001F0FFFB002001F0FCFB002001F0C4
:1068B000F9FB002001F0F6FB002001F0F3FB0020C3
:1068C00001F0F0FB002001F0EDFB002001F0EAFBFD
:1068D000002001F0E7FB002001F0E4FB002001F0C4
:1068E000E1FB002001F0DEFBF02001F0E7FB0020DF
:1068F00001F0D8FB502001F0D5FB002001F0D2FBC5
:10690000002001F0CFFB002001F0CCFBF32001F0D0
:10691000D5FB002001F0C6FBF92001F0CFFB0620DB
:1069200001F0C0FB102001F0BDFB292001F0BAFBF3
:10693000002001F0B7FB3A2001F0C0FB552001F028
:10694000B1FB112001F0BAFB642006F045F92920C3
:1069500001F0B4FB352001F0B1FB002001F0A2FBF7
:10696000512001F0ABFBFF2001F09CFB532001F014
:10697000A5FB2C2001F096FB552001F09FFB822007
:1069800001F090FB2C2001F099FB01F048B8FE4883
:10699000808845F2105188427ED155214FF47040D5
:1069A00001F0A2FBAA214FF2010001F09DFB522150
:1069B0004FF2020001F098FB08214FF2030001F0B2
:1069C00093FB01214FF2040001F08EFB0D214FF4E7
:1069D000304001F089FB0D214BF2010001F084FBF6
:1069E0000D214BF2020001F07FFB34214FF43640C1
:1069F00001F07AFB34214BF2016001F075FB342188
:106A00004BF2026001F070FB0D214FF4314001F0B8
:106A10006BFB0D214BF2011001F066FB0D214BF2D7
:106A2000021001F061FB34214FF4374001F05CFBB0
:106A300034214BF2017001F057FB34214BF202700C
:106A400001F052FB00214FF4324001F04DFB0021D8
:106A50004BF2012001F048FB00214BF2022001F033
:106A600043FB24214FF4384001F03EFB24214BF638
:106A7000010001F039FB24214BF6020001F034FB48
:106A800001214FF43F4001F02FFB0F214FF4334021
:106A900001F02AFB0F2100E0FEE34BF2013001F090
:106AA00023FB0F214BF2023001F01EFB34214FF487
:106AB000394001F019FB34214BF6011001F014FBB1
:106AC00034214BF6021001F00FFB08214FF4354042
:106AD00001F00AFB08214BF2015001F005FB0821EF
:106AE0004BF2025001F000FB03214FF4424001F051
:106AF000FBFA24214FF43A4001F0F6FA24214BF638
:106B0000012001F0F1FA24214BF6022001F0ECFA09
:106B100000214FF43C4001F0E7FA78214BF60140A8
:106B200001F0E2FA00214BF6024001F0DDFA00210B
:106B30004FF43D4001F0D8FA78214BF6015001F0B6
:106B4000D3FA00214BF6025001F0CEFA00214FF4A7
:106B50003E4001F0C9FA64214BF6016001F0C4FA2D
:106B600000214FF4514001F0BFFA33214DF20110E2
:106B700001F0BAFA00214DF2021001F0B5FA342109
:106B80004DF2031001F0B0FA00214DF2041001F0B3
:106B9000ABFA3A214DF2051001F0A6FA00214DF2B0
:106BA000061001F0A1FA4A214DF2071001F09CFAFB
:106BB00000214DF2081001F097FA5C214DF2091006
:106BC00001F092FA00214DF20A1001F08DFA8121B4
:106BD0004DF20B1001F088FA00214DF20C1001F07B
:106BE00083FAA6214DF20D1001F07EFA00214DF23C
:106BF0000E1001F079FAE5214DF20F1001F074FA50
:106C000001214DF2101001F06FFA13214DF2111015
:106C100001F06AFA01214DF2121001F065FA5421D7
:106C20004DF2131001F060FA01214DF2141001F041
:106C30005BFA82214DF2151001F056FA01214DF256
:106C4000161001F051FACA214DF2171001F04CFA5A
:106C500002214DF2181001F047FA00214DF21910EF
:106C600001F042FA02214DF21A1001F03DFA012121
:106C70004DF21B1001F038FA02214DF21C1001F008
:106C800033FA34214DF21D1001F02EFA02214DF29B
:106C90001E1001F029FA67214DF21F1001F024FAAD
:106CA00002214DF2201001F01FFA84214DF2211033
:106CB00001F01AFA02214DF2221001F015FAA42176
:106CC0004DF2231001F010FA02214DF2241001F0D0
:106CD0000BFAB7214DF2251001F006FA02214DF210
:106CE000261001F001FACF214DF2271001F0FCF936
:106CF00002214DF2281001F0F7F9DE214DF22910A2
:106D000001F0F2F902214DF22A1001F0EDF9F22121
:106D10004DF22B1001F0E8F902214DF22C1001F098
:106D2000E3F9FE214DF22D1001F0DEF903214DF2C1
:106D30002E1001F0D9F910214DF22F1001F0D4F9E5
:106D400003214DF2301001F0CFF933214DF2311013
:106D500001F0CAF903214DF2321001F0C5F96D219D
:106D60004DF2331001F0C0F900214FF4524001F010
:106D7000BBF933214DF2012001F0B6F900214DF2AB
:106D8000022001F0B1F901E0E406002434214DF2C3
:106D9000032001F0A9F900214DF2042001F0A4F92B
:106DA0003A214DF2052001F09FF900214DF2062015
:106DB00001F09AF94A214DF2072001F095F90021DE
:106DC0004DF2082001F090F95C214DF2092001F00C
:106DD0008BF900214DF20A2001F086F981214DF254
:106DE0000B2001F081F900214DF20C2001F07CF91B
:106DF000A6214DF20D2001F077F900214DF20E2071
:106E000001F072F9E5214DF20F2001F06DF9012139
:106E10004DF2102001F068F913214DF2112001F01C
:106E200063F901214DF2122001F05EF954214DF277
:106E3000132001F059F901214DF2142001F054F909
:106E400082214DF2152001F04FF901214DF216205B
:106E500001F04AF9CA214DF2172001F045F902214B
:106E60004DF2182001F040F900214DF2192001F0F7
:106E70003BF902214DF21A2001F036F901214DF2C1
:106E80001B2001F031F902214DF21C2001F02CF9F8
:106E900034214DF21D2001F027F902214DF21E2070
:106EA00001F022F967214DF21F2001F01DF90221A6
:106EB0004DF2202001F018F984214DF2212001F03B
:106EC00013F902214DF2222001F00EF9A4214DF216
:106ED000232001F009F902214DF2242001F004F9E8
:106EE000B7214DF2252001F0FFF802214DF22620B6
:106EF00001F0FAF8CF214DF2272001F0F5F8022138
:106F00004DF2282001F0F0F8DE214DF2292001F0A9
:106F1000EBF802214DF22A2001F0E6F8F2214DF2C1
:106F20002B2001F0E1F802214DF22C2001F0DCF8D9
:106F3000FE214DF22D2001F0D7F803214DF22E2035
:106F400001F0D2F810214DF22F2001F0CDF80321ED
:106F50004DF2302001F0C8F833214DF2312001F01C
:106F6000C3F803214DF2322001F0BEF86D214DF23D
:106F7000332001F0B9F800214FF4534001F0B4F888
:106F800033214DF2013001F0AFF800214DF2023013
:106F900001F0AAF834214DF2033001F0A5F80021E8
:106FA0004DF2043001F0A0F83A214DF2053001F025
:106FB0009BF800214DF2063001F096F84A214DF27F
:106FC000073001F091F800214DF2083001F08CF803
:106FD0005C214DF2093001F087F800214DF20A30B2
:106FE00001F082F881214DF20B3001F07DF8002193
:106FF0004DF20C3001F078F8A6214DF20D3001F081
:1070000073F800214DF20E3001F06EF8E5214DF2DB
:107010000F3001F069F801214DF2103001F064F8F1
:1070200013214DF2113001F05FF801214DF21230C1
:1070300001F05AF854214DF2133001F055F80121B6
:107040004DF2143001F050F882214DF2153001F06C
:107050004BF801214DF2163001F046F8CA214DF2ED
:10706000173001F041F802214DF2183001F03CF8E0
:1070700000214DF2193001F037F802214DF21A309B
:1070800001F032F801214DF21B3001F02DF8022100
:107090004DF21C3001F028F834214DF21D3001F082
:1070A00023F802214DF21E3001F01EF867214DF247
:1070B0001F3001F019F802214DF2203001F014F8D0
:1070C00084214DF2213001F00FF802214DF22230DF
:1070D00001F00AF8A4214DF2233001F005F8022155
:1070E0004DF2243001F000F8B7214DF2253000F0C8
:1070F000FBFF02214DF2263000F0F6FFCF214DF2CA
:10710000273000F0F1FF02214DF2283000F0ECFFB3
:10711000DE214DF2293000F0E7FF02214DF22A3046
:1071200000F0E2FFF2214DF22B3000F0DDFF0221F2
:107130004DF22C3000F0D8FFFE214DF22D3000F042
:10714000D3FF03214DF22E3000F0CEFF10214DF27F
:107150002F3000F0C9FF03214DF2303000F0C4FFA2
:1071600033214DF2313000F0BFFF03214DF23230B8
:1071700000F0BAFF6D214DF2333000F0B5FF002171
:107180004FF4544000F0B0FF33214DF2014000F0C5
:10719000ABFF00214DF2024000F0A6FF34214DF27A
:1071A000034000F0A1FF00214DF2044000F09CFFDD
:1071B0003A214DF2054000F097FF00214DF20640C4
:1071C00000F092FF4A214DF2074000F08DFF0021B0
:1071D0004DF2084000F088FF5C214DF2094000F0BC
:1071E00083FF00214DF20A4000F07EFF81214DF225
:1071F0000B4000F079FF00214DF20C4000F074FFCD
:10720000A6214DF20D4000F06FFF00214DF20E401F
:1072100000F06AFFE5214DF20F4000F065FF01210B
:107220004DF2104000F060FF13214DF2114000F0CC
:107230005BFF01214DF2124000F056FF54214DF248
:10724000134000F051FF01214DF2144000F04CFFBB
:1072500082214DF2154000F047FF01214DF216400A
:1072600000F042FFCA214DF2174000F03DFF02211D
:107270004DF2184000F038FF00214DF2194000F0A7
:1072800033FF02214DF21A4000F02EFF01214DF292
:107290001B4000F029FF00E003E302214DF21C40F7
:1072A00000F022FF34214DF21D4000F01DFF0221AD
:1072B0004DF21E4000F018FF67214DF21F4000F014
:1072C00013FF02214DF2204000F00EFF84214DF209
:1072D000214000F009FF02214DF2224000F004FF9E
:1072E000A4214DF2234000F0FFFE02214DF2244084
:1072F00000F0FAFEB7214DF2254000F0F5FE022124
:107300004DF2264000F0F0FECF214DF2274000F074
:10731000EBFE02214DF2284000F0E6FEDE214DF2A8
:10732000294000F0E1FE02214DF22A4000F0DCFE8F
:10733000F2214DF22B4000F0D7FE02214DF22C40FD
:1073400000F0D2FEFE214DF22D4000F0CDFE0321D3
:107350004DF22E4000F0C8FE10214DF22F4000F0FB
:10736000C3FE03214DF2304000F0BEFE33214DF24A
:10737000314000F0B9FE03214DF2324000F0B4FE7E
:107380006D214DF2334000F0AFFE00214FF4554027
:1073900000F0AAFE33214DF2015000F0A5FE0021BD
:1073A0004DF2025000F0A0FE34214DF2035000F0E7
:1073B0009BFE00214DF2045000F096FE3A214DF262
:1073C000055000F091FE00214DF2065000F08CFEB9
:1073D0004A214DF2075000F087FE00214DF208507F
:1073E00000F082FE5C214DF2095000F07DFE00218C
:1073F0004DF20A5000F078FE81214DF20B5000F062
:1074000073FE00214DF20C5000F06EFEA6214DF2ED
:107410000D5000F069FE00214DF20E5000F064FEA8
:10742000E5214DF20F5000F05FFE01214DF21050AA
:1074300000F05AFE13214DF2115000F055FE0121CB
:107440004DF2125000F050FE54214DF2135000F056
:107450004BFE01214DF2145000F046FE82214DF208
:10746000155000F041FE01214DF2165000F03CFE97
:10747000CA214DF2175000F037FE02214DF218508C
:1074800000F032FE00214DF2195000F02DFE0221D5
:107490004DF21A5000F028FE01214DF21B5000F071
:1074A00023FE02214DF21C5000F01EFE34214DF24D
:1074B0001D5000F019FE02214DF21E5000F014FE86
:1074C00067214DF21F5000F00FFE02214DF22050B7
:1074D00000F00AFE84214DF2215000F005FE022149
:1074E0004DF2225000F000FEA4214DF2235000F096
:1074F000FBFD02214DF2245000F0F6FDB7214DF2C4
:10750000255000F0F1FD02214DF2265000F0ECFD77
:10751000CF214DF2275000F0E7FD02214DF2285017
:1075200000F0E2FDDE214DF2295000F0DDFD0221E8
:107530004DF22A5000F0D8FDF2214DF22B5000F010
:10754000D3FD02214DF22C5000F0CEFDFE214DF274
:107550002D5000F0C9FD03214DF22E5000F0C4FD66
:1075600010214DF22F5000F0BFFD03214DF230509D
:1075700000F0BAFD33214DF2315000F0B5FD03218A
:107580004DF2325000F0B0FD6D214DF2335000F05D
:10759000ABFD00214FF4564000F0A6FD33214DF223
:1075A000016000F0A1FD00214DF2026000F09CFDA1
:1075B00034214DF2036000F097FD00214DF204608C
:1075C00000F092FD3A214DF2056000F08DFD0021A2
:1075D0004DF2066000F088FD4A214DF2076000F090
:1075E00083FD00214DF2086000F07EFD5C214DF22C
:1075F000096000F079FD00214DF20A6000F074FD91
:1076000081214DF20B6000F06FFD00214DF20C6006
:1076100000F06AFDA6214DF20D6000F065FD00212D
:107620004DF20E6000F060FDE5214DF20F6000F0BC
:107630005BFD01214DF2106000F056FD13214DF26B
:10764000116000F051FD01214DF2126000F04CFD7F
:1076500054214DF2136000F047FD01214DF21460FA
:1076600000F042FD82214DF2156000F03DFD012148
:107670004DF2166000F038FDCA214DF2176000F09F
:1076800033FD02214DF2186000F02EFD00214DF275
:10769000196000F029FD02214DF21A6000F024FD6E
:1076A00001214DF21B6000F01FFD02214DF21C6014
:1076B00000F01AFD34214DF21D6000F015FD02218D
:1076C0004DF21E6000F010FD67214DF21F6000F0CA
:1076D0000BFD02214DF2206000F006FD84214DF2E9
:1076E000216000F001FD02214DF2226000F0FCFC5F
:1076F000A4214DF2236000F0F7FC02214DF224603A
:1077000000F0F2FCB7214DF2256000F0EDFC022103
:107710004DF2266000F0E8FCCF214DF2276000F02A
:10772000E3FC02214DF2286000F0DEFCDE214DF288
:10773000296000F0D9FC02214DF22A6000F0D4FC4F
:10774000F2214DF22B6000F0CFFC02214DF22C60B3
:1077500000F0CAFCFE214DF22D6000F0C5FC0321B3
:107760004DF22E6000F0C0FC10214DF22F6000F0B1
:10777000BBFC03214DF2306000F0B6FC33214DF22A
:10778000316000F0B1FC03214DF2326000F0ACFC3E
:107790006D214DF2336000F0A7FC55214FF470408D
:1077A00000F0A2FCAA214FF2010000F09DFC522142
:1077B0004FF2020000F098FC08214FF2030000F0A5
:1077C00093FC00214FF2040000F08EFCCC214FF41A
:1077D000314000F089FC00214BF2011000F084FCE4
:1077E00005214FF4364000F07FFC70214FF4374004
:1077F00000F07AFC70214BF2017000F075FC012161
:107800004FF4384000F070FC03214BF6010000F00B
:107810006BFC03214BF6020000F066FC03214BF6E3
:10782000030000F061FC02214FF43C4000F05CFCDE
:1078300000214BF6014000F057FC00214BF60240BE
:1078400000F052FCD0214FF4494000F04DFC0221E1
:107850004CF6011000F048FC50214CF6021000F0EC
:1078600043FC50214CF6031000F03EFC50214CF636
:10787000041000F039FC00214FF4545000F034FCA7
:1078800055214FF4685000F02FFC4FF4885000F061
:1078900015FC782005F0ACF94FF4245000F00EFCF4
:1078A000BDE07948808841F663118842F8D1E22032
:1078B00000F004FC1D2000F0F5FB022000F0F2FBBC
:1078C000042000F0EFFB642005F092F9E02000F0C6
:1078D000F5FB012000F0E6FB0A2005F07DF9E02031
:1078E00000F0ECFB032000F0DDFB0C2005F074F948
:1078F000012000F0E3FB0A2005F06EF9E62000F01D
:10790000DDFB2F2000F0CEFBFF2000F0CBFBFF20A3
:1079100000F0C8FBB02000F0D1FB202000F0C2FB3B
:10792000002000F0BFFB032000F0BCFB40F21F3042
:1079300000F0B8FB012000F0B5FB40F2DF1000F0D2
:10794000B1FB002000F0AEFBB42000F0B7FB042038
:1079500000F0A8FB40F21F4000F0A4FB002000F064
:10796000A1FB2E2000F09EFB002000F09BFB0020DE
:1079700000F098FB002000F095FB002000F092FB47
:10798000B62000F09BFB022000F08CFB4FF403704C
:1079900000F088FB002000F085FB172000F082FB40
:1079A000152000F07FFB002000F07CFB002000F0A1
:1079B00079FBF02000F082FB032000F073FB29200C
:1079C00000F07CFBD02000F079FB002000F06AFB87
:1079D000BE2000F073FB052000F064FBFE2000F0E9
:1079E00061FB012000F05EFB002000F05BFB00204B
:1079F00000F058FB002000F055FBB82000F05EFBC3
:107A0000032000F04FFB012000F04CFBBA2000F0F7
:107A100055FB012000F046FB642000F073F81A4883
:107A2000808849F24131884211D01748808845F258
:107A3000103188420BD01448808845F2105188429A
:107A400005D01148808841F66311884209D105208C
:107A5000029004900D49CB6A8A68486802A9F8F739
:107A6000E7FF094881880AA004F000FC0020FDF728
:107A700093FC012220210948F9F7F0FA4FF6FF7034
:107A8000FDF766FC15B000BDE4060024980600244E
:107A90004C43442049443A25780D0A00000402581A
:107AA0001FB5F9F7FDFC01208DF8000003208DF8CB
:107AB0000100400701901B208DF8080000208DF880
:107AC00009008DF80A0003208DF80B0000208DF8C6
:107AD0000C008DF80D008DF80E0001208DF80F00C0
:107AE0006846F9F7AFFC0420F9F7F0FC1FBD000071
:107AF00008B5034800880090BDF8000008BD0000EC
:107B00000000086000B50246BE2000F0D7FA05204C
:107B100000F0C8FA00EE102AB8EE400B9FED0B1BE8
:107B200020EE010BBCEEC00B10EE101A88B200F074
:107B3000B9FA012000F0B6FAFF2000F0B3FA0020F5
:107B400000F0B0FA002000F0ADFA00BD666666668F
:107B500066660440F0B50546002400279948807900
:107B6000012805D19748808841F66311884208D1E1
:107B700094488079F0B99348808841F6631188422F
:107B800018D1082D15D2DFE805F00406080A0C0EFE
:107B9000101206250DE007250BE0042509E0052558
:107BA00007E0012505E0002503E0032501E00225AB
:107BB00000BF00BF8348808849F24131884211D01C
:107BC0008048808845F2103188420BD07D488088FB
:107BD00045F21051884205D07A48808841F66311F9
:107BE00088427DD1082D1CD2DFE805F00406090C7F
:107BF0000F12151800BF14E044F0800411E044F0A7
:107C000040040EE044F0C0040BE044F0200408E01F
:107C100044F0600405E044F0A00402E044F0E00415
:107C200000BF00BF6748808845F21051884202D1EA
:107C30004FF4585700E036276248808845F21031EB
:107C400088420DD05F48808845F21051884207D0A5
:107C50005C48808841F66311884201D044F00804F2
:107C60002146384600F040FA5648808841F66311B4
:107C700088421DD004F0200068B152480088514964
:107C80004988884214DA4F48068840884D49088060
:107C9000084646800CE04B4800884A49498888429B
:107CA00006DD4848068840884649088008464680E0
:107CB0004448808845F21051884254D1414948894E
:107CC00000F0FCF9002000F0EDF93E494989491C1B
:107CD00088B200F0F3F9002000F0E4F9394900E03F
:107CE0006FE04989891C88B200F0E8F935490988B4
:107CF000491EC1F30F2000F0D5F932494989C91C4A
:107D000088B200F0DBF92F490978491EC8B200F0AB
:107D1000C9F92C49888900F0D1F9002000F0C2F996
:107D200028498989491C88B200F0C8F9002000F070
:107D3000B9F924498989891C88B200F0BFF9214921
:107D40004988491EC1F30F2000F0ACF91D4989890B
:107D5000C91C88B200F0B2F91A498978491EC8B224
:107D600000F0A0F92DE01749488900F0A7F900209C
:107D700000F098F9002000F095F912490988491E91
:107D8000C1F30F2000F08EF90E490978491EC8B2E0
:107D900000F088F90B49888900F090F9002000F084
:107DA00081F9002000F07EF906494988491EC1F397
:107DB0000F2000F077F903498978491EC8B200F016
:107DC00071F9F0BDE406002410B502460C464B489C
:107DD000808849F24131884205D04848808845F280
:107DE0001031884214D14549488900F067F91012D2
:107DF00000F058F9D0B200F055F94049888900F0F8
:107E00005DF9201200F04EF9E0B200F04BF973E09A
:107E10003A48808841F66311884247D137488079D3
:107E2000A8B936480088401E801A82B23349488972
:107E300000F044F9002000F035F9002000F032F99C
:107E4000101200F02FF9D0B200F02CF916E02B49F7
:107E5000488900F033F9101200F024F9D0B200F094
:107E600021F926490988491EC1F30F2000F01AF9AB
:107E700022490978491EC8B200F014F91F498889BF
:107E800000F01CF9201200F00DF9E0B200F00AF940
:107E90001A494988491EC1F30F2000F003F9174918
:107EA0008978491EC8B200F0FDF825E013488088A3
:107EB00045F2105188421FD11049488900F0FEF860
:107EC000101200F0EFF80D494989491C88B200F002
:107ED000F5F8D0B200F0E6F80849888900F0EEF82D
:107EE000201200F0DFF805498989491C88B200F0AA
:107EF000E5F8E0B200F0D6F810BD0000E40600247A
:107F00002DE9F84F80460F4616461C46BB462046D4
:107F1000E31704EB5373DB1021464FEAE47C04EBD8
:107F20005C7C4FEAEC0CA4EBCC0CBCF1000F02D053
:107F30004FF0010C01E04FF0000C6344224604EBCB
:107F4000D27C4FEA6C0C03FB0CF3DBB20093A6F17E
:107F50002000C6B200255EE00C2C07D106EB4600DF
:107F60002F4901EB800010F805901BE0102C05D183
:107F70002C4800EB061010F8059013E0182C07D1E0
:107F800006EBC600284901EB800010F8059009E0D7
:107F9000202C05D1254800EBC61010F8059001E013
:107FA000BDE8F88F4FF0000A2FE009F0800030B1F3
:107FB0001F48394602684046FDF7AEFA07E00A98C6
:107FC00028B91C48394602684046FDF7A5FA4FEA31
:107FD00049604FEA1069781C87B217484088B84258
:107FE00000DCDDE7A7EB0B00A0420AD15F4608F1F9
:107FF00001001FFA80F810480088404500DCCFE7F8
:1080000006E00AF1010000F0FF0ABAF1080FCCDB2C
:1080100000BF681CC5B2009885429DDB00BFBFE76A
:1080200064E30008D8E70008C8ED000824FB000856
:108030002000002424000024E40600242DE9F84F49
:1080400004460D4690469946DDE90A6704F0FF0AAA
:1080500008EB04001FFA80F809EB05001FFA80F90D
:1080600016E0444502DB5446A81985B24D4500DBB5
:1080700014E0002000903A78334629462046FFF766
:108080003FFF304606EBD07104EB61018CB27F1CE0
:1080900038787E2802DC38782028E2DA00BFBDE894
:1080A000F88F000001B5BDF800000090BDF8000099
:1080B0000149088008BD00000000086001B5BDF856
:1080C00000000090BDF800000149088008BD0000D4
:1080D000FEFF0760024800890249088070470000DF
:1080E000E4060024FEFF0760024A1080921C118003
:1080F00070470000FEFF076000B587B000BF124860
:10810000006840F00200104908600846006800F06E
:108110000200019000BF00BF0320029001200390E5
:1081200004900320059002A90848F8F765FE012293
:1081300011460648F8F792FF012202210348F8F79A
:108140008DFF07B000BD0000E04402580004025853
:1081500018B5044606480094008B401E83B20448BC
:10816000C08A401E82B20021084600F059F818BDAE
:10817000FC07002470B5B0B004460E4615464FF01B
:10818000005001900A940B9602210C910D910E95CE
:1081900001A8FAF7D9FB10B9002030B070BD01205A
:1081A000FBE700000949487530B98988074AD18240
:1081B00011460988118308E0012806D1034909887E
:1081C000024AD1821146898811837047FC07002436
:1081D00070B5114B5B7D6BB10F4BDB690E4D2D689C
:1081E00005FB01056B430C4D2D7D0C4E56F82550BB
:1081F000EA520FE0084B1D685B681B1A5B1E05FB0B
:108200000313054DED696B43034D2D7D034E56F869
:108210002550EA5270BD0000FC070024280000240D
:108220002DE9F04F04460D4616464FF0000CDFF8DE
:10823000289199F81590B9F1000F04D020462946ED
:1082400032461F4611E02846DFF80C91D9F8049019
:10825000A9EB0609A9F101011A46DFF8FC90D9F84B
:108260000490A9EB0409A9F10107DFF8EC90B9F833
:108270000090A2EB000A0AF1010AA9EB0A091FFA11
:1082800089F8DFF8D49099F81490DFF8D0A05AF864
:108290002990DFF8C4A0DAF81CA0DFF8BCB0DBF846
:1082A00000B00BFB010B0AFB0B9EDFF8B490D9F872
:1082B000009049F40009DFF8A8A0CAF800904FF434
:1082C0004039DFF8A0A0CAF800904FF00209CAF8C0
:1082D0003490D146C9F84080D9F8009029F00109BE
:1082E000CAF80090D146C9F83CE0A7EB010909F1B2
:1082F0000109A2EB000A0AF1010A49EA0A49DFF87A
:1083000064A0CAF84490DDF82490CAF83890D146A9
:10831000D9F8009049F00109CAF8009005E00CF185
:10832000010CBCF5001F00D308E0DFF83890D9F845
:10833000049009F00209B9F1000FF0D000BFDFF896
:108340002490D9F8089049F00209DFF818A0CAF87B
:108350000890BDE8F08F0000FC07002428000024EE
:10836000D8440258001000521FB5002400F050FA03
:10837000044644F24230844217D14FF4F070F2497F
:1083800008604FF4887048600120088148812820E7
:1083900088810820C8810520088208204882582248
:1083A000A0210520FFF7E6FE2FE147F2840084427A
:1083B00017D14FF44870E44908604FF4F0704860FA
:1083C0000120088148812E2088811720C881D22071
:1083D0000882162048821822A0210520FFF7CAFE35
:1083E00013E147F21600844218D14FF48060D64959
:1083F00008604FF4167048601420088103204881FB
:108400008C2088811420C881A02008820C204882FA
:108410001222A0210520FFF7ADFEF6E047F218007A
:10842000844207D14FF4A060C74908604FF44870F8
:108430004860EAE048F21600844206D14011C24981
:1084400008604FF416704860DFE041F21800844283
:1084500015D14FF4A060BC4908604FF448704860E3
:108460008C2088810A2008820881C88148820320E4
:1084700048811022A0210520FFF77CFEC5E04AF2CA
:108480000100844218D140F25650AF4908604FF4C1
:10849000407048608F20088146200882D52088815E
:1084A000032048811820C881032048821C22A02173
:1084B0000520FFF75FFEA8E04AF20200844217D1D0
:1084C0004011A14908604FF448704860202008819D
:1084D0003020088250208881062048810E20C881E3
:1084E000032048821622A0210520FFF743FE8CE0DE
:1084F0004AF20300844217D14011934908604FF4B7
:1085000040704860202008815020888130200882F7
:10851000072048810C20C881032048821722A0210F
:108520000520FFF727FE70E04AF20400844218D1CC
:108530004FF48060844908604FF4407048608820A0
:10854000088118200882A0208881062048811D20EB
:10855000C881032048821222A0210520FFF70AFECD
:1085600053E04AF20500844217D14FF45470764923
:1085700008604FF4F07048607020088188811020F6
:108580000882082048811720C881062048822F22AF
:10859000A0210520FFF7EEFD37E04AF206008442F5
:1085A00018D14FF44870684908604FF4167048605D
:1085B0008020088158208881282008820420488152
:1085C0001720C881012048822822A0210520FFF71A
:1085D000D1FD1AE04AF20700844216D180115A49AF
:1085E00008604FF4F070486060200881082008821D
:1085F00038208881022048812920C88102204882B1
:108600003E22A0210520FFF7B5FD4F4800884F49C5
:1086100008804D488088488002204B49C8614C48FA
:108620004C4908604C484D490860002048600021D2
:108630004A488160C160016141F21800844203D15F
:108640004FF08051454801613F480089401E434931
:1086500048613D484089401E88613B4800893A494D
:1086600089890844401E3D49C861374840893649D8
:10867000C9890844401E3949086233480089324993
:1086800089890844304909680844401E33494862D2
:108690002D4840892C49C98908442B494968084418
:1086A000401E2E4988622848008927498989084444
:1086B0002549096808442449098A0844401E274975
:1086C000C862214840892049C98908441E4949682F
:1086D00008441D49498A0844401E20490863002176
:1086E0001E4880F8361080F8351080F83410F8F7FE
:1086F00031FD002007210622CDE90002CDE902105C
:108700001448FF2302220168002000F02BF80E48D5
:10871000808880B200900C48008883B20022114605
:10872000104600F05DF80020FFF73CFD002000F04F
:10873000D7F8012220210A48F8F790FC4FF0FF30CB
:10874000FFF706FD1FBD0000FC070024E40600241F
:10875000000000C02800002400100050F40600248F
:10876000000402582DE9F04F8DB005460E4617461D
:108770009846DDE917ABDDF85890199C0020009071
:1087800002901548006801901348406803900497D0
:10879000CDF81480CDF818904FEA0A2007904FEAE0
:1087A0000B20089009960C4800680A900A48406817
:1087B0000B90002001148DF8321001128DF8311049
:1087C000E0B28DF830002A4669460448F8F792FC7A
:1087D0000DB0BDE8F08F0000FC070024F406002473
:1087E0002DE9F04104460E4617461D46DDF8188077
:1087F00023463A4631460548F8F7B8FD2346424637
:1088000029460248F8F7E8FDBDE8F081F4060024A7
:1088100010B586B0002400BF2E48006840F40070F8
:108820002C4908600846006800F40070009000BF02
:1088300000BF00BF0846006840F48060086008463A
:10884000006800F48060009000BF00BF40200190ED
:10885000002002900320049001A91F48F8F7CCFAE9
:108860004420019001A91D48F8F7C6FA40211A4892
:10887000F8F7E8FB044604211848F8F7E3FB44EA5C
:108880004000C4B240211548F8F7DCFB44EA800000
:10889000C4B21CB944F2423006B010BD012C02D162
:1088A00047F28400F8E7022C02D147F21600F3E702
:1088B000032C02D147F21800EEE7042C02D148F253
:1088C0001600E9E7052C02D141F21800E4E7002088
:1088D000E2E70000E0440258002402580028025851
:1088E0000149087570470000FC070024F0B500231B
:1088F000002400258E880768FF68C7F30B473E44B5
:10890000330406688436802707FB0266766806F41F
:108910007047066884364FF0800C0CFB0266776067
:108920000E680768FF68C7F30B473E44761C1E437A
:10893000076884370CFB02777E608E890768FF68C2
:10894000C7F30A073E44330406688436802707FBD2
:108950000266B66806F47047066884360CFB026649
:10896000B7608E680768FF68C7F30A073E44761C45
:108970001E43076884370CFB0277BE6006688436A6
:10898000802707FB0266366926F0070706688436EB
:108990000CFB026637610F69066884360CFB0266C1
:1089A00037613126765C33023226765C34040E7EE3
:1089B000350606688436802707FB0266B6690027FD
:1089C000066884360CFB0266B76191F830601E437E
:1089D00026432E43076884370CFB0277BE61066886
:1089E0008436802707FB0266766926F0FF07066853
:1089F00084360CFB026677614F69066884360CFB8F
:108A00000266776106688436802707FB0266F7698D
:108A100040F20776B743066884360CFB0266F761BE
:108A2000D1E907673E43076884370CFB0277FE6194
:108A300006688436802707FB0266B66A0027066848
:108A400084360CFB0266B7624F6A066884360CFBFC
:108A50000266B7620E690EB9042313E00E69012E97
:108A600001D103230EE00E69042E08D00E69022EF8
:108A700005D00E69032E02D00E69072E01D1022304
:108A800000E0012306688436802707FB0266F66A49
:108A900006F0E027066884364FF0800C0CFB026677
:108AA000F762D1E90076F61B5E43F71D0E8D5E433B
:108AB00047EA0647066884360CFB0266F7620668DA
:108AC0008436802707FB0266366BF70AFF020668CA
:108AD00084360CFB02663763CF6A066884360CFB6B
:108AE0000266376306688436D701F65946F00107F7
:108AF000066884364FEAC21C46F80C70F0BD0EB50D
:108B000000200121009103230A46CDE90110122122
:108B1000480600F00CF801200022CDE900200323D4
:108B2000022219210290980700F001F80EBD2DE9EC
:108B3000FF4704460D4616461F46DDE90D9ADDF84F
:108B40003080F8F7ADFC01208DF80000F0B28DF810
:108B500001000194E8B28DF8080000208DF80900AA
:108B60008DF80A008DF80B708DF80C008DF80D80D3
:108B70008DF80E908DF80FA06846F8F763FC04207E
:108B8000F8F7A4FC002004B0BDE8F08700BFFEE7C2
:108B90007047000010B50248F8F710FF10BD000044
:108BA000E40800242DE9F84F07460E46D7F8008068
:108BB00000240025A146A246C6EBC60107F13800F5
:108BC00000EB8104D4E90501451AA068A84200D24F
:108BD000A568E81CC11700EB91714FEAA1091AE0E2
:108BE000D4E90501451AA068A84200D2A568E81C8E
:108BF000C11700EB91714FEAA109387CABB2F2B218
:108C000000904046E16803F01FFAE0682844E06005
:108C1000A0692844A06108F5106000EB4610806947
:108C200080B2484506D9D4E90510884202D260696D
:108C30000028D5D1002D0CDC012000FA06FA40F600
:108C4000340050F8080020EA0A0040F6340141F8E8
:108C500008000020BDE8F88F10B586B0002400BFE2
:108C60001548006840F04000134908600846006855
:108C700000F04000009000BF00BF4FF48060019002
:108C800000200290012003900320049001A90B48CA
:108C9000F8F7B2F8FCF796F9FCF75EFA4020FCF71B
:108CA0001DFAFCF7ADFA0446FCF780FAFF2000F04D
:108CB0002BF8204606B010BDE044025800180258B8
:108CC00010B50024FCF748FA4120FCF707FAFCF73E
:108CD00097FA0020FCF7CCF90446FCF767FA204627
:108CE00010BD70B504460E46FFF7EAFF05461EB9F3
:108CF0000120A040854303E00120A0402843C5B2E5
:108D0000284600F001F870BD10B50446FCF724FABF
:108D10004020FCF7E3F9FCF773FA2046FCF7DEF994
:108D2000FCF76EFAFCF742FA0A2003F055FF10BD7B
:108D3000704700002DE9F04104460E4600274848E0
:108D4000006800F00300032802D10120BDE8F08193
:108D500043482838006820F080604149283908607D
:108D6000F8F782F9054606E0F8F77EF9401B02287D
:108D700001D90320EAE73A4828380068C0F3C06008
:108D80000028F1D100BF3648006820F47C3021680B
:108D900040EA013032490860A088401EC0F3080054
:108DA000A168491E4FF47E4202EA41210843A1898D
:108DB000491ED20102EA01410843217C491E1202E8
:108DC00002EA0161084326491031086000BF2448C7
:108DD000001D006820F0C000616908432049091D9A
:108DE00008600846006820F02000A16908431C497B
:108DF000091D08602EB90846006840F4002008608C
:108E000012E0012E08D11648001D006840F48010C1
:108E10001349091D086007E01148001D006840F46F
:108E200000100F49091D08600D482838006840F0FF
:108E300080600B4928390860F8F716F9054606E006
:108E4000F8F712F9401B022801D903207EE70448F5
:108E500028380068C0F3C0600028F1D0384675E7B4
:108E6000284402582DE9F04104460E4600274848A0
:108E7000006800F00300032802D10120BDE8F08162
:108E800043482838006820F080504149283908605C
:108E9000F8F7EAF8054606E0F8F7E6F8401B02287E
:108EA00001D90320EAE73A4828380068C0F3407047
:108EB0000028F1D100BF3648006820F07C7021887E
:108EC00040EA015032490860A088401EC0F3080003
:108ED000A168491E4FF47E4202EA41210843A1895C
:108EE000491ED20102EA01410843217C491E1202B7
:108EF00002EA0161084326491831086000BF24488E
:108F0000001D006820F44060616908432049091D84
:108F100008600846006820F40070A16908431C49F5
:108F2000091D08602EB90846006840F480000860FA
:108F300012E0012E08D11648001D006840F4000020
:108F40001349091D086007E01148001D006840F042
:108F500080700F49091D08600D482838006840F0EE
:108F600080500B4928390860F8F77EF8054606E07E
:108F7000F8F77AF8401B022801D903207EE704485D
:108F800028380068C0F340700028F1D0384675E7F3
:108F90002844025830B50A460446202300BF00BFCB
:108FA00000BFBFF34F8F00BF00BF00BF03E00B4DFA
:108FB0002C601C44D21A002AF9DC00BF00BF00BF9D
:108FC000BFF34F8F00BF00BF00BF00BF00BF00BF97
:108FD000BFF36F8F00BF00BF00BF30BD68EF00E080
:108FE00010B50023234C236000BF00BF00BFBFF3B8
:108FF0004F8F00BF00BF00BF231F1868C0F34E3162
:1090000000BFC0F3C90200BF43F6E07303EA411397
:109010004FF0404404EA82742343174C236000BF9E
:1090200000BF131EA2F10102EED10B1EA1F101013E
:10903000E7D100BF00BF00BFBFF34F8F00BF00BF2D
:1090400000BF0C4B703B1B6843F48033094C703CF1
:10905000236000BF00BF00BFBFF34F8F00BF00BF42
:1090600000BF00BF00BF00BFBFF36F8F00BF00BFD6
:1090700000BF10BD84ED00E060EF00E000BF00BF66
:1090800000BFBFF34F8F00BF00BF00BF00BF00BFD6
:1090900000BFBFF36F8F00BF00BF00BF00201449A7
:1090A000086000BF00BF00BFBFF34F8F00BF00BF0D
:1090B00000BF00BF00BF00BFBFF36F8F00BF00BF86
:1090C00000BF0C48006840F400300A49086000BF47
:1090D00000BF00BFBFF34F8F00BF00BF00BF00BF86
:1090E00000BF00BFBFF36F8F00BF00BF00BF70475E
:1090F00050EF00E014ED00E000B587B016481749C6
:109100000860002048600121144881600821C16086
:109110002021016140214161890081610021C161FB
:109120004FF4006101624900416200218162022026
:1091300000900820019006200290039002200490E5
:109140000590069069460548FAF78EFF034800F03F
:1091500007F807B000BD000040410052640600243B
:1091600070B505460024002301221146184600F080
:1091700021F84FF4FA7003F03BFD00230122022195
:10918000184600F017F8002308220321184600F0C3
:1091900011F840F22224234601220421002000F08D
:1091A00009F840F2A5210248FBF750F870BD000015
:1091B000640600242DE9FF4104460D4616461F466D
:1091C0004FF0000814B94FF0100803E0012C01D152
:1091D0004FF008080095CDF80480029603974FF6EB
:1091E000FF7269460448FBF745F818B9002004B03F
:1091F000BDE8F0810120FAE76406002410B51748A5
:10920000174908604FF480004860002114488160CD
:109210000721C1604FF0007101614910416189006F
:109220008161002141634FF0004141654FF0E04111
:10923000C16100210162416281620721C162FBF7C5
:1092400037F807480068006840F0010004490968E1
:109250000860FF2000F006F810BD00000038004054
:109260001C08002401B582B04FF47A70012301AAD2
:1092700002A900900248FBF78BF99DF804000EBD8F
:109280001C0800240F490968096821F001010D4AF2
:10929000126811600B490968896821F0E041094AA8
:1092A000126891600749096889680143054A126894
:1092B000916004490968096841F00101014A126896
:1092C000116070471C0800240268516902689269A5
:1092D00042F0080203689A610268926942F0100243
:1092E00003689A610268126822F0010203681A603A
:1092F0000268126940F26B339A4303681A6102688C
:10930000926822F4404203689A6090F88120042A0F
:109310000ED001F020025AB1D0F8842042F0800231
:10932000C0F884200268926942F0200203689A61C2
:1093300090F88120032A21D001F040025AB1D0F8E0
:10934000842042F00402C0F884200268926942F04E
:10935000400203689A61826AB2F5800F0ED101F073
:1093600080025AB1D0F8842042F00202C0F8842072
:109370000268926942F0800203689A6101F4007207
:109380005AB1D0F8842042F00102C0F8842002686B
:10939000926942F4007203689A6101F480725AB1D2
:1093A000D0F8842042F00802C0F884200268926954
:1093B00042F4807203689A610022A0F86220A0F84B
:1093C0006A20704710B501460124C86B04EB5013A6
:1093D000C868421CD01DC20802FB03F010BD2DE975
:1093E000F04106460C4617469846069D0BE0681C61
:1093F00048B12DB1F7F738FEA0EB0800A84202D91A
:109400000320BDE8F081306840692040A04201D1CE
:10941000012000E00020B842E9D00020F1E77047C9
:109420002DE9F0419CB080460C4615461E460027AB
:109430003948006820F004003749086000BF002068
:10944000009035480C30006840F4404032490C31FF
:1094500008600846006800F44040009000BF00BF6C
:1094600000BF2D480C30006800F40050B0F5005FDC
:10947000F7D1212001904FF4803002900120079015
:1094800000200490089002200A9002210B91CDF850
:1094900034800C940E950F960021129108211191A1
:1094A0000021139101A8FAF77DFA07460FB100BF1A
:1094B000FEE73F201490032015900020169008200E
:1094C00017904020199000011A90402018905020C9
:1094D0001B90022114A8F9F7D3FF07460FB100BF74
:1094E000FEE70E48006840F080000C49086000BFAD
:1094F0000A48F430006840F002000849F43108607E
:109500000846006800F00200009000BF00BFF7F7B7
:1095100069FC1CB0BDE8F0810C48025800440258B8
:1095200010B5F7F7A7FD10BD2048006840F47000A3
:109530001E4908601E48006840F001001C49086090
:1095400000201B491031086019480068194908407B
:10955000174908600020164918310860091D086085
:10956000091D0860124928310860091D0860091D9D
:109570000860091D0860091D0860091D0860091DB3
:109580000860091D08600A48006820F48020084926
:109590000860002006496031086001200649086023
:1095A000C0060249803908607047000088ED00E07D
:1095B000004402587FEDF6EA0881005110B50E48CC
:1095C0000068C06800F0010078B10C490869804764
:1095D000002009490968486200BF642006490968FB
:1095E000C86264210448C16000BF6FF001000249F5
:1095F0000968086110BD0000A40800246000002470
:1096000010B500220288294B98420ED0B0F1804F4D
:109610000BD0274B984208D0264B984205D0264BBA
:10962000984202D0254B984203D122F070024B6839
:109630001A431E4B984217D0B0F1804F14D01C4BE8
:10964000984211D01B4B98420ED01B4B98420BD026
:109650001A4B984208D01A4B984205D0194B9842A1
:1096600002D0194B984203D122F44072CB681A43BE
:1096700022F080034C6943EA040202808B68C362D3
:109680000B880385094B98420BD00C4B984208D0AD
:109690000B4B984205D00B4B984202D00A4B984294
:1096A00001D10B8A03860123436110BD00000140F4
:1096B0000004004000080040000C0040000401408D
:1096C00000400140004401400048014038B50446D4
:1096D0000D4600BF1148006840F004000F490860C3
:1096E0000846006800F00400009000BF00BF03229D
:1096F00011461E20F7F71BFF1E20F7F708FF08484A
:10970000084908600846456000218160C460016125
:10971000FBF7DAF90348FBF7F2F938BDE8440258E1
:1097200000080040A408002490F8341001F0010162
:1097300039B10168496821F40031826B1143026834
:10974000516090F8341001F0020139B101684968A4
:1097500021F48031C26B11430268516090F83410DB
:1097600001F0040139B10168496821F48021026CDB
:1097700011430268516090F8341001F0080139B1CA
:109780000168496821F40041426C1143026851604C
:1097900090F8341001F0100139B10168896821F4A2
:1097A0008051826C11430268916090F8341001F08E
:1097B000200139B10168896821F40051C26C11435C
:1097C0000268916090F8341001F0400199B101688D
:1097D000496821F48011026D114302685160016DE6
:1097E000B1F5801F07D10168496821F4C001426DBD
:1097F00011430268516090F8341001F0800139B1D2
:109800000168496821F40021826D114302685160AA
:10981000704738B5044600250020E067F7F724FCC0
:1098200005462068006800F0080008280CD16FF099
:109830007E402B4600224FF400110090204600F09D
:10984000A6FD08B1032038BD2068006800F00400C0
:1098500004280CD16FF07E402B4600224FF480018B
:109860000090204600F093FD08B10320EBE7202094
:1098700084F8790084F87A0000BF002084F878002A
:1098800000BF00BFDFE770B50546AC6B0020A4F851
:109890006A00A4F862002046FBF741F970BD016838
:1098A000096821F49071026811600168896821F0EB
:1098B000010102689160202180F87A10704710B58C
:1098C00004462068006820F04000216808602020DD
:1098D00084F879002046FBF747FB002010BD2DE9F6
:1098E000F0410446B4F86C7094F87A00222833D121
:1098F0002068858CA068B0F5805F09D1206938B9EF
:10990000666E05EA07003080606E801C606605E0C8
:10991000F8B22840626E511C61661070B4F86A009B
:10992000401E80B2A4F86A00A0B92068006820F444
:109930009070216808602068806820F0010021682C
:109940008860202084F87A002046FBF7C9FA0020BE
:10995000BDE8F0810020FBE72068008B40F00800A4
:10996000216808830220F3E72DE9F04F89B004460F
:1099700000254FF08008A946AA4600200890FA4921
:109980002068884201D1012000E0002000B100E001
:1099900000BFA06AB0F1005F00D100BF2169A068DC
:1099A000084361690843E16940EA0105A06A05438B
:1099B00020680068ED490840284321680860206855
:1099C000406820F44050E168084321684860A56978
:1099D000E5492068884201D1012000E0002008B953
:1099E000206A0543A06AB0F1005F03D1D4E90B01FE
:1099F0000843054320688068DD4908402843216802
:109A000088602068C06A20F00F00616A08432168FE
:109A1000C86200BFD7492068884224D1D648006870
:109A200000F03800182814D005DC48B108280AD006
:109A3000102817D10AE020280ED0282812D10EE0D5
:109A40004FF001080EE04FF004080BE04FF0400823
:109A500008E04FF0080805E04FF0100802E04FF072
:109A6000200800BF17E1C549206888421DD1C248BF
:109A7000006800F00700062816D2DFE800F00306B1
:109A8000090C0F124FF000080EE04FF004080BE035
:109A90004FF0400808E04FF0080805E04FF01008CC
:109AA00002E04FF0200800BFF5E0B5492068884289
:109AB0001DD1B148006800F00700062816D2DFE883
:109AC00000F00306090C0F124FF000080EE04FF0F3
:109AD00004080BE04FF0400808E04FF0080805E0EC
:109AE0004FF0100802E04FF0200800BFD3E0A54976
:109AF000206888421DD1A048006800F007000628B1
:109B000016D2DFE800F00306090C0F124FF0000830
:109B10000EE04FF004080BE04FF0400808E04FF073
:109B2000080805E04FF0100802E04FF0200800BFE1
:109B3000B1E09549206888421DD18F48006800F047
:109B40000700062816D2DFE800F00306090C0F1202
:109B50004FF000080EE04FF004080BE04FF0400813
:109B600008E04FF0080805E04FF0100802E04FF061
:109B7000200800BF8FE085492068884224D17E48B4
:109B8000006800F03800182814D005DC48B1082817
:109B90000AD0102817D10AE020280ED0282812D188
:109BA0000EE04FF001080EE04FF004080BE04FF01C
:109BB000400808E04FF0080805E04FF0100802E008
:109BC0004FF0200800BF66E07149206888421DD12F
:109BD0006948006800F00700062816D2DFE800F0A8
:109BE0000306090C0F124FF000080EE04FF00408B6
:109BF0000BE04FF0400808E04FF0080805E04FF098
:109C0000100802E04FF0200800BF44E061492068DE
:109C100088421DD15848006800F00700062816D277
:109C2000DFE800F00306090C0F124FF000080EE009
:109C30004FF004080BE04FF0400808E04FF0080830
:109C400005E04FF0100802E04FF0200800BF22E0CE
:109C50004549206888421ED14748001D006800F031
:109C60000700062816D2DFE800F00306090C0F12E1
:109C70004FF002080EE04FF004080BE04FF04008F0
:109C800008E04FF0080805E04FF0100802E04FF040
:109C9000200800BF00BF00BF33492068884201D1BF
:109CA000012000E0002000285DD00025B8F1100F51
:109CB00033D009DCB8F1020F10D0B8F1040F11D085
:109CC000B8F1080F2ED117E0B8F1200F27D0B8F166
:109CD000400F0CD0B8F1800F24D124E0F8F7F2FB4C
:109CE000054623E005A8F8F703FC069D1EE002A840
:109CF000F8F714FD039D19E01F4854380068C0F3BD
:109D0000401040B11C4854380068C0F3C1012248DB
:109D100020FA01F500E0204D08E0204D06E04FF468
:109D2000004503E000BF0120089000BF00BF002DE8
:109D30000AD0606800EB4000A84203D860680003C6
:109D4000A84202D201200890D4E2B8F1100F7CD0D2
:109D500026DCB8F1020F2DD0B8F1040F52D0B8F1C3
:109D6000080F73D19EE03FE1000C0058F369FFCF6C
:109D7000FFF4FF1100100140544402580044004019
:109D800000480040004C00400050004000140140DA
:109D900000780040007C00400090D00300093D00A6
:109DA000B8F1200F7DD0B8F1400F54D0B8F1800F3A
:109DB000D7D109E1F8F786FB00270646FB49606A20
:109DC00031F810C062463B4630463946F6F780FA15
:109DD0004FF4807600220346A3FB060701FB0671C1
:109DE00003FB021361684908064671185A41CDE920
:109DF000001266683246002308460199F6F768FAB1
:109E00000546E4E005A8F8F773FBDDF818C0E7495C
:109E1000606A31F810B05A46002360461946F6F7DA
:109E200057FA4FF4807C0022A0FB0C3B01FB0CB1E5
:109E300000FB0210616849085E1840EB0201D4F88B
:109E400004C062460023304601E079E0BBE0F6F74B
:109E50003FFA0546BBE002A8F8F760FCDDF80CC04D
:109E6000D249606A31F810B05A460023604619465C
:109E7000F6F72EFA4FF4807C0022A0FB0C3B01FB8E
:109E80000CB100FB0210616849085E1840EB02014A
:109E9000D4F804C0624600233046F6F719FA0546A6
:109EA00095E06EE0C2480068C0F3401038B3C04887
:109EB0000068C0F3C101BF4820FA01FCBB49606AD9
:109EC00031F810B05A46002360461946F6F700FAFA
:109ED0004FF4807C0022A0FB0C3B01FB0CB100FB8B
:109EE0000210616849085E1840EB0201D4F804C012
:109EF000624600233046F6F7EBF905461FE0AB4912
:109F0000606A31F810C062460023AA481946F6F785
:109F1000DFF94FF4807C0022A0FB0C3B01FB0CB16D
:109F200000FB0210616849085E1840EB0201D4F89A
:109F300004C0624600233046F6F7CAF9054646E0FB
:109F40009A49606A31F810C0624600239A4819465F
:109F5000F6F7BEF94FF4807C0022A0FB0C3B01FB1E
:109F60000CB100FB0210616849085E1840EB020169
:109F7000D4F804C0624600233046F6F7A9F9054636
:109F800025E08A49606A31F810C0624600234FF428
:109F900000401946F6F79CF94FF4807C0022A0FBA4
:109FA0000C3B01FB0CB100FB0210616849085E1814
:109FB00040EB0201D4F804C0624600233046F6F7B5
:109FC00087F9054603E000BF0120089000BF00BFED
:109FD000B5F5407F05D3B5F5801F02D22068C56076
:109FE00088E10120089085E1E069B0F5004F7CD15F
:109FF000B8F1100F7AD00CDCB8F1000F13D0B8F123
:10A00000010F21D0B8F1040F2FD0B8F1080F6ED195
:10A0100051E0B8F1200F6BD0B8F1400F38D0B8F153
:10A02000800F64D197E0F9F76FFB604A616A32F8FC
:10A030001110B0FBF1F04000616800EB5100B0FB83
:10A04000F1F01FFA80FA89E0F9F774FB574A616A68
:10A0500032F81110B0FBF1F04000616800EB5100E4
:10A06000B0FBF1F01FFA80FA78E005A8F8F740FAA3
:10A0700006994E4A606A32F81000B1FBF0F04000D9
:10A08000616800EB5100B0FBF1F01FFA80FA65E067
:10A0900002A8F8F743FB0399444A606A32F81000BB
:10A0A000B1FBF0F04000616800EB5100B0FBF1F053
:10A0B0001FFA80FA52E03E480068C0F34010C0B179
:10A0C0003B480068C0F3C1013A48C840374A616A5A
:10A0D00032F81110B0FBF1F04000616800EB510064
:10A0E000B0FBF1F01FFA80FA12E044E011E031E039
:10A0F0001FE02E49606A31F810002E49B1FBF0F0E4
:10A100004000616800EB5100B0FBF1F01FFA80FAEB
:10A1100024E02649606A31F810002749B1FBF0F0CD
:10A120004000616800EB5100B0FBF1F01FFA80FACB
:10A1300014E01E49606A31F810004FF40041B1FB91
:10A14000F0F04000616800EB5100B0FBF1F01FFA45
:10A1500080FA03E000BF0120089000BF00BF4FF667
:10A16000F0700AEA0009CAF3420049EA00092068CF
:10A17000C0F80C90BEE0B8F1100F7CD00CDCB8F148
:10A18000000F1BD0B8F1010F29D0B8F1040F37D060
:10A19000B8F1080F70D159E0B8F1200F6DD0B8F1C7
:10A1A000400F40D0B8F1800F66D19FE034E3000843
:10A1B000004402580090D00300093D00F9F7A4FACA
:10A1C0004E4A616A32F81110B0FBF1F0616800EBA1
:10A1D0005100B0FBF1F080B22168C86089E0F9F766
:10A1E000A9FA464A616A32F81110B0FBF1F06168D1
:10A1F00000EB5100B0FBF1F080B22168C86078E05C
:10A2000005A8F8F775F906993C4A606A32F810001B
:10A21000B1FBF0F0616800EB5100B0FBF1F080B2EF
:10A220002168C86065E002A8F8F778FA0399334A14
:10A23000606A32F81000B1FBF0F0616800EB510089
:10A24000B0FBF1F080B22168C86052E02C48006891
:10A25000C0F34010C0B12A480068C0F3C1012948CA
:10A26000C840264A616A32F81110B0FBF1F061680B
:10A2700000EB510002E017E037E025E0B0FBF1F021
:10A2800080B22168C8600EE01C49606A31F8100095
:10A290001C49B1FBF0F0616800EB5100B0FBF1F03C
:10A2A00080B22168C86024E01449606A31F8100067
:10A2B0001549B1FBF0F0616800EB5100B0FBF1F023
:10A2C00080B22168C86014E00C49606A31F810005F
:10A2D0004FF40041B1FBF0F0616800EB5100B0FBBE
:10A2E000F1F080B22168C86003E000BF012008904F
:10A2F00000BF00BF089809B0BDE8F08F34E3000844
:10A30000004402580090D00300093D00014691F836
:10A310007900212839D1B1F86200C8B9086800680D
:10A3200000F0005030B10868806820F400000B682D
:10A33000986005E00868006820F080000B681860ED
:10A340000868006840F040000B6818600020704703
:10A350008868B0F5805F0BD1086948B9CA6D10886C
:10A36000C0F308000B681885C86D801CC86505E03F
:10A37000CB6D581CC86518780B681885B1F8620059
:10A38000401EA1F862000020E1E70220DFE72DE98E
:10A39000F04104460D4617469846069E21E0701C83
:10A3A000F8B12EB1F6F760FEA0EB0800B04218D964
:10A3B0002068006820F4D0702168086020688068F8
:10A3C00020F0010021688860202084F8790084F85A
:10A3D0007A0000BF002084F8780000BF0320BDE8A9
:10A3E000F0812068C0692840A84201D1012000E026
:10A3F0000020B842D3D00020F1E7000070B500245F
:10A400000F4D1048FAF796FB00BF03E0641CAC4206
:10A4100000D904E00B48FAF783FB2028F6D100BFEF
:10A42000002403E0641CAC4200D906E00122064986
:10A430000448FAF7E5FC0028F4D100BF70BD000025
:10A44000FFFF0100E40500241200002402460B4631
:10A45000D2F81812D2F8180218B10020C1F814026C
:10A4600070470220FCE770B504460E46D4F8185237
:10A470003146204600F014FCC5F80C02D4F818024E
:10A4800048B1D5F80402D4F81C12CA6805F5037166
:10A490009047002070BD0220FCE770B504460E46D0
:10A4A00000258121204600F031FB0121204600F0EB
:10A4B0002DFB8221204600F029FBD4F8180258B168
:10A4C000D4F81C12486880470020D4F8181202F013
:10A4D00007FE0020C4F81802284670BD70B5054676
:10A4E000D5F81842D5F81C0278B194F80002FF287C
:10A4F0000BD094F8012294F80002D5F81C128B6856
:10A5000021469847FF2084F80002002070BD00001B
:10A5100001460A20088001487047000054010024C9
:10A52000014643200880014870470000DC010024F8
:10A53000014643200880014870470000980100242C
:10A540000146432008800148704700002002002493
:10A550002DE9F04104460F460026207C70B94FF4E7
:10A56000007302228121204600F0F8FB4FF40073B3
:10A5700002220121204600F0F1FB0BE040230222E1
:10A580008121204600F0EAFB4023022201212046DF
:10A5900000F0E4FB082303228221204600F0DEFBCA
:10A5A0004FF40771002002F0ADFDC4F81802D4F892
:10A5B000180208B901261CE0D4F81852D4F81C126D
:10A5C000086880470020C5F81402C5F81802207CEE
:10A5D00040B94FF4007301212046D5F8042200F061
:10A5E000CDFB06E0402301212046D5F8042200F0EF
:10A5F000C5FB3046BDE8F08170B50446D4F818526A
:10A60000D4F8180298B1207C40B94FF400730121AE
:10A610002046D5F8042200F0B1FB06E040230121DA
:10A620002046D5F8042200F0A9FB002070BD0220CE
:10A63000FCE70246022011B1C2F81C12002070474C
:10A640000246D2F81832C3F804120020704710B541
:10A650000346D3F81842C4F80812C4F810220020A8
:10A6600010BD000070B505460C46D5F8186220787C
:10A6700000F0600040B3202835D1E088E0B12078B8
:10A6800000F0800060B1E2886078D5F81C128B6819
:10A6900031469847E2883146284600F0B9F812E082
:10A6A000607886F80002A07986F80102E2883146D7
:10A6B000284600F08CF806E06078D5F81C120022DD
:10A6C0008B68214698470FE060780A2802D00B2853
:10A6D00007D105E001220649284600F099F800E07C
:10A6E00000BF00BF00BF00BF00BF002070BD000062
:10A6F0006302002470B50546D5F81842D5F8180253
:10A7000090B1D4F8140268B90120C4F81402B4F866
:10A71000100283B281212846D4F8082200F0DFFB22
:10A72000002070BD0120FCE70220FAE770B5044666
:10A730000D46D4F81402294642682046904700206E
:10A7400070BD70B504460D4694F8FC01022802D095
:10A75000032811D100E000BF688801280BD1002038
:10A76000C4F80402D4F814022946826820469047AF
:10A77000204600F05EF804E02946204600F01BF871
:10A7800000BF00BF70BD70B506460C4615462B468F
:10A7900022460021304600F0F1FA002070BD70B56D
:10A7A00006460C4615462B4622460021304600F050
:10A7B00096FB002070BD70B504460D4680212046F2
:10A7C00000F071FB0021204600F06DFB70BD70B5FC
:10A7D00004460E4615460320C4F8F4014FF4847075
:10A7E0000551001D05512B4632460021204600F040
:10A7F000C5FA002070BD10B504460520C4F8F40168
:10A8000000231A461946204600F0B8FA002010BD71
:10A8100070B504460E4615460220C4F8F401A56141
:10A82000E5612B4632460021204600F058FB00200F
:10A8300070BD10B504460420C4F8F40100231A4684
:10A840001946204600F04BFB002010BD70B50446B1
:10A850000D46E888012804D029462046FFF7ABFFC3
:10A860001BE094F8FC01022802D003280FD108E075
:10A870000020A060012204F108012046FFF7C8FF74
:10A880000AE00122211D2046FFF7C2FF04E029460D
:10A890002046FFF790FF00BF00BF70BDF8B504462B
:10A8A0000E467088001208287FD2DFE800F07E0490
:10A8B0000C207E7E5F6D207CD4F810120A686946F9
:10A8C0009047054676E0207C40B9D4F81402816AAE
:10A8D0006846884705460221697007E0D4F81402EB
:10A8E000C16A6846884705460221697062E0B0780F
:10A8F000062834D2DFE800F0030B131B232B207C47
:10A90000D4F810124A686946904705462CE0207C2E
:10A91000D4F810128A6869469047054624E0207CE6
:10A92000D4F81012CA686946904705461CE0207C9E
:10A93000D4F810120A6969469047054614E0207C55
:10A94000D4F810124A696946904705460CE0207C0D
:10A95000D4F810128A6969469047054604E03146EA
:10A960002046FFF728FFF8BD00BF23E0207C30B968
:10A97000D4F81402416B6846884705461AE0314610
:10A980002046FFF718FFEEE7207C48B9D4F8140200
:10A99000016B684688470546072169700AE004E0B4
:10A9A00031462046FFF707FFDDE731462046FFF737
:10A9B00002FFD8E700BFBDF8000088B1F08878B189
:10A9C000F088BDF80010884202DDBDF8000000E00C
:10A9D000F0880090BDF8002029462046FFF718FFB8
:10A9E00000BFC0E70146002002E0421CD0B2491C73
:10A9F0000A78002AF9D1704770B504460D4694F8DC
:10AA0000FC01022802D0032811D100E000BF012080
:10AA1000E060D4F8040218B1E06840F00200E060A1
:10AA2000022204F10C012046FFF7F2FE04E0294661
:10AA30002046FFF7C0FE00BF00BF70BD2DE9F0410A
:10AA400004460D4617460026FCB12046FFF7CAFF14
:10AA5000022101EB400038803A783046711CCEB2BA
:10AA60002A5403223046711CCEB22A540AE014F84C
:10AA7000012B3046711CCEB22A5400223046711C84
:10AA8000CEB22A5420780028F1D1BDE8F081000030
:10AA900070B504460D46164654B90EA001F0E6FB0B
:10AAA0000EA001F0E3FB13A001F0E0FB022070BD5B
:10AAB000D4F8140210B10020C4F814020DB1C4F887
:10AAC0001052012084F8FC012670204600F0F2F8B4
:10AAD0000020ECE74552524F523A2000496E766111
:10AAE0006C6964204465766963652068616E646C96
:10AAF000650000000D0A000070B504460D462946A9
:10AB0000D4F82002F6F738FE002070BD70B5044678
:10AB10000D462946D4F82002F6F7F8FD002070BD56
:10AB20002DE9F04104460E461746002E54D104F19B
:10AB30001405D4F8F401022843D1D5E90201884272
:10AB400010D9D5E90201401AA860288982B2394695
:10AB50002046FFF724FE00231A461946204600F03F
:10AB60000DF92EE0E9686868B0FBF1F201FB120014
:10AB7000B8B9E9686868884213D36868D4F8F811EE
:10AB800088420ED2002211462046FFF708FE002020
:10AB9000C4F8F80100231A461946204600F0EEF8E2
:10ABA0000FE0D4F81402C06840B194F8FC01032807
:10ABB00004D1D4F81402C168204688472046FFF724
:10ABC0001AFE94F80002012814D1204600F0D2F9B0
:10ABD000002084F800020DE0D4F81402406948B166
:10ABE00094F8FC01032805D1D4F8140231464269D7
:10ABF000204690470020BDE8F0812DE9F041054650
:10AC00000E4617465EBB05F58274D5F8F40103289D
:10AC100033D1D4E90201884210D9D4E90201401AA3
:10AC2000A060D4E90201884201D2A06800E0E06897
:10AC300082B239462846FFF7A6FD1EE0D5F8140279
:10AC4000006940B195F8FC01032804D1D5F814023D
:10AC50000169284688472846FFF7EBFD0DE0D5F847
:10AC60001402806948B195F8FC01032805D1D5F894
:10AC7000140231468269284690470020BDE8F081E1
:10AC800001460020704710B50446012084F8FC01FD
:10AC90002179D4F81402426820469047002010BD64
:10ACA00070B504460D462946D4F82002F6F799FD02
:10ACB00070BD000010B5044615481649086008200C
:10ACC0004860002113480163402141610021016275
:10ACD000022181610021C1610221C1600021C162A4
:10ACE0008162C0F8FC43C4F82002F7F711FA802112
:10ACF0000848F6F792FC402200210648F6F792FC3D
:10AD0000802201210348F6F78DFC002010BD0000D1
:10AD100000000840E408002410B50246D2F82032B2
:10AD200001F08000802809D101F07F00C0EBC00451
:10AD300003F1380000EB8400807810BD01F07F0043
:10AD4000C0EBC00403F5FC7000EB84008078F4E7EE
:10AD50000246002070470246002070472DE9F0416E
:10AD600004460F4615461E462B4632463946D4F851
:10AD70002002F6F742FD0020BDE8F0812DE9F04108
:10AD800004460D4616461F463B4632462946D4F831
:10AD90002002F6F779FD0020BDE8F08110B50446E9
:10ADA0004023002211462046FFF7D8FF40214FF4F0
:10ADB000887001514023002280212046FFF7CEFFFA
:10ADC00040212162012084F8FC01D4F8180228B146
:10ADD0002179D4F81402426820469047002010BD23
:10ADE000014691F8FD0181F8FC010020704710B583
:10ADF000044694F8FC01032808D1D4F81402C06971
:10AE000020B1D4F81402C16920468847002010BD43
:10AE1000024611740020704770B504460D460120AB
:10AE2000044908702946D4F82002F7F7DAFA00201E
:10AE300070BD00006502002470B504460D46294629
:10AE400004F5027000F05BF80120C4F8F40140F250
:10AE50000E20005BC4F8F80194F8080200F01F000F
:10AE600020B1012808D0022812D10BE004F50271AC
:10AE7000204600F046F913E004F50271204600F088
:10AE800024FA0DE004F50271204600F073F907E0A2
:10AE900094F8080200F08001204600F004F800BF9A
:10AEA00000BF002070BD70B504460D462946D4F899
:10AEB0002002F6F716FD002070BD10B50446D4F848
:10AEC0002002F7F7B0FA002010BD014691F8FC010E
:10AED00081F8FD01042081F8FC01002070472DE974
:10AEE000F04104460D4616461F463B46324629466B
:10AEF000D4F82002F6F733FD0020BDE8F0810A788F
:10AF000002704A7842708B78CA7803EB0222428042
:10AF10000B794A7903EB022282808B79CA7903EBA1
:10AF20000222C2807047000070B505460C4600261C
:10AF300014B1C5F8144209E005A001F097F906A084
:10AF400001F094F90AA001F091F90226304670BD93
:10AF50004552524F523A2000496E76616C69642026
:10AF6000436C6173732068616E646C65000000005F
:10AF70000D0A000001460020704770B504460D46DA
:10AF8000A888F8B9E888E8B9A87800F07F0694F8AE
:10AF9000FC01032804D129462046FFF70CFC15E0EC
:10AFA00084F8FE6131462046FFF736FF2046FFF762
:10AFB00040FC1EB1022084F8FC0107E0012084F867
:10AFC000FC0103E029462046FFF7F5FB70BD70B594
:10AFD00004460D460226D4F8140238B1D4F81402FF
:10AFE000294602682046904700B90026304670BDC9
:10AFF00070B504460D46A8783449087008460078B4
:10B00000012804DD29462046FFF7D5FB5BE094F8D4
:10B01000FC01022802D003284FD11CE02B48007805
:10B02000A8B12A4800786060032084F8FC01274812
:10B0300001782046FFF7CBFF022804D1294620469D
:10B04000FFF7B9FB70BD2046FFF7F3FB02E0204697
:10B05000FFF7EFFB36E01D48007870B9022084F856
:10B06000FC011A4800786060184801782046FFF714
:10B070005DFB2046FFF7DDFB1EE0144909786068A0
:10B08000884216D021792046FFF750FB0F48007800
:10B0900060600E4801782046FFF799FF022804D12E
:10B0A00029462046FFF787FBCCE72046FFF7C1FB88
:10B0B00002E02046FFF7BDFB04E029462046FFF7EB
:10B0C0007AFB00BF00BF00BFBCE7000064020024A1
:10B0D00070B504460D46688801280AD1C4F80402F8
:10B0E000D4F8140229468268204690472046FFF78C
:10B0F000A0FB70BD10B504462046FFF7DEFE002021
:10B1000010BD70B505460C46002660780A2829D285
:10B11000DFE800F01923281E280A0528140F21460D
:10B120002846FFF7BBFB22E021462846FFF725FF14
:10B130001DE021462846FFF75BFF18E02146284620
:10B14000FFF784FB13E021462846FFF755FC0EE08D
:10B1500021462846FFF7BCFF09E021462846FFF7B5
:10B16000F0FA04E021462846FFF725FB00BF00BFA8
:10B17000304670BD2DE9F04105460E464FF00008FF
:10B180003479307800F06000202808D1D5F8140216
:10B1900031468268284690470020BDE8F0817078EB
:10B1A000002855D001282AD003287AD195F8FC012F
:10B1B000022802D003281BD107E02CB1802C03D039
:10B1C00021462846FFF76FFE17E0708830B92CB192
:10B1D000802C03D021462846FFF765FED5F81402DF
:10B1E00031468268284690472846FFF722FB04E054
:10B1F00031462846FFF7DFFA00BF00BF62E095F84E
:10B20000FC01022802D003281BD107E02CB1802CBE
:10B2100003D021462846FFF746FE17E0708878B92C
:10B2200004F07F0048B121462846FFF765FCD5F8B9
:10B23000140231468268284690472846FFF7F9FAFB
:10B2400004E031462846FFF7B6FA00BF00BF39E0F8
:10B2500095F8FC01022802D003282BD107E004F066
:10B260007F0018B121462846FFF71DFE27E004F0B5
:10B270008000802806D104F07F0105F1140000EB66
:10B28000011005E004F07F0105F5827000EB01106C
:10B29000074621462846FFF73FFD18B101203860D8
:10B2A00002E00EE000203860022239462846FFF70F
:10B2B000AFFA04E031462846FFF77DFA00BF00BF31
:10B2C00000E000BF00BF404667E770B504460D468A
:10B2D000002694F8FC01032814D1287901280CDCFD
:10B2E000D4F814022946826820469047E88840B97D
:10B2F0003EB92046FFF79DFA03E029462046FFF7B6
:10B300005AFA04E029462046FFF755FA00BF00BF6D
:10B31000002070BD70B505460C462DB92246064981
:10B3200006A0FFF78BFB04E02246034903A0FFF7CA
:10B3300085FB014870BD0000E40C002456435020FA
:10B34000436F6E666967000002461220088001485C
:10B35000704700008402002470B505460C462DB9E4
:10B360002246064906A0FFF769FB04E0224603498E
:10B3700003A0FFF763FB014870BD0000E40C00244C
:10B3800056435020496E7465726661636500000023
:10B3900002460420088001487047000098020024FB
:10B3A00070B505460C462246024903A0FFF746FB4E
:10B3B000004870BDE40C002453544D6963726F65FE
:10B3C0006C656374726F6E696373000070B50546D7
:10B3D0000C462DB92246064906A0FFF72FFB04E0D4
:10B3E000224603490CA0FFF729FB014870BD00006D
:10B3F000E40C002453544D33322056697274756145
:10B400006C20436F6D506F727420696E204853201A
:10B410004D6F64650000000053544D33322056696F
:10B42000727475616C20436F6D506F727420696E19
:10B43000204653204D6F64650000000070B505463E
:10B440000C461A202080F5F729FC014870BD000049
:10B450009C02002410B50246487801282BD140F602
:10B460001C0080580C780123A3409BB2184340F67F
:10B470001C039850087802F5106303EB4010006835
:10B4800000F40040F0BB0889C0F30A00CB7840EA22
:10B4900083400B7840EA835040F0805040F40040F5
:10B4A00002F5106404EB43131B6818430B7804EB9C
:10B4B000431318602CE040F61C0080580C780123E0
:10B4C000A340144C04EA0343184340F61C0398506D
:10B4D000087802F5306303EB4010006800F4004088
:10B4E00080B90889C0F30A00CB7840EA834040F075
:10B4F000805040F400400B7802F5306404EB4313B5
:10B500001B6800E004E018430B7804EB4313186059
:10B51000002010BD0000FFFF01464FF410604058AE
:10B52000C20AD2024FF41060425040F60800405860
:10B5300000F00600042807D14FF41060405840F096
:10B5400003024FF41060425040F60400405840F4AB
:10B55000807240F604004250002070470FB410B5CE
:10B5600004460898012816D1A06B20F48030A0630F
:10B57000E06815490840E060E06820F44010E060B1
:10B580000F98012803D1E06840F48010E060204665
:10B5900000F01CF809E0E06840F04000E060204660
:10B5A00000F014F84FF48030A0630698012807D10A
:10B5B000A06840F00C00A060A06840F02000A060EF
:10B5C000002010BC5DF814FBBFFFBDFF0146002248
:10B5D00000BF501C02460F4B984201D90320704710
:10B5E000086900F000400028F3D00022086940F00C
:10B5F0000100086100BF501C0246064B984201D969
:10B600000320ECE7086900F001000028F3D100BF37
:10B61000E5E70000400D030010B502464878012818
:10B6200022D140F63C0080580C780123A3409BB205
:10B63000984340F63C03985040F61C0080580C7824
:10B640000123A3409BB2984340F61C03985008780E
:10B6500002F5106303EB4010006820F40044087802
:10B6600003EB4010046026E040F63C0080580C7864
:10B670000123A340114C04EA0343984340F63C03E2
:10B68000985040F61C0083580C780120A0400B4CC9
:10B6900004EA004023EA000040F61C0398500878B2
:10B6A00002F5306303EB4010006820F40044087892
:10B6B00003EB40100460002010BD00000000FFFFFD
:10B6C00010B5044640F60400005920F0020140F68F
:10B6D000040001510320F5F771FB002010BD10B5E7
:10B6E000044640F60400005940F0020140F6040010
:10B6F00001510320F5F762FB002010BD0FB430B5F7
:10B7000004460025A06B40F40010A0630E9858B9C1
:10B71000A06B20F40010A063206840F0400020607F
:10B72000206840F0800020600020C4F8000ED4F8AB
:10B730000008C4F80008099801280BD1069820B920
:10B740000021204600F078FC08E00121204600F0AE
:10B7500073FC03E00321204600F06EFC102120461C
:10B7600000F0B4FB204600F09BFB00214FF4016089
:10B770000151001D0151491E001D01510021001DF4
:10B780000151002524E004F5106000EB451000682D
:10B7900000F00040B0F1004F07D14FF0904104F5A8
:10B7A000106000EB4510016005E0002104F5106019
:10B7B00000EB45100160002104F5106000EB45101E
:10B7C0000161FF2104F5106000EB451081606D1CE4
:10B7D0000498A842D7D8002524E004F5306000EB97
:10B7E0004510006800F00040B0F1004F07D14FF065
:10B7F000904104F5306000EB4510016005E0002148
:10B8000004F5306000EB45100160002104F5306064
:10B8100000EB45100161FF2104F5306000EB45109D
:10B8200081606D1C0498A842D7D84FF4016000597C
:10B8300020F480714FF401600151079801280BD169
:10B8400015494FF4036001510059144908434FF45E
:10B8500003610851084605590020A0616FF080403F
:10B860006061079818B9A06940F01000A061A06954
:10B870000B490843A0610A9818B1A06940F008007C
:10B88000A0610E98012803D1A06906490843A06170
:10B89000002030BC5DF814FB000400020300010826
:10B8A00000383C80040000400146886820F0010018
:10B8B000886000207047000030B5034648780128B2
:10B8C0007DD1486918BB087803F5106404EB40107B
:10B8D0000069644C20400C7803F5106505EB4414B6
:10B8E000206108782C4604EB4010006940F40025E4
:10B8F000087804EB40100561087804EB40100069FB
:10B90000C50CED04087804EB4010056137E00878B9
:10B9100003F5106404EB40100069C50CED040878D1
:10B9200004EB40100561087804EB401004694D48B1
:10B930000440087803F5106505EB401004618C683D
:10B940004869A04201D988684861087803F5106405
:10B9500004EB4010006940F40025087804EB401027
:10B960000561087804EB401004694869C0F31200CF
:10B970000443087803F5106505EB40100461012AC3
:10B9800007D1087803F5106404EB40100D69456198
:10B990000BE0486948B140F63400C0580D780124E6
:10B9A000AC40204340F63404E050087803F51064BE
:10B9B00004EB4010006840F00445087800E003E024
:10B9C00004EB401005604AE0087803F5306404EBAE
:10B9D00040100069C50CED04087804EB40100561C7
:10B9E000087804EB401000691E4C20400C7803F5E9
:10B9F000306505EB44142061486908B188684861E6
:10BA0000087803F5306404EB4010006940F4002529
:10BA1000087804EB40100561087804EB40100069D9
:10BA20008C68C4F3120420430C7803F5306505EBF1
:10BA300044142061012A06D1087803F5306404EB30
:10BA40004010CD684561087803F5306404EB401080
:10BA5000006840F00445087804EB401005600020C1
:10BA600030BD0000FFFF07E010B503460024C3F817
:10BA7000104BD3F8100B40F40024C3F8104BD3F84C
:10BA8000100B40F01804C3F8104BD3F8100B40F023
:10BA9000C044C3F8104B012906D1C3F8142B4FF052
:10BAA00080244FF43060C450002010BD10B5024611
:10BAB000487801281ED1087802F5106303EB401086
:10BAC000006820F40014087803EB40100460C87884
:10BAD000032802D0C87802282AD1087802F510631A
:10BAE00003EB4010006840F08054087803EB4010EE
:10BAF00004601DE0087802F5306303EB4010006835
:10BB000020F40014087803EB40100460C878032880
:10BB100002D0C87802280BD1087802F5306303EB15
:10BB20004010006840F08054087803EB4010046037
:10BB3000002010BD10B50246487801281FD10878B2
:10BB400002F5106303EB4010006800F0004048B9B4
:10BB5000087803EB4010006820F08044087803EB7D
:10BB600040100460087802F5106303EB4010006891
:10BB700040F40014087803EB401004601EE00878DD
:10BB800002F5306303EB4010006800F0004048B954
:10BB9000087803EB4010006820F08044087803EB3D
:10BBA00040100460087802F5306303EB4010006831
:10BBB00040F40014087803EB40100460002010BD2E
:10BBC000F8B505460C4616460027607801287DD159
:10BBD000606918BB207805F5106101EB4010006921
:10BBE000AA490840217805F5106202EB411108616D
:10BBF0002078114601EB4010006940F400222078C3
:10BC000001EB40100261207801EB40100069C20C8A
:10BC1000D204207801EB401002614FE0207805F556
:10BC2000106101EB40100069C20CD204207801EBD6
:10BC300040100261207801EB4010006993490840F0
:10BC4000217805F5106202EB41110861A168606975
:10BC50000844401EB0FBF1F08C49C94301EAC040E2
:10BC6000217802EB411109690843217802EB411167
:10BC700008612078114601EB401001696069C0F34A
:10BC800012000143207802EB40100161E0780128A6
:10BC900014D12078114601EB4010006920F0C04219
:10BCA000207801EB40100261207801EB4010006920
:10BCB00040F00052207801EB40100261012E09D1C2
:10BCC000207805F5106101EB401000E04BE022699F
:10BCD00042610EE0E07801280BD0606948B140F67F
:10BCE00034004059227801219140084340F6340144
:10BCF0004851E07801281ED140F60800405900F470
:10BD0000807060B9207805F5106101EB4010006883
:10BD100040F00052207801EB401002600BE02078E8
:10BD200005F5106101EB4010006840F0805220786A
:10BD300001EB40100260207805F5106101EB401026
:10BD4000006840F00442207801EB40100260E07887
:10BD5000012807D10096A08A83B222782846E1689C
:10BD600000F072F98FE0207805F5306101EB4010AA
:10BD70000069C20CD204207801EB401002612078E7
:10BD800001EB4010016941480140207805F530621F
:10BD900002EB401001616069C0B92078114601EBE7
:10BDA00040100069A168C1F312010843217802EB39
:10BDB000411108612078114601EB4010006940F400
:10BDC0000022207801EB4010026125E0A168606943
:10BDD0000844401EB0FBF1F087B2207805F53061D1
:10BDE00001EB401000692949C94301EAC7410843F2
:10BDF000217805F5306202EB411108612078114687
:10BE000001EB40100169A0687843C0F312000843B9
:10BE1000217802EB41110861012E06D1207805F549
:10BE2000306101EB4010E2684261E07801281ED1E8
:10BE300040F60800405900F4807060B9207805F59C
:10BE4000306101EB4010006840F00052207801EBB7
:10BE5000401002600BE0207805F5306101EB4010E6
:10BE6000006840F08052207801EB4010026020789A
:10BE700005F5306101EB4010006840F00442207885
:10BE800001EB401002600020F8BD0000FFFF07E05A
:10BE90000146886840F0010088600020704700007B
:10BEA000014600221020086100BF501C0246064BCC
:10BEB000984201D903207047086900F0100010284B
:10BEC000F3D00020F7E70000400D030010B5024654
:10BED0000023202040EA8110106100BF581C034657
:10BEE000054CA04201D9032010BD106900F02000CC
:10BEF0002028F3D00020F7E7400D03000146002082
:10BF000040F60802525802F0060202B917E040F665
:10BF10000802525802F00602022A06D040F6080231
:10BF2000525802F00602062A01D1032007E040F62B
:10BF30000802525802F00602042A00D1022070477B
:10BF40000146486900F001007047014640F61800BC
:10BF50004258001D4058024090B27047014640F6DA
:10BF600018004258001D40580240100C704730B570
:10BF700002464FF40165AB5840F63405AC5824FA3C
:10BF800001F505F0010543EAC51302F5106505EB5F
:10BF90004115AD6805EA030030BD024602F5306385
:10BFA00003EB4113986840F614039B581840704700
:10BFB0000146002048698A691040704770B5034601
:10BFC0000024D01CC61700EB9676B51000BF05E024
:10BFD0004FF48050C0580860091D641CAC42F7D370
:10BFE000084670BD70B504460D46E06820F0C040BC
:10BFF000E060012D04D1E06840F00050E06004E012
:10C000001DB9E06840F08040E0603220F4F7D6FED1
:10C01000002070BD0246D2F8000820F4FE60C2F88D
:10C020000008D2F800084FF4FE6303EA0113184336
:10C03000C2F80008002070470246D2F80008084302
:10C04000C2F8000800207047F0B50446059E00279E
:10C050000025A6B9D81C4FEAE07C00EB9C7C4FEA97
:10C06000AC0700BF09E0D1F800C004F5805000EB38
:10C070000230C0F800C0091D6D1CBD42F3D3002082
:10C08000F0BD00BFFEE7000030B503460C460022BD
:10C0900033E0995C1B48008800F4004058BB194805
:10C0A000008800F4804060B10A2903D00020154DBB
:10C0B000288020E01348008840F40040114D28807B
:10C0C00019E00D2906D10F48008840F480400D4D3D
:10C0D000288010E00B480088C0F30D000A4D295459
:10C0E00008480088401C074D288028460088C7283B
:10C0F00001DD00202880501CC2B2A242C9D300201A
:10C1000030BD0000C0020024AC0E002470B504460F
:10C110000D46AAB221460548FEF799FA0348FEF7F4
:10C12000E9FA012000F058FD70BD0000F80200247B
:10C1300010B586B000BF2248006840F020002049BA
:10C1400008600846006800F02000009000BF00BFB3
:10C150004FF480600190012002900390032004902E
:10C1600001A91848F4F748FE012291021548F4F796
:10C1700075FFFDF743F84FF00050FDF783F800F02E
:10C1800025F811490880084600884EF61871884243
:10C1900014D1032000F040F8044604F0010068B90F
:10C1A00000224FF480610748F4F758FFB720FDF7ED
:10C1B00059F8012291020348F4F750FF06B010BD70
:10C1C000E0440258001402583000002410B5002446
:10C1D00000224FF480610F48F4F740FF9020FDF7F4
:10C1E00041F80020FDF73EF80020FDF73BF8002065
:10C1F000FDF738F8FF20FDF735F844EA0024FF206A
:10C20000FDF730F80443012291020248F4F726FFBB
:10C21000204610BD0014025870B5044600250026C3
:10C22000012C04D0022C04D0032C06D103E00526F7
:10C2300005E0352603E0152601E0052600BF00BF16
:10C2400000224FF480610848F4F708FF3046FDF7FC
:10C2500009F8FF20FDF706F8054601229102024881
:10C26000F4F7FCFE284670BD001402580FB4054BCD
:10C2700010B503A9044A029800F008F910BC5DF853
:10C2800014FB000039CC00080C00002437B514461C
:10C290000846064B6A46214600F0F8F8044669460F
:10C2A000002000F08AFC20463EBD0000BBCB000809
:10C2B00002480068C0F30220704700000CED00E067
:10C2C00010B5002804DB0A07130E054A135406E0D4
:10C2D0000A07140E034A00F00F031B1FD45410BDAD
:10C2E00000E400E018ED00E002E008C8121F08C1F9
:10C2F000002AFAD170477047002001E001C1121FE7
:10C30000002AFBD1704700002DE9FF5F82B00021B9
:10C31000DDE90430020DDDF840B0034318D044F6E7
:10C320001050A2F2FF3242431514119801281FD079
:10C33000A5EB0B00401C5FEA000A4FF000064E4FD1
:10C34000DFF83891B046504615D5CAF1000413E025
:10C35000119801244AA3012801D16FEA0B01029828
:10C36000119AC0E90031C0E9024206B0BDE8F09F71
:10C37000CBF10000DFE704460021404A491842EBB8
:10C380000450CDE9001012E0E00707D032463B46EA
:10C3900040464946F4F7C2F88046894632463B4655
:10C3A00010461946F4F7BAF806460F466410002CFA
:10C3B000EAD1DDE90401DDE90023BAF1000F06DA74
:10C3C000F4F7ACF842464B46F4F7A8F805E0F4F76A
:10C3D00017F942464B46F4F713F904460E4600227D
:10C3E000284BF4F795F903D84FF0FF30014607E0EA
:10C3F0000022254B20463146F3F7E9FFF4F76FF9A9
:10C40000102409E0002C0ADB0A220023F3F760FF66
:10C41000039B30321A55641E50EA0102F2D1641CAB
:10C42000039AC4F111031444119A012A03D0012282
:10C4300008430DD10AE0084304D000204FF0110B4F
:10C44000119072E7A3EB0B056D1E0DE05B4504DD5B
:10C450004FF0000205F1010504E003DA4FF000029D
:10C46000A5F10105002AECD002981199C0E902312A
:10C47000C0E9004579E70000000014400000F03FEB
:10C48000300000000000F0430000E03F2DE9FF4FC6
:10C4900095B09B468946064600250FE2252877D1B0
:10C4A00000242746F84A0121059400E0044316F8C9
:10C4B000013F203B01FA03F01042F7D130782A28DF
:10C4C00011D06FF02F033078A0F13002092A16D86E
:10C4D000059A44F0020402EB820203EB420210448C
:10C4E000761C0590EFE759F8042B0592002A03DA31
:10C4F000504244F40054059044F00204761C307815
:10C500002E2816D116F8010F44F004042A280DD065
:10C510006FF02F023078A0F13003092B09D807EB18
:10C52000870302EB4303C718761CF3E759F8047B33
:10C53000761C30786C280FD006DC4C2817D0682881
:10C540000DD06A2814D104E0742810D07A280FD1B5
:10C550000DE044F400140AE044F4801401E044F4D3
:10C5600040147278824202D104F58014761C761C45
:10C57000307866280BD013DC582877D009DC0028E7
:10C5800075D04528F6D04628F4D047281AD19DE129
:10C5900018E0632835D0642879D0652812D195E158
:10C5A000702873D008DC6728F1D069286FD06E2816
:10C5B0000DD06F2806D1B5E073282CD0752875D022
:10C5C000782874D05A46179990476D1C75E1C4F3CA
:10C5D0000250022809D003280DD0D9F800100428F1
:10C5E0000DD00D6009F1040967E1D9F80010EA17D0
:10C5F000C1E90052F6E7D9F800100D80F2E70D709E
:10C60000F0E719F8041B8DF8001000208DF80100E8
:10C61000EA46012003E059F804AB4FF0FF30610710
:10C620004FF0000102D40DE008F101018846B94243
:10C630000FDA8045F8DB1AF808100029F4D108E079
:10C6400008F1010188468142FADB1AF80810002936
:10C65000F6D105985B46A0EB080721463846179AA5
:10C6600000F094FA284400EB080507E04DE029E1CA
:10C670000DE01AF8010B5A4617999047B8F10108D6
:10C68000F7D25B4621463846179A13E142E00A2268
:10C690000092C4F302524FF0000A022A08D059F85F
:10C6A00004CB032A4FEAEC710AD00DE029E02AE01E
:10C6B00009F1070121F00702F2E802C1914609E001
:10C6C0000FFA8CFC4FEAEC71042A03D14FFA8CFC70
:10C6D0004FEAEC71002907DA0A460021DCF1000C70
:10C6E00061EB02012D2202E0220504D52B228DF8F8
:10C6F0000420012203E0E20701D02022F7E7904660
:10C7000059E00A2102E010220DE010214FF0000A4A
:10C7100000910BE010224FF0000A44F004040827B7
:10C72000009203E008224FF0000A0092C4F3025284
:10C73000022A05D059F804CB0021032A08D009E0C9
:10C7400009F1070121F00702F2E802C1914605E074
:10C750001FFA8CFC042A01D10CF0FF0C4FF00008EA
:10C76000220728D5702806D0009B83F0100353EAD7
:10C770000A0305D00EE040228DF80420012208E0D3
:10C780005CEA010206D030228DF804208DF8050005
:10C7900002229046009B83F0080353EA0A030AD161
:10C7A0005CEA010201D1620705D530228DF8042030
:10C7B0004FF001087F1E582804D034A003900EA823
:10C7C00002900DE036A0F9E753466046009AF3F771
:10C7D0007FFD84460398825C0298401E029002709E
:10C7E0005CEA0100F0D1029806A9081A00F1200ABB
:10C7F000600702D524F4803400E00127574502DDAC
:10C80000A7EB0A0000E0002000EB0A010090059869
:10C810004144401A0590E00306D45B462146179A2E
:10C82000059800F0B3F90544002706E001A85A4630
:10C83000C05D179990476D1C7F1C4745F6DBE003F0
:10C840000CD55B462146179A059800F09FF90544E0
:10C8500004E030205A46179990476D1C0099481EF5
:10C8600000900029F5DC08E0029802995A46007809
:10C87000491C0291179990476D1CBAF10001AAF169
:10C88000010AF1DC65E10000092801003031323392
:10C8900034353637383961626364656600000000FC
:10C8A00030313233343536373839414243444546E6
:10C8B0000000000000F058F90544761C307800288C
:10C8C0007FF4ECAD19B02846BDE8F08F620700D4C4
:10C8D000062709F1070222F0070CFCE80223E146D3
:10C8E00003F000485FEA080C02D00FF2702C0DE054
:10C8F0005FEA045C02D50FF2682C07E05FEAC47CB3
:10C9000002D00FF2602C01E0AFF2700C4FF0FF3854
:10C9100023F00043CDF850C065280CD006DC452834
:10C9200009D046281DD047283DD13DE0662818D0C3
:10C9300067287ED138E00021112F01DB112000E0B3
:10C94000781CCDE9000106A90EA8FFF7DDFCDDE9A2
:10C950000F010E9A03910021009207F1010A049140
:10C960004DE04FF000400097CDE9011006A90EA858
:10C97000FFF7CAFCDDE90F0203920E9B119900221A
:10C98000DDF80CA00093049211B9791C00EB010AA8
:10C99000B7EB0A0004D4C0F1FF3007F1010A04909C
:10C9A000AAEB0700019044E0012F00DA01270021E3
:10C9B000112F01DD112000E03846CDE9000106A964
:10C9C0000EA8FFF7A1FCDDE90F010E9A03910021EB
:10C9D00004910092BA4621070CD40399514500DA1C
:10C9E0008A46BAF1010F05DD009AAAF10101515CF6
:10C9F000302908D0B84202DA10F1040F06DA01211A
:10CA0000CDE9011015E0AAF10101E9E7002805DCF4
:10CA1000049901440491AAEB000102E0411C514534
:10CA200000DD8A460499401A401C01904FF00040F6
:10CA30000290200704D40198504501DBCDF8048012
:10CA400000208DF84F0002980DF14F07B0F1004F14
:10CA500025D02B200E9002984FF0020800280CDA07
:10CA6000404202902D200E9007E00A210298F3F731
:10CA700079FC3031029007F8011DB8F10001A8F1EE
:10CA80000108F2DC02980028EFD1791E0E98087098
:10CA9000307800F0200040F0450007F8020D12A8A1
:10CAA000C01B00F107081498007800B1012000EBCA
:10CAB0000A01019801EBE07105984144401A401EBB
:10CAC0000590E00306D45B462146179A059800F0CE
:10CAD0005DF805441498007818B15A4617999047A4
:10CAE0006D1CE00324D55B462146179A059800F09B
:10CAF0004DF805441CE00498002807DBDDE903013C
:10CB0000884203DD0098405C179901E017993020B6
:10CB10005A469047049805F10105401C049001987D
:10CB2000401E019004D12E205A46179990476D1C43
:10CB3000BAF10001AAF1010ADDDC05E017F8010BEA
:10CB40005A46179990476D1CB8F10001A8F10108E9
:10CB5000F4DC5B462146179A0598ABE62D000000F1
:10CB60002B000000200000002DE9F04104460025C4
:10CB70001E461746880404D405E039462020B047F5
:10CB80006D1C641EF9D52846BDE8F0812DE9F04101
:10CB9000044600251E469046C80301D5302700E014
:10CBA0002027880404D505E041463846B0476D1C6F
:10CBB000641EF9D52846BDE8F0810A68531C0B6055
:10CBC0001070704710B504460420F7F74FFF014876
:10CBD000046010BD0800002430B50446002504E0C0
:10CBE0004FF47A7000F004F86D1CA542F8D330BD04
:10CBF00070B5034600224FF0E02675690D4E366889
:10CC000003FB06F44FF0E026B16910E04FF0E02698
:10CC1000B06988420BD0884202D20E1A324402E038
:10CC20002E1A0E4432440146A24200D300E0EDE742
:10CC300000BF70BD0800002400BF054AD26902F0A1
:10CC40004002002AF9D0C2B2014B1A857047000099
:10CC5000001001401CB500240026F3F7D9FEFBF7B5
:10CC60004EFFF4F713FA042302220521A020FCF75B
:10CC7000D7FB4FF4C870FFF7A5FF4FF4E13000F089
:10CC800063FA6B484168C8208847FBF735FAF8F724
:10CC90000BFBFCF731FAF8F7D1FCFFF749FA00205B
:10CCA00000F094F9012000F091F9022000F08EF9D3
:10CCB000FBF7D2FF002000F089F9012000F086F98F
:10CCC000022000F083F94FF478405A4908605AA0D6
:10CCD00010210B46C822CDE9001032211E20FBF79F
:10CCE000ADF959A010210B46C822CDE9001046210C
:10CCF0001E20FBF7A3F95AA010210B46C822CDE94C
:10CD000000105A211E20FBF799F959A010210B465B
:10CD1000C822CDE900106E211E20FBF78FF957A025
:10CD200010210B46C822CDE9001082211E20FBF7FE
:10CD300085F9002256495748FDF7AAFE564955483D
:10CD4000FEF7F2F855495348FDF773FC5148FEF7DA
:10CD5000D1F9F5F791FB6AE051480078864229D075
:10CD60004F480678012E12D11F20324908604DA08D
:10CD700010210B46C822CDE9001082211E20FBF7AE
:10CD80005DF9002201214C48F4F768F912E04FF4F4
:10CD900078402849086049A010210B46C822CDE9F7
:10CDA000001082211E20FBF749F90122114642485A
:10CDB000F4F754F94648008800F4004090B1444824
:10CDC0000088C0F30D05294642A000F0D9F9294694
:10CDD0004748FFF79BF947A000F0D2F900203C49F3
:10CDE000088024E0601C84B241F2883094FBF0F1AA
:10CDF00000FB114028B941A000F0C2F94BA000F09F
:10CE0000BFF9C82094FBF0F100FB114010B94DA010
:10CE100000F0B6F91E2094FBF0F100FB114018B9A8
:10CE200002212548F4F716F90A20FFF7D5FE93E70B
:10CE30006000002420000024504F4C4152495320F0
:10CE400053544D333248370055534220566972745B
:10CE500075616C2055534152542054455354000081
:10CE600041544F4D40414C49454E54454B00000004
:10CE7000323031392F352F313900000055534220DF
:10CE8000436F6E6E656374696E672E2E2E00000010
:10CE900068020024F802002460010024C402002477
:10CEA0006502002455534220436F6E6E65637465BE
:10CEB0006420202020000000000402585553422026
:10CEC000646973436F6E6E6563746564200000006F
:10CED000C00200240D0AC4FAB7A2CBCDB5C4CFFB63
:10CEE000CFA2B3A4B6C8CEAA3A25640D0A0D0A0093
:10CEF000AC0E00240D0A0D0A000000000D0AB0A2BD
:10CF0000B2A8C2DE53544D333246342F46372F4831
:10CF100037BFAAB7A2B0E5555342D0E9C4E2B4AED8
:10CF2000BFDACAB5D1E90D0A00000000D5FDB5E3AE
:10CF3000D4ADD7D340414C49454E54454B0D0A0D15
:10CF40000A000000C7EBCAE4C8EBCAFDBEDD2CD264
:10CF5000D4BBD8B3B5BCFCBDE1CAF80D0A000000D3
:10CF60002DE9F04104460E461548005D38B91448D5
:10CF700020380168204688470120BDE8F08111482B
:10CF800050F82400B04219D90F4850F82400B6FBDD
:10CF9000F0F10B480C3850F8240050F821200025FF
:10CFA00008E0002306480C3850F824004F1940F8D8
:10CFB00027306D1C9542F4DB0020DEE70220DCE721
:10CFC000F4020024D42A0108C82A010810B5044636
:10CFD000074951F824108A00064951F8240000211D
:10CFE00000F0A4F8012103480C30015510BD0000E9
:10CFF000BC2A0108E80200242DE9F04704460F4648
:10D000000025A9462348005D20B922482038016840
:10D01000204688471FB94FF0FF30BDE8F0871E4813
:10D0200050F82400B7FBF0F61B4850F82400B7FB7B
:10D03000F0F100FB117000B1761C184850F8240084
:10D04000451E22E013480C3850F8240050F8250003
:10D0500010B909F1010901E04FF00009B14513D100
:10D060004FF0000809E00B480C3850F8240005EB9D
:10D07000080140F8216008F10108B045F3D30648E3
:10D0800050F824006843C8E76D1E002DDADA4FF02F
:10D09000FF30C2E7F4020024C82A0108BC2A0108B4
:10D0A00010B501460023002207E00B4850F821008C
:10D0B00050F8220000B15B1C521C084850F82100B7
:10D0C0009042F2D84FF47A705843044C54F82140FF
:10D0D000B0FBF4F080B210BDE8020024BC2A0108C5
:10D0E00070B505460C4604B970BD054850F82500DA
:10D0F000261A31462846FFF733FF00BFF4E7000049
:10D10000DC02002470B504460E4631462046FFF787
:10D1100073FF0546681C08B9002070BD024850F82E
:10D1200024002844F9E70000DC02002430B503465F
:10D1300001E003F8011B141EA2F10102F9D130BD78
:10D14000014608687047000010B5044609480A49BE
:10D1500008600846446000218160C160016181610E
:10D160000C214161F7F7C4FD012204490248F7F799
:10D1700047FE10BD00100140E40500241200002409
:10D180000FB438B505A800900A48009A0499FFF733
:10D190007DF8002000900748F3F7DDF884B22146BF
:10D1A0000448FEF7B3FF21460248FBF7F3FE38BC04
:10D1B0005DF814FBE40D002430B595B0054613ABC3
:10D1C00012AA09A9284600F03FFA044614B12046E5
:10D1D00015B030BD0020149026E0224909689DF862
:10D1E000502001EBC20113AB11AA486801A900F05D
:10D1F0002BFA04460CB12046EAE709A901A800F081
:10D20000E1FC60B99DF844009DF84810884201DDBA
:10D210000220DDE79DF85000124988750AE09DF86C
:10D220005000401CC0B214900E48007D9DF8501074
:10D230008842D2DC00BF0B48007D9DF85010884228
:10D2400001D10420C4E714A9284600F0DDFA044601
:10D250000CB12046BCE79DF85000024948750020FB
:10D26000B6E70000600000242DE9F0419AB09C4828
:10D27000847D007DA04202DC1AB0BDE8F0819849AF
:10D28000096801EBC40106AB07AA486808A900F0C9
:10D29000DBF908A993A0FEF7E9FF002644E09048D7
:10D2A000008B0121B1400840D8B122218FA0FEF7A8
:10D2B000DDFF304600F02EFB8949243147183946FE
:10D2C0008BA0FEF7D3FF222188A0FEF7CFFF3046C8
:10D2D00000F020FB82492431084410A941F82600BF
:10D2E00018E0304600F016FB7D492431085810A99B
:10D2F00041F826007A48C07D30B910A850F82610B1
:10D300007CA0FEF7B3FF05E010A850F826107AA025
:10D31000FEF7ACFF9DF81C00401EB04202D078A082
:10D32000FEF7A4FF701CC6B29DF81C008642B6DB57
:10D3300074A0FEF79BFF00F03FFB6948407D0B287F
:10D340000DD2DFE800F0060D151E27323F4E5F724A
:10D3500087006349096851F834008047054690E02A
:10D360005F4A126852F8341010988847054688E0E2
:10D370005B4B1B6853F83420DDE9100190470546EC
:10D380007FE0574F3F6857F8343010A807C89847D8
:10D39000054676E0DFF848C1DCF800C05CF8347080
:10D3A00010A80FC8B84705466BE01498DFF830C1E5
:10D3B0000090DCF800C05CF8347010A80FC8B847C3
:10D3C00005465EE0DDE91401DFF814C1CDE9000196
:10D3D000DCF800C05CF8347010A80FC8B8470546E8
:10D3E0004FE0DDE914121698DFF8F4C0CDE9001221
:10D3F0000290DCF800C05CF8347010A80FC8B84781
:10D4000005463EE0DDE91423DDE91610DFF8D0C063
:10D41000CDE90023CDE90210DCF800C05CF83470DF
:10D4200010A80FC8B84705462BE0DDE91523DDE954
:10D430001710CDE90123CDE903101498DFF8A0C03F
:10D440000090DCF800C05CF8347010A80FC8B84732
:10D45000054616E0DDE91623DDE91810CDE90223C3
:10D46000CDE90410DDE91401DFF874C0CDE9000155
:10D47000DCF800C05CF8347010A80FC8B847054647
:10D4800000BF00BF00F056FA9DF8180001280CD12B
:10D490001348C07D20B929461BA0FEF7E7FE07E030
:10D4A00029461BA0FEF7E2FE02E018A0FEF7DEFE12
:10D4B0000B4890F8EC0088B10948D0F8F0000A2138
:10D4C000B0FBF1F201FB12070548D0F8F000B0FB09
:10D4D000F1F83A46414611A0FEF7C8FE00BFCBE680
:10D4E000600000240D0A2573280000002563000059
:10D4F00025730000256C640030582558000000009A
:10D500002C000000290000003D256C753B0D0A0031
:10D510003D305825583B0D0A0000000046756E63EB
:10D5200074696F6E2052756E2054696D653A25647A
:10D530002E2531646D730D0A00000000F0B503461E
:10D54000154600200022002600245BE01F782C2FC7
:10D5500001D104B901221F78292F01D01F780FB9FA
:10D5600004B950E0002E3AD11F78302F02DB1F782B
:10D57000392F17DD1F782D2F14D01F782B2F11D0A6
:10D580001F78612F02DB1F78662F0BDD1F78412F7C
:10D5900002DB1F78462F05DD1F78582F02D01F7839
:10D5A000782F0CD102B12EE01F78612F03DB1F789A
:10D5B000203F0F7001E01F780F70491C1FE01F789B
:10D5C000222F04D102B11EE00126012417E01F78AA
:10D5D000202F14D01F782C2F11D0FF2613E01F7896
:10D5E000222F00D1002402B10DE044B11F785C2F3E
:10D5F00002D15B1C471CF8B21F780F70491C471CF6
:10D60000F8B25B1CA2E700BF00270F702E70F0BDC0
:10D6100010B50446002010700BE020780870641CE0
:10D62000491C1078401C10701078984201DB0120D2
:10D6300010BD2078202802D020780028EDD10020CD
:10D64000087000BFF4E700002DE9FF4F85B0804669
:10D6500089460027002004900390012002904FF09B
:10D66000000B002544461DE02078202816D005F048
:10D670007F00052812DA0DB945F0800505F07F001E
:10D68000042803D120782A2800D00EE0207805F065
:10D690007F010DF80100681CC5B202E0852D00D1A4
:10D6A00003E0641C20780028DED100BF8DB100208B
:10D6B00005F07F010DF8010051A1684600F082FAE3
:10D6C00018B900210898017002E001210898017042
:10D6D00000254FF0000A444614E0641C0AF10100E2
:10D6E00000F0FF0A2078202802D020782A2809D1CB
:10D6F000204600F0D9F90646282E03D02A2E01D064
:10D70000CDF810A02078282802D020780028E4D175
:10D710004446049810B10498401C04444FF0000A99
:10D72000002654E0207810B94FF0010A50E020782C
:10D73000282803D116B9781CC7B213E0207829280D
:10D7400008D13EB917B1781EC7B201E04FF0010A07
:10D7500047B93DE02078222804D10EB9012000E02D
:10D760000020064647B9207820282FD0207889F855
:10D77000000009F1010929E020782C2804D10120BA
:10D780000290681CC5B214E02078202811D02078BF
:10D7900028280ED04DB9BBF1050F06DA20780DF818
:10D7A0000B000BF1010000F0FF0B0298401CC0B20F
:10D7B0000290012F0AD10298022807D10298401C3A
:10D7C000C0B202900398401CC0B20390641CA9E749
:10D7D00000BF0398012809D100200DF80B0008A113
:10D7E000684600F0EFF908B9002003900799039804
:10D7F0000870002089F80000504609B0BDE8F08F9D
:10D80000766F6964000000002DE9F043B5B005466D
:10D810000F460024002604E000213D488155701C7D
:10D82000C6B20A2EF8DB06E06D1C287818B9012074
:10D8300035B0BDE8F08328782828F5D16D1C61E06B
:10D8400034AA69462846FFF779FE064635449DF816
:10D85000D00020B1012827D0FF284CD149E09DF805
:10D86000000000B333A9684600F029F906460EB15E
:10D870000220DDE7204600F04DF825490A31339AB1
:10D880000A50A1F12400008B0121A14088432049C6
:10D890001A39088304211E480155601CC4B20A2CA1
:10D8A00001DD0320C4E726E0684600F0A7F9401C2C
:10D8B00000F0FF08204600F02DF815490A3100EB72
:10D8C00001094946684600F08EF911481A38018B63
:10D8D0000120A040014388B20D491A3908830C4841
:10D8E00000F80480601CC4B20A2C01DD03209FE70D
:10D8F00001E002209CE700BF2878292801D0287881
:10D9000000B900E09CE700BF3C70002090E70000F9
:10D910007A00002402460020002105E0044B5B5CF5
:10D920000344D8B24B1CD9B29142F7DB70470000D8
:10D930007A0000240E480068006900F0010040B140
:10D940000C48D0F8F0004FF6FF7108440949C1F8BF
:10D95000F0000848D0F8F00005490968496A084411
:10D960000449C1F8F0000846D0F8F0007047000004
:10D97000A40800246000002410B5044604EBC40091
:10D9800000EB04100122C2EB800081B24FF47A70E8
:10D99000FBF79CFE01200149C87510BD6000002402
:10D9A00010B50246012000E050430B1EA1F1010416
:10D9B000E1B2F9D110BD00006FF00100094909681A
:10D9C000086100BF000C07490968C86201460548A4
:10D9D000C16000BF00200349096848620249C1F8DC
:10D9E000F0007047A40800246000002470B51D48B2
:10D9F000008800F40040002833D01A480578002041
:10DA000019494855194881681748884704461CB980
:10DA10001649C868804721E0134800F0FBF8054626
:10DA2000012D00D02C46CCB1012C06D0022C08D000
:10DA3000032C0AD0042C10D10BE00DA0FEF716FC2D
:10DA40000BE00EA0FEF712FC07E00FA0FEF70EFCA5
:10DA500003E010A0FEF70AFC00BF00BF0020014950
:10DA6000088070BD100000241C0500246000002404
:10DA7000BAAFCAFDB4EDCEF3210D0A00B2CECAFD95
:10DA8000B4EDCEF3210D0A00B2CECAFDCCABB6E0A8
:10DA9000210D0A00CEB4D5D2B5BDC6A5C5E4B5C426
:10DAA000BAAFCAFD210D0A000146491C00E0491C1D
:10DAB0000878202801D10029F9D1087870472DE98C
:10DAC000F04F05460F4600264FF00A09B3462C4694
:10DAD0000020386034E02078392802DC20783028B3
:10DAE00011DA28782D2802D028782B2800D156B1B9
:10DAF0002078462802DC2078412804DA207858284B
:10DB000017D1012E15D12078412801DB4FF01009E3
:10DB100028782D2803D14FF0020B6D1C0FE02878D8
:10DB20002B2803D14FF0010B6D1C08E0701CC6B20E
:10DB300005E0207800B904E00120BDE8F08F641C06
:10DB4000C9E700BF2C46B9F1100F0FD1032E01DA3F
:10DB50000220F2E72078302806D16078582803D1D7
:10DB6000A41CB01EC6B204E00320E6E70EB90420F0
:10DB7000E3E71BE00EB1701EC6B22078392806DC40
:10DB80002078302803DB2078A0F1300A02E02078EA
:10DB9000A0F1370A31464846FFF702FF39680AFB11
:10DBA00000103860641C207800B900E0E2E700BF94
:10DBB000BBF1020F04D13868C0F10008C7F800803B
:10DBC0000020BAE702460AE010780B78984201D0AC
:10DBD00001207047107800B902E0521C491CF3E79D
:10DBE00000BF0020F5E706E002780A70027802B96B
:10DBF00002E0401C491CF7E700BF704701460020C7
:10DC000005E00A7802B903E0421CD0B2491CF8E7EB
:10DC100000BF704710B58CB004461E230BAA03A9A1
:10DC20002046FFF7F5FC0090009810B101200CB0E1
:10DC300010BD9DF82C00044400200B900EE04048DD
:10DC40009DF82C2050F8221003A8FFF7BBFF00B965
:10DC500008E09DF82C00401CC0B20B909DF82C00F1
:10DC60000728ECD300BF9DF82C00072863D2DFE81B
:10DC700000F004053C5E6564630000BF31A0FEF760
:10DC8000F5FA31A0FEF7F2FA3FA0FEF7EFFA4EA048
:10DC9000FEF7ECFA5CA0FEF7E9FA6BA0FEF7E6FAF5
:10DCA00079A0FEF7E3FA87A0FEF7E0FA8CA0FEF772
:10DCB000DDFA94A0FEF7DAFA98A0FEF7D7FA9DA055
:10DCC000FEF7D4FAA2A0FEF7D1FAA8A0FEF7CEFA8A
:10DCD000B4A0FEF7CBFAC1A0FEF7C8FACCA0FEF7BD
:10DCE000C5FAD8A0FEF7C2FAA2E216A0FEF7BEFA65
:10DCF000E4A0FEF7BBFA00200B900EE0F1480068AC
:10DD00009DF82C2000EBC2004168EFA0FEF7AEFAB0
:10DD10009DF82C00401CC0B20B90EA48007D9DF895
:10DD20002C108842EADC07A0FEF7A0FA80E205A0EA
:10DD3000FEF79CFACCE179E24DE221E2F4E1000049
:10DD4000340000240D0A00002D2D2D2D2D2D2D2DFC
:10DD50002D2D2D2D2D2D2D2D2D2D2D2D2D2D2D2DF3
:10DD600055534D4152542056332E332D2D2D2D2DEC
:10DD70002D2D2D2D2D2D2D2D2D2D2D2D2D2D2D2DD3
:10DD80002D2D2D200D0A00002020202055534D411F
:10DD90005254CAC7D3C9414C49454E54454BBFAAFA
:10DDA000B7A2B5C4D2BBB8F6C1E9C7C9B5C4B4AE51
:10DDB000BFDAB5F7CAD4BBA5BDBBD7E9BCFE2CCD35
:10DDC000A8B9FD200D0A0000CBFC2CC4E3BFC9D2CA
:10DDD000D4CDA8B9FDB4AEBFDAD6FACAD6B5F7D35A
:10DDE000C3B3CCD0F2C0EFC3E6B5C4C8CEBACEBA86
:10DDF000AFCAFD2CB2A2D6B4D0D02ED2F2B4CB2C66
:10DE0000C4E3BFC90D0A0000D2D4CBE6D2E2B8FC0D
:10DE1000B8C4BAAFCAFDB5C4CAE4C8EBB2CECAFD35
:10DE200028D6A7B3D6CAFDD7D62831302F3136BD74
:10DE3000F8D6C62CD6A7B3D6B8BACAFD29A1A2D7A0
:10DE4000D6B7FBB4AE0D0A00A1A2BAAFCAFDC8EBAB
:10DE5000BFDAB5D8D6B7B5C8D7F7CEAAB2CECAFD05
:10DE6000292CB5A5B8F6BAAFCAFDD7EEB6E0D6A74D
:10DE7000B3D63130B8F6CAE4C8EBB2CECAFD2CB284
:10DE8000A2D6A7B3D60D0A00BAAFCAFDB7B5BBD8A4
:10DE9000D6B5CFD4CABE2ED6A7B3D6B2CECAFDCF82
:10DEA000D4CABEBDF8D6C6C9E8D6C3B9A6C4DC2C50
:10DEB000D6A7B3D6BDF8D6C6D7AABBBBB9A6C4DC15
:10DEC0002E0D0A00BCBCCAF5D6A7B3D63A77777731
:10DED0002E6F70656E6564762E636F6D0D0A00009F
:10DEE00055534D415254D3D037B8F6CFB5CDB3C307
:10DEF000FCC1EE28B1D8D0EBD0A1D0B4293A0D0A9C
:10DF0000000000003F3A202020202020BBF1C8A1C3
:10DF1000B0EFD6FAD0C5CFA20D0A000068656C70CC
:10DF20003A202020BBF1C8A1B0EFD6FAD0C5CFA2CD
:10DF30000D0A00006C6973743A202020BFC9D3C356
:10DF4000B5C4BAAFCAFDC1D0B1ED0D0A0A000000D8
:10DF500069643A2020202020BFC9D3C3BAAFCAFDCC
:10DF6000B5C44944C1D0B1ED0D0A0A006865783ADC
:10DF700020202020B2CECAFD3136BDF8D6C6CFD47F
:10DF8000CABE2CBAF3B8FABFD5B8F12BCAFDD7D6A2
:10DF9000BCB4D6B4D0D0BDF8D6C6D7AABBBB0D0A88
:10DFA0000A0000006465633A20202020B2CECAFD3A
:10DFB0003130BDF8D6C6CFD4CABE2CBAF3B8FABF3A
:10DFC000D5B8F12BCAFDD7D6BCB4D6B4D0D0BDF8E5
:10DFD000D6C6D7AABBBB0D0A0A00000072756E74C4
:10DFE000696D653A312CBFAAC6F4BAAFCAFDD4CB6D
:10DFF000D0D0BCC6CAB13B302CB9D8B1D5BAAFCAA3
:10E00000FDD4CBD0D0BCC6CAB13B0D0A0A0000007B
:10E01000C7EBB0B4D5D5B3CCD0F2B1E0D0B4B8F141
:10E02000CABDCAE4C8EBBAAFCAFDC3FBBCB0B2CE2E
:10E03000CAFDB2A2D2D4BBD8B3B5BCFCBDE1CAF80C
:10E040002E0D0A002D2D2D2D2D2D2D2D2D2D2D2D6F
:10E050002D2D2D2D2D2D2D2D2D2D2D2D2D2D414CBD
:10E0600049454E54454B2D2D2D2D2D2D2D2D2D2D2E
:10E070002D2D2D2D2D2D2D2D2D2D2D2D2D2D2D20DD
:10E080000D0A00002D2D2D2D2D2D2D2D2D2D2D2D5D
:10E090002D2D2D2D2D2D2D2D2D2D2D2D2DBAAFCA04
:10E0A000FDC7E5B5A52D2D2D2D2D2D2D2D2D2D2D7E
:10E0B0002D2D2D2D2D2D2D2D2D2D2D2D2D2D2D2D90
:10E0C000200D0A006000002425730D0A00000000E6
:10E0D00059A0FEF7CBF800200B901AE066490968BA
:10E0E0009DF82C2001EBC20101AB02AA486803A9EC
:10E0F000FFF7AAFA604800689DF82C1050F831200C
:10E1000003A95EA0FEF7B2F89DF82C00401CC0B237
:10E110000B905948007D9DF82C108842DEDCAFF250
:10E12000DC30FEF7A3F883E0AFF2E830FEF79EF8AC
:10E130000BAA03A92046FFF701FA9DF82C00C8B9E5
:10E14000694603A8FFF7BBFC0B909DF82C0020B993
:10E150004FA00099FEF78AF80EE09DF82C000428E5
:10E1600001D0022063E54DA0FEF780F8012042496E
:10E17000C87501E002205AE547A0FEF777F857E09E
:10E1800045A0FEF773F80BAA03A92046FFF7D6F9BE
:10E190009DF82C00C8B9694603A8FFF790FC0B90C6
:10E1A0009DF82C0020B942A00099FEF75FF80EE020
:10E1B0009DF82C00042801D0022038E53FA0FEF78E
:10E1C00055F800202C49C87501E002202FE532A047
:10E1D000FEF74CF82CE030A0FEF748F80BAA03A994
:10E1E0002046FFF7ABF99DF82C00C8B9694603A893
:10E1F000FFF765FC0B909DF82C0078B91E4900983C
:10E2000081F8EC00084690F8EC0018B130A0FEF759
:10E210002DF807E035A0FEF729F803E0022006E517
:10E22000022004E51CA0FEF721F801E00120FEE435
:10E2300000BF0020FBE400002D2D2D2D2D2D2D2DB8
:10E240002D2D2D2D2D2D2D2D2D2D2D2D2D2D2D2DFE
:10E250002DBAAFCAFD204944202D2D2D2D2D2D2D59
:10E260002D2D2D2D2D2D2D2D2D2D2D2D2D2D2D2DDE
:10E270002D2D2D2D200D0A0060000024257320690E
:10E28000642069733A0D0A3058253038580D0A0059
:10E290004845583A305825580D0A00003136BDF827
:10E2A000D6C6B2CECAFDCFD4CABE210D0A00000028
:10E2B0004445433A256C750D0A0000003130BDF825
:10E2C000D6C6B2CECAFDCFD4CABE210D0A00000008
:10E2D00052756E2054696D652043616C63756C6185
:10E2E00074696F6E204F4E0D0A00000052756E204B
:10E2F00054696D652043616C63756C6174696F6E00
:10E30000204F46460D0A00000160704701000200E0
:10E310000400060008000A000C0010002000400065
:10E320008000000100000000010203040102030458
:10E3300006070809010002000400060008000A00A0
:10E340000C001000200040008000000101000200CD
:10E350000400060008000A000C0010002000400025
:10E36000800000010000000000000000000000002C
:10E37000000000003F4000000000000000003000EE
:10E38000400030004000000009000BC03D000BC001
:10E390003D00090018C024407FE022403180000089
:10E3A000180024C01B000D803240018003801C40F7
:10E3B00027401C8007400040100060000000000063
:10E3C000000000000000000000001F8020404020EE
:10E3D0000000402020401F800000000009000600CF
:10E3E0001F80060009000000040004003F800400B4
:10E3F00004000000001000600000000000000000A9
:10E4000004000400040004000400000000000040B8
:10E410000000000000000000002001C006003800DD
:10E42000400000001F802040204020401F8000004E
:10E43000000010403FC000400000000018C0214014
:10E4400022402440184000001080204024402440F6
:10E450001B80000002000D0011003FC001400000C1
:10E460003C80244024402440238000001F8024401E
:10E4700024403440038000003000200027C03800D2
:10E48000200000001B802440244024401B8000000A
:10E490001C0022C0224022401F800000000000001B
:10E4A00008400000000000000000000004600000C0
:10E4B00000000000000004000A001100208040401D
:10E4C000090009000900090009000000000040409F
:10E4D000208011000A0004001800200023402400BE
:10E4E000180000001F802040274029401F400000E6
:10E4F000004007C039000F0001C0004020403FC06D
:10E50000244024401B8000001F80204020402040E9
:10E510003080000020403FC0204020401F8000008D
:10E5200020403FC024402E4030C0000020403FC06B
:10E5300024402E00300000000F00108020402240B8
:10E540003380020020403FC0040004003FC0204050
:10E55000204020403FC0204020400000006020209C
:10E5600020203FC02000200020403FC024400B005E
:10E5700030C0204020403FC020400040004000C04C
:10E580003FC03C0003C03C003FC0000020403FC0F3
:10E590000C4023003FC020001F802040204020402E
:10E5A0001F80000020403FC02440240018000000CD
:10E5B0001F802140214020E01FA0000020403FC0DC
:10E5C0002440260019C0004018C0244024402240A6
:10E5D00031800000300020403FC02040300000006B
:10E5E00020003F80004000403F80200020003E008F
:10E5F00001C0070038002000380007C03C0007C0F9
:10E6000038000000204039C0060039C0204000001A
:10E610002000384007C0384020000000304021C0B2
:10E620002640384020C00000000000007FE040206D
:10E6300040200000000070000C000380004000003B
:10E640000000402040207FE000000000000020008B
:10E65000400020000000000000100010001000101A
:10E66000001000100000000040000000000000004A
:10E67000000002800540054003C0004020003FC06C
:10E680000440044003800000000003800440044074
:10E690000640000000000380044024403FC00040CA
:10E6A00000000380054005400340000000000440D6
:10E6B0001FC0244024402000000002E00550055007
:10E6C0000650042020403FC00440040003C0004026
:10E6D0000000044027C000400000000000100010AF
:10E6E000041027E00000000020403FC00140070068
:10E6F00004C00440204020403FC0004000400000D3
:10E7000007C0040007C0040003C00000044007C0A5
:10E710000440040003C000400000038004400440A3
:10E7200003800000041007F0045004400380000040
:10E73000000003800440045007F00010044007C0AC
:10E7400002400400040000000000064005400540AF
:10E7500004C00000000004001F80044000400000CE
:10E76000040007800040044007C000400400070088
:10E7700004C0018006000400060001C0070001C0BB
:10E7800006000000044006C0010006C0044000006E
:10E790000410071004E0018006000400000004409B
:10E7A00005C00640044000000000000004007BE0BB
:10E7B00040200000000000000000FFF0000000000A
:10E7C000000040207BE004000000000040008000CA
:10E7D0004000200020004000000000000000000079
:10E7E00000000000000000000000000000001FCC3E
:10E7F000000C000000000000000008003000600075
:10E800000800300060000000022003FC1E200220EF
:10E8100003FC1E200220000000000E1811043FFF20
:10E8200010840C78000000000F0010840F3800C026
:10E83000077818840078000000780F8410C4112431
:10E840000E9800E4008400080800680070000000D2
:10E85000000000000000000000000000000007E0D1
:10E86000181820044002000000004002200418187C
:10E8700007E00000000000000240024001800FF0AD
:10E8800001800240024000000080008000800FF8FC
:10E8900000800080008000000001000D000E0000DC
:10E8A00000000000000000000000008000800080E8
:10E8B00000800080008000800000000C000C000040
:10E8C00000000000000000000000000600180060CA
:10E8D0000180060018002000000007F0080810045E
:10E8E0001004080807F000000000080408041FFCDA
:10E8F000000400040000000000000E0C101410249E
:10E90000104411840E0C000000000C1810041104B7
:10E91000110412880C700000000000E003200424A1
:10E9200008241FFC0024000000001F98108411041C
:10E930001104108810700000000007F0088811040E
:10E94000110418880070000000001C00100010FC6A
:10E9500013001C001000000000000E381144108449
:10E96000108411440E38000000000700088C104489
:10E970001044088807F00000000000000000030CAD
:10E98000030C000000000000000000000001010670
:10E990000000000000000000000000800140022094
:10E9A00004100808100400000220022002200220A7
:10E9B00002200220022000000000100408080410B9
:10E9C000022001400080000000000E001200100C28
:10E9D000106C10800F00000003E00C1813E41424E6
:10E9E00017C4082807D000000004003C03C41C40E2
:10E9F000074000E4001C000410041FFC1104110473
:10EA000011040E880070000003E00C1810041004BC
:10EA1000100410081C10000010041FFC1004100447
:10EA20001004080807F0000010041FFC1104110472
:10EA300017C410040818000010041FFC1104110072
:10EA400017C010000800000003E00C1810041004A8
:10EA500010441C780040000010041FFC108400804B
:10EA6000008010841FFC10040000100410041FFC20
:10EA70001004100400000000000300011001100148
:10EA80001FFE10001000000010041FFC1104038082
:10EA90001464181C1004000010041FFC100400046F
:10EAA00000040004000C000010041FFC1F0000FC08
:10EAB0001F001FFC1004000010041FFC0C040300C6
:10EAC00000E010181FFC100007F0080810041004E4
:10EAD0001004080807F0000010041FFC10841080C8
:10EAE000108010800F00000007F008181024102478
:10EAF000101C080A07F2000010041FFC110411008A
:10EB000011C011300E0C000400000E1C1104108402
:10EB1000108410441C3800001800100010041FFC62
:10EB2000100410001800000010001FF8100400046A
:10EB3000000410041FF8100010001E0011E0001C5B
:10EB4000007013801C0010001FC0103C00E01F006C
:10EB500000E0103C1FC000001004180C163401C067
:10EB600001C01634180C100410001C00130400FC23
:10EB700013041C00100000000804101C1064108412
:10EB800013041C04101800000000000000007FFEA9
:10EB90004002400240020000000030000C000380F0
:10EBA0000060001C00030000000040024002400220
:10EBB0007FFE000000000000000000002000400078
:10EBC00040004000200000000001000100010001A1
:10EBD0000001000100010001000040004000200091
:10EBE0000000000000000000000000980124014423
:10EBF0000144014400FC000410001FFC00880104D3
:10EC0000010400880070000000000070008801040A
:10EC10000104010400880000000000700088010465
:10EC2000010411081FFC0004000000F80144014425
:10EC30000144014400C800000000010401040FFC6D
:10EC40001104110411001800000000D60129012947
:10EC5000012901C90106000010041FFC0084010005
:10EC60000100010400FC000400000104190419FC67
:10EC70000004000400000000000000030001010186
:10EC8000190119FE0000000010041FFC00240040C0
:10EC900001B4010C010400000000100410041FFC6A
:10ECA0000004000400000000010401FC0104010054
:10ECB00001FC0104010000FC010401FC00840100CE
:10ECC0000100010400FC0004000000F8010401043C
:10ECD0000104010400F80000010101FF00850104A6
:10ECE000010400880070000000000070008801042A
:10ECF0000104010501FF00010104010401FC00847D
:10ED00000104010001800000000000CC0124012466
:10ED1000012401240198000000000100010007F80F
:10ED20000104010400000000010001F800040004D7
:10ED30000004010801FC0004010001800170000CC6
:10ED4000001001600180010001F0010C003001C0E1
:10ED50000030010C01F0010000000104018C00747E
:10ED60000170018C01040000010101810171000E9C
:10ED7000001801600180010000000184010C0134D1
:10ED800001440184010C00000000000000000000AC
:10ED900001003EFC400240020000000000000000B4
:10EDA000FFFF0000000000000000400240023EFCA7
:10EDB00001000000000000000000600080008000F2
:10EDC0004000400020002000000000000000000083
:10EDD0000000000000000000000000000000000033
:10EDE0000000000000000000000000000000000023
:10EDF00000000000000000000000000F80380FFE3F
:10EE0000380F803800000000000000000000000003
:10EE10000000000000000100000600000C000038A7
:10EE200000003100000600000C0000380000300037
:10EE3000000000000000000061800067F807F98012
:10EE40000061800061800061800061800067F807D8
:10EE5000F98000618000000000000000000001C097
:10EE6000E003E0F00630080418081FFFFE040E0857
:10EE70000787F00381E000000000000001F00006B9
:10EE80000C00040408060C7001F9C0000E00003BE1
:10EE9000E000EC18070808040C180003E00000006C
:10EEA0000001E00007F003F818041C080417080725
:10EEB000E1D003C0E00023B0003C080020080000BF
:10EEC00010000000000000010000310000320000CE
:10EED0001C00000000000000000000000000000016
:10EEE0000000000000000000000000000000000022
:10EEF00000000000000000007F0001FFC00780F05C
:10EF00000C00181000042000020000000000002087
:10EF100000021000040C00180780F001FFC0007F01
:10EF200000000000000000000000000000000000E1
:10EF3000000000004200006600006600003C000087
:10EF4000180003FFC0001800003C000066000066C7
:10EF50000000420000000000080000080000080057
:10EF600000080000080001FFC000080000080000C1
:10EF70000800000800000800000000000001000078
:10EF80003100003200001C00000000000000000002
:10EF90000000000000000000000000000000000071
:10EFA0000800000800000800000800000800000831
:10EFB0000000080000080000080000080000000031
:10EFC0000000000000000000380000380000380099
:10EFD0000000000000000000000000000000000031
:10EFE0000000000000000000000600001C0000708F
:10EFF000000180000E0000380000C0000700001C67
:10F000000000300000000000000000007F8001FFD1
:10F01000E0038070060018040008040008060018C9
:10F0200003807001FFE0007F80000000000000000E
:10F03000000001000801000801000803FFF807FFB5
:10F04000F8000008000008000008000000000000B0
:10F0500000000001C03802C05804009804011804E0
:10F060000218040418061C1803F81801E0F8000040
:10F070000000000000000001C0E003C0F004000830
:10F0800004080804080806180803F41801E7F0004B
:10F0900001E0000000000000000000000300000D7F
:10F0A0000000110000610000810803010807FFF85B
:10F0B0000FFFF80001080001080000000000000038
:10F0C00000E007FCD0060808061008061008061025
:10F0D00008061838060FF00607C000000000000000
:10F0E000000000003F8001FFE003843002081804A4
:10F0F0001008041008041008071810030FF0000788
:10F10000C000000000000000000003C00007000075
:10F110000600000600F80607F806180006E00007DB
:10F12000000006000000000000000001E1E003F71D
:10F13000F0063410041808041808040C08040C081D
:10F1400006161803F3F001C1E00000000000000003
:10F15000F80003FC30030638040208040208040225
:10F16000080404100308F001FFC0007F0000000045
:10F17000000000000000000000000000000000008F
:10F180007038007038007038000000000000000087
:10F19000000000000000000000000000000000006F
:10F1A00000000000301A00301C00000000000000C9
:10F1B0000000000000000000000000000000000847
:10F1C0000000140000220000410000808001004087
:10F1D00002002004001008000800000000000000E9
:10F1E0002100002100002100002100002100002159
:10F1F000000021000021000021000021000000008B
:10F2000000000000000008000804001002002001B7
:10F21000004000808000410000220000140000082F
:10F220000000000000000003C00004C00004000053
:10F23000080038080F380808380810000C3000079C
:10F24000E00003C000000000000000003F8000FF5D
:10F25000E0038070020F1006708804C088048308E1
:10F26000047F8802C09003012000FE4000000800D7
:10F2700000180001F8003E0801C20007020007E282
:10F280000000FE00001FC80001F800003800000860
:10F2900004000807FFF807FFF8040808040808043A
:10F2A000080804080806180803F41801E7F000012C
:10F2B000E0000000000000003F8001FFE0038070DC
:10F2C00002001804000804000804000804001006E6
:10F2D00000200780C000000004000807FFF807FFB7
:10F2E000F8040008040008040008040018020010D4
:10F2F00003807001FFE0007F800000000400080729
:10F30000FFF807FFF80408080408080408080408C0
:10F3100008043E0804000806001801006000000010
:10F3200004000807FFF807FFF804080804080004B1
:10F330000800040800043E000600000600000180EA
:10F3400000000000000000003F8001FFE00380702B
:10F350000600180400080402080402080203F0076B
:10F3600083F000020000020004000807FFF807FF16
:10F37000F804080800080000080000080000080061
:10F3800004080807FFF807FFF80400080000000061
:10F39000000004000804000804000807FFF807FF45
:10F3A000F804000804000804000800000000000041
:10F3B0000000000000060000070000010400010436
:10F3C000000104000307FFFE07FFFC040000040027
:10F3D0000004000004000807FFF807FFF8040C0809
:10F3E000001800003E0004C7800503C80600F804AA
:10F3F000003804001800000804000807FFF807FFA1
:10F40000F8040008000008000008000008000008D8
:10F410000000080000180000600000000400080759
:10F42000FFF807800807FC00007FC00003F8000712
:10F43000C000780007800807FFF807FFF8040008FD
:10F4400004000807FFF807000803C00000E0000000
:10F450003800001E000007000001C00400F007FF94
:10F46000F8040000000000007F8001FFE0038070CE
:10F470000600180400080400080600180300300104
:10F48000FFE0007F8000000004000807FFF807FF8E
:10F49000F804040804040004040004040004040044
:10F4A000060C0003F80001F000000000000000005E
:10F4B0007F8001FFE003807006008804008804005C
:10F4C000C806003C03003E01FFE6007F8400000008
:10F4D00004000807FFF807FFF80408080408000400
:10F4E0000C00040F00040BC00610F003F03801E01C
:10F4F0000800000800000001E0F803F030063010BA
:10F50000041808041808040C08040C080206180261
:10F5100007F00781E0000000018000060000040001
:10F520000004000004000807FFF807FFF8040008C3
:10F530000400000400000600000180000400000731
:10F54000FFE007FFF00400180000080000080000BA
:10F550000800000800000804001007FFE004000095
:10F5600004000006000007E00007FE00041FE000A2
:10F5700001F80000380001E0043E0007C00006006A
:10F580000004000004000007E00007FFC0041FF8AB
:10F590000007C007F80007FF80043FF80007C00419
:10F5A000F800070000040000000000040008060046
:10F5B0001807C07805F1C8003E00001F800463E80A
:10F5C0000780F80600180400080000000400000688
:10F5D000000007800007E008047C08001FF800070F
:10F5E000F800180804E00807000006000004000006
:10F5F0000000000100080600380400F80403E804D5
:10F600000F08047C0805F00807C00807001804006C
:10F61000600000000000000000000000000000008A
:10F620000000003FFFFE2000022000022000022018
:10F63000000220000200000000000000000008009E
:10F640000007000000C0000038000006000001C0F4
:10F6500000003000000E000001000000000000006B
:10F6600000002000022000022000022000022000F2
:10F67000023FFFFE0000000000000000000000004C
:10F680000000000000000000000800001000003032
:10F690000000200000300000100000080000000002
:10F6A0000000000000000100000100000100000156
:10F6B0000000010000010000010000010000010045
:10F6C0000001000001000001000000000000000037
:10F6D00000200000200000100000100000000000CA
:10F6E000000000000000000000000000000000001A
:10F6F00000F00019F8001B1800220800260800245A
:10F7000008002410003FF8001FF80000080000184F
:10F7100000000004000007FFF80FFFF000181800B9
:10F720001008002008002008003018001FF0000F0B
:10F73000C00000000000000007C0001FF0001830EB
:10F74000002008002008002008003C08001C1000D1
:10F7500000600000000000000000000007C0001F63
:10F76000F0003818002008002008002008041010BD
:10F7700007FFF80FFFF0000010000000000000007D
:10F7800000000007C0001FF0001230002218002205
:10F7900008002208003208001E10000E20000000A1
:10F7A00000000000200000200800200801FFF803EE
:10F7B000FFF80620080420080420080720000300A2
:10F7C0000000000000000000000E000E6E001FF39D
:10F7D0000031B10020B10020B1003191001F1300B1
:10F7E0002E1E00200E00300000000004000807FF5D
:10F7F000F80FFFF80010080020000020000020088B
:10F80000003FF8001FF800000800000000000000A2
:10F810000000002008002008002008063FF8063FEE
:10F82000F8000008000008000008000000000000C8
:10F8300000000000000000000300000300200100A1
:10F840002001002003063FFE063FFC0000000000F0
:10F850000000000000000004000807FFF80FFFF898
:10F86000000188000300002FC00038F80020380095
:10F870002008000008000000000000000000040054
:10F880000804000804000807FFF80FFFF80000084C
:10F890000000080000080000000000000020080030
:10F8A0003FF8003FF8001008002000003FF8003F3C
:10F8B000F8001008002000003FF8003FF8000008A2
:10F8C000000000002008003FF8003FF8001008008A
:10F8D0001000002000002008003FF8001FF8000082
:10F8E000080000000000000007C0000FF000183002
:10F8F0000030080020080020080030080018300000
:10F900000FF00007C0000000000000002001003FD1
:10F91000FF003FFF00101100200900200800200810
:10F92000003038001FF0000FC00000000000000091
:10F9300007C0001FF0003818002008002008002031
:10F9400009001011001FFF003FFF00000100000030
:10F95000002008002008002008003FF8003FF800C1
:10F9600008080010080020080020000030000030C7
:10F9700000000000000000000000000C78001E18CD
:10F980000033080023080021080021880021980086
:10F9900030F000386000000000000000200000206F
:10F9A0000000200000FFF003FFF8002008002008FE
:10F9B00000200800003000000000000000000000EF
:10F9C0002000003FF0007FF8000018000008000051
:10F9D00008002010003FF8007FF000001000000039
:10F9E000000000002000003000003C00003F8000CC
:10F9F00023F0000078000070002380003C000030FD
:10FA000000002000002000003C00003FE00023F840
:10FA10000000E0002700003E00003FE00021F80069
:10FA200001E0003E0000200000000000200800204F
:10FA300008003838003E680027800003C8002CF812
:10FA400000383800201800200800000000000000E6
:10FA50002000003003003C01003F830023EC000045
:10FA600070002380003C0000200000200000000007
:10FA70000000000000000038080020380020F800D6
:10FA800023E8002F88003E080038080020180000F6
:10FA900070000000000000000000000000000000F6
:10FAA0000000000008000014001FF7FC30000620D2
:10FAB0000002000000000000000000000000000044
:10FAC00000000000000000000000FFFFFF00000039
:10FAD0000000000000000000000000000000000026
:10FAE00000002000023000061FF7FC001400000890
:10FAF0000000000000000000000000000000000006
:10FB000000000018000060000040000040000020DD
:10FB100000001000000800000400000400000C00B9
:10FB200000100000000000000000000000000000C5
:10FB300000000000000000000000000000000000C5
:10FB400000000000000000000000000000000000B5
:10FB500000000000000000000000000000000000A5
:10FB60000000000000000000000000000000000095
:10FB70000000000000000000000000000000000085
:10FB80000000000000000000000000000000000075
:10FB90000000000000000000000000000000000065
:10FBA0000000000000000000000000000000000055
:10FBB00000000000000000000000000007F000C08E
:10FBC00007FFE1E007F001E0000000C000000000D6
:10FBD0000000000000000000000000000000000025
:10FBE0000000000000000000000000000000000015
:10FBF0000000000000000000000000000000000005
:10FC000000000000000000000000000000000000F4
:10FC100000000000000000000000000000000000E4
:10FC200000000000000000000000000000200000B4
:10FC300001C00000078000001F0000001E0000003F
:10FC40001C20000001C00000078000001F00000011
:10FC50001E0000001C00000000000000000000006A
:10FC60000000000000000000000000000000000094
:10FC70000000000000000000000000000000000084
:10FC80000000000000000000000000000000000074
:10FC90000000000000000000000000000000000064
:10FCA000000000000000000000180C0000180C000C
:10FCB00000180FE0001FFC0003F80C0000180C00F7
:10FCC00000180C0000180C0000180C0000180FE0C1
:10FCD000001FFC0003F80C0000180C0000180C00BA
:10FCE0000000000000000000000000000000000014
:10FCF0000000000000000000000000000000000004
:10FD000000000000000000000000000000000000F3
:10FD100000000000000000000000000000000000E3
:10FD2000000000000000000000000000000007804C
:10FD3000007807C000FC0640010E002003070020E9
:10FD4000020380200FFFFFFC0201C0200200E060E0
:10FD50000130704001F03F8000F01F000000000003
:10FD60000000000000000000000000000000000093
:10FD70000000000000000000000000000000000083
:10FD80000000000000000000000000000000000073
:10FD90000000000000000000000000000000000063
:10FDA0000000000000FE000001FF000003018000D1
:10FDB00002008060030181C001FF070000FE1800FF
:10FDC0000000E0000003BF00000CFFC00071806075
:10FDD00001C10020030180600000FFC000003F005F
:10FDE0000000000000000000000000000000000013
:10FDF0000000000000000000000000000000000003
:10FE000000000000000000000000000000000000F2
:10FE100000000000000000000000000000000000E2
:10FE20000000000000001F0000007FC000FCC0C0F8
:10FE300001FF80600303E0200202782002061E20FA
:10FE400003FC074001F00380000103C000011C60B7
:10FE50000001E020000100200001004000000180BE
:10FE60000000000000000000000000000000000092
:10FE70000000000000000000000000000000000082
:10FE80000000000000000000000000000000000072
:10FE90000000000000000000000000000000000062
:10FEA0000000000000000000002000001C600000B6
:10FEB0001C4000001F8000000F0000000000000038
:10FEC0000000000000000000000000000000000032
:10FED0000000000000000000000000000000000022
:10FEE0000000000000000000000000000000000012
:10FEF0000000000000000000000000000000000002
:10FF000000000000000000000000000000000000F1
:10FF100000000000000000000000000000000000E1
:10FF200000000000000000000000000000000000D1
:10FF300000000000000000000000000000000000C1
:10FF40000007F800003FFF00007807C001C000E094
:10FF50000300003004000008080000041000000244
:10FF60000000000000000000000000000000000091
:10FF70000000000000000000000000000000000081
:10FF80000000000000000000000000000000000071
:10FF90000000000000000000000000000000000061
:10FFA0000000000000000000100000020800000433
:10FFB000040000080300003001C000E0007807C022
:10FFC000003FFF000007F8000000000000000000F4
:10FFD0000000000000000000000000000000000021
:10FFE0000000000000000000000000000000000011
:10FFF0000000000000000000000000000000000001
:020000040801F1
:1000000000000000000000000000000000000000F0
:1000100000000000000000000000000000000000E0
:10002000000000000000000000000000000C1800AC
:10003000000E3800000E380000063000000360009B
:100040000061438000FFFF80006143000003600007
:1000500000063000000E3800000E3800000C1800BA
:100060000000000000000000000000000000000090
:100070000000000000000000000000000000000080
:100080000000000000000000000000000000000070
:100090000000000000000000000000000000000060
:1000A00000000000000000000000000000008000D0
:1000B0000000800000008000000080000000800040
:1000C00000008000007FFF00000080000000800032
:1000D0000000800000008000000080000000800020
:1000E0000000000000000000000000000000000010
:1000F0000000000000000000000000000000000000
:1001000000000000000000000000000000000000EF
:1001100000000000000000000000000000000000DF
:10012000000000000000000000000001000000E3EB
:10013000000000E2000000FC000000780000000069
:1001400000000000000000000000000000000000AF
:10015000000000000000000000000000000000009F
:10016000000000000000000000000000000000008F
:10017000000000000000000000000000000000007F
:10018000000000000000000000000000000000006F
:10019000000000000000000000000000000000005F
:1001A000000000000000000000008000000080004F
:1001B000000080000000800000008000000080003F
:1001C000000080000000800000008000000080002F
:1001D000000080000000800000008000000080001F
:1001E000000000000000000000000000000000000F
:1001F00000000000000000000000000000000000FF
:1002000000000000000000000000000000000000EE
:1002100000000000000000000000000000000000DE
:10022000000000000000000000000000000000C00E
:10023000000001E0000001E0000000C0000000003C
:1002400000000000000000000000000000000000AE
:10025000000000000000000000000000000000009E
:10026000000000000000000000000000000000008E
:10027000000000000000000000000000000000007E
:10028000000000000000000000000000000000006E
:10029000000000000000000000000000000000005E
:1002A00000000000000000000000000C000000380A
:1002B000000000E00000038000000E000000380095
:1002C0000000E00000038000000E00000038000085
:1002D00000E00000038000000E0000001800000095
:1002E000000000000000000000000000000000000E
:1002F00000000000000000000000000000000000FE
:1003000000000000000000000000000000000000ED
:1003100000000000000000000000000000000000DD
:10032000000000000000000000000000000FF800C6
:10033000007FFF0000F00780018000C00300006024
:1003400002000020020000200200002003000060E4
:10035000018000C000E00380007FFF00000FF80074
:10036000000000000000000000000000000000008D
:10037000000000000000000000000000000000007D
:10038000000000000000000000000000000000006D
:10039000000000000000000000000000000000005D
:1003A000000000000000000000000000000000004D
:1003B000008000200080002000800020008000607D
:1003C00001FFFFE003FFFFE00000006000000020ED
:1003D00000000020000000200000000000000000DD
:1003E000000000000000000000000000000000000D
:1003F00000000000000000000000000000000000FD
:1004000000000000000000000000000000000000EC
:1004100000000000000000000000000000000000DC
:10042000000000000000000000000000007800E074
:100430000098016001000260020004600200086090
:100440000200106002002060020040600300806033
:100450000183006001FE00E0007C078000000000D6
:10046000000000000000000000000000000000008C
:10047000000000000000000000000000000000007C
:10048000000000000000000000000000000000006C
:10049000000000000000000000000000000000005C
:1004A00000000000000000000000000000F00780D5
:1004B00001F007C0010000400200002002010020FE
:1004C00002010020020100200303802001868040F9
:1004D00001FCC0C000787F8000001E00000000000A
:1004E000000000000000000000000000000000000C
:1004F00000000000000000000000000000000000FC
:1005000000000000000000000000000000000000EB
:1005100000000000000000000000000000000000DB
:10052000000000000000000000000800000038008B
:10053000000048000001880000060800000C0810B8
:10054000003008100040081001FFFFF003FFFFF02B
:1005500003FFFFF000000810000008100000081062
:10056000000000000000000000000000000000008B
:10057000000000000000000000000000000000007B
:10058000000000000000000000000000000000006B
:10059000000000000000000000000000000000005B
:1005A00000000000000000000000000000000780C4
:1005B000001F864003E10020030200200304002006
:1005C000030400200304002003040020030600406D
:1005D000030301C00301FF8003007E000000000050
:1005E000000000000000000000000000000000000B
:1005F00000000000000000000000000000000000FB
:1006000000000000000000000000000000000000EA
:1006100000000000000000000000000000000000DA
:100620000000000000000000000000000007FC00C7
:10063000003FFF000070C380008180C001010060A6
:100640000302002002020020020200200202002019
:100650000203004001C180C000C0FF8000007E0096
:10066000000000000000000000000000000000008A
:10067000000000000000000000000000000000007A
:10068000000000000000000000000000000000006A
:10069000000000000000000000000000000000005A
:1006A00000000000000000000000000000F000005A
:1006B00003C000000380000003000000030007E007
:1006C00003003FE00301C000030600000318000020
:1006D0000360000003800000030000000000000031
:1006E000000000000000000000000000000000000A
:1006F00000000000000000000000000000000000FA
:1007000000000000000000000000000000000000E9
:1007100000000000000000000000000000000000D9
:10072000000000000000000000001F0000783F8073
:1007300000FC60C0018EC04003078020020300203F
:1007400002018020020180200201C0200301E0405C
:10075000018670C000FC3F8000781F000000000090
:100760000000000000000000000000000000000089
:100770000000000000000000000000000000000079
:100780000000000000000000000000000000000069
:100790000000000000000000000000000000000059
:1007A0000000000000000000003F000000FF81C0CA
:1007B00001C0C1C0010060200200202002002020F2
:1007C0000200202002002060020040C00100C18021
:1007D00000C18F00007FFE00001FF000000000003D
:1007E0000000000000000000000000000000000009
:1007F00000000000000000000000000000000000F9
:1008000000000000000000000000000000000000E8
:1008100000000000000000000000000000000000D8
:1008200000000000000000000000000000000000C8
:10083000000000000000000000000000000300C0F5
:10084000000781E0000781E0000300C00000000015
:100850000000000000000000000000000000000098
:100860000000000000000000000000000000000088
:100870000000000000000000000000000000000078
:100880000000000000000000000000000000000068
:100890000000000000000000000000000000000058
:1008A0000000000000000000000000000000000048
:1008B00000000000000000000000000000060066CC
:1008C00000060078000000000000000000000000AA
:1008D0000000000000000000000000000000000018
:1008E0000000000000000000000000000000000008
:1008F00000000000000000000000000000000000F8
:1009000000000000000000000000000000000000E7
:1009100000000000000000000000000000000000D7
:100920000000000000000000000000000000800047
:100930000001C0000003600000063000000C180039
:1009400000180C00003006000060030000C00180A9
:100950000100004002000020040000100000000020
:100960000000000000000000000000000000000087
:100970000000000000000000000000000000000077
:100980000000000000000000000000000000000067
:100990000000000000000000000000000000000057
:1009A000000000000000000000041000000410001F
:1009B00000041000000410000004100000041000E7
:1009C00000041000000410000004100000041000D7
:1009D00000041000000410000004100000041000C7
:1009E0000000000000000000000000000000000007
:1009F00000000000000000000000000000000000F7
:100A000000000000000000000000000000000000E6
:100A100000000000000000000000000000000000D6
:100A200000000000000000000000000004000010B2
:100A3000020000200100004000C0018000600300AF
:100A40000030060000180C00000C180000063000F2
:100A5000000360000001C0000000800000000000F2
:100A60000000000000000000000000000000000086
:100A70000000000000000000000000000000000076
:100A80000000000000000000000000000000000066
:100A90000000000000000000000000000000000056
:100AA00000000000000000000000000000780000CE
:100AB00001F800000238000002000000040000C03D
:100AC000040079E0040081E0040100C00403000098
:100AD000020200000306000001FC000000F8000014
:100AE0000000000000000000000000000000000006
:100AF00000000000000000000000000000000000F6
:100B000000000000000000000000000000000000E5
:100B100000000000000000000000000000000000D5
:100B20000000000000000000000FF800003FFE0081
:100B30000070078000C000C00101F8400307FC20DE
:100B4000021E04200230082002203020023FFC2038
:100B5000013F044001800CC000E03180001FC20052
:100B60000000000000000000000000000000000085
:100B70000000000000000000000000000000000075
:100B80000000000000000000000000000000000065
:100B90000000000000000000000000000000000055
:100BA000000000000000002000000060000003E0E2
:100BB00000003E200003E020003E200003E0200073
:100BC0000380200007FC2000003FE0000003FE201F
:100BD00000003FE0000001E00000002000000020D5
:100BE0000000000000000000000000000000000005
:100BF00000000000000000000000000000000000F5
:100C000000000000000000000000000000000000E4
:100C100000000000000000000000000000000000D4
:100C20000000000000000000020000200200002080
:100C300003FFFFE003FFFFE00201002002010020AC
:100C40000201002002010020020100200303002015
:100C50000186806001FCC0C000F87F8000001F009A
:100C60000000000000000000000000000000000084
:100C70000000000000000000000000000000000074
:100C80000000000000000000000000000000000064
:100C90000000000000000000000000000000000054
:100CA00000000000000000000007F800003FFF0007
:100CB0000070078000C000C0010000400300002059
:100CC000020000200200002002000020020000209C
:100CD00001000040018000C003C001800030060018
:100CE0000000000000000000000000000000000004
:100CF00000000000000000000000000000000000F4
:100D000000000000000000000000000000000000E3
:100D100000000000000000000000000000000000D3
:100D2000000000000000000002000020020000207F
:100D300003FFFFE003FFFFE00200002002000020AD
:100D400002000020020000200300006001000040BB
:100D5000018000C000F00780007FFE00000FF80057
:100D60000000000000000000000000000000000083
:100D70000000000000000000000000000000000073
:100D80000000000000000000000000000000000063
:100D90000000000000000000000000000000000053
:100DA00000000000000000000200002002000020FF
:100DB00003FFFFE003FFFFE002010020020100202B
:100DC0000201002002010020020100200203802015
:100DD000020FE0200300006003C000E00060030099
:100DE0000000000000000000000000000000000003
:100DF00000000000000000000000000000000000F3
:100E000000000000000000000000000000000000E2
:100E100000000000000000000000000000000000D2
:100E2000000000000000000002000020020000207E
:100E300003FFFFE003FFFFE00201002002010020AA
:100E40000201000002010000020100000201000096
:100E500002038000030FE0000300000003C0000055
:100E60000060000000000000000000000000000022
:100E70000000000000000000000000000000000072
:100E80000000000000000000000000000000000062
:100E90000000000000000000000000000000000052
:100EA00000000000000000000007F800003FFE0006
:100EB0000070078001C001C0010000400300002055
:100EC000020000200200002002000020010020207B
:100ED0000100204003C03F8000303F800000200020
:100EE00000002000000000000000000000000000E2
:100EF00000000000000000000000000000000000F2
:100F000000000000000000000000000000000000E1
:100F100000000000000000000000000000000000D1
:100F200000000000020000200200002003FFFFE09C
:100F300003FFFFE00200802002008020000080000C
:100F4000000080000000800002008020020080205D
:100F500003FFFFE003FFFFE002000020020000208B
:100F60000000000000000000000000000000000081
:100F70000000000000000000000000000000000071
:100F80000000000000000000000000000000000061
:100F90000000000000000000000000000000000051
:100FA0000000000000000000000000000000000041
:100FB00002000020020000200200002002000020A9
:100FC00003FFFFE003FFFFE002000020020000201B
:100FD00002000020020000200000000000000000CD
:100FE0000000000000000000000000000000000001
:100FF00000000000000000000000000000000000F1
:1010000000000000000000000000000000000000E0
:1010100000000000000000000000000000000000D0
:1010200000000000000000000000000E0000000FA3
:101030000000000F0000000102000001020000019A
:10104000020000030200000603FFFFFC03FFFFF89D
:101050000200000002000000020000000200000088
:101060000000000000000000000000000000000080
:101070000000000000000000000000000000000070
:101080000000000000000000000000000000000060
:101090000000000000000000000000000000000050
:1010A00000000000000000000200002002000020FC
:1010B00003FFFFE003FFFFE00200C0200201002069
:1010C00000078000000FE0000030F80002603E20C2
:1010D00003800F20030003E0020000E00200002074
:1010E00000000020000000000000000000000000E0
:1010F00000000000000000000000000000000000F0
:1011000000000000000000000000000000000000DF
:1011100000000000000000000000000000000000CF
:10112000000000000000000002000020020000207B
:1011300003FFFFE003FFFFE00200002002000020A9
:10114000000000200000002000000020000000201F
:101150000000002000000060000000E0000003002C
:10116000000000000000000000000000000000007F
:10117000000000000000000000000000000000006F
:10118000000000000000000000000000000000005F
:10119000000000000000000000000000000000004F
:1011A00000000000020000200200002003FFFFE01A
:1011B00003E0002003FF0020001FF0000001FF807B
:1011C00000000FE000001E000003E000003E0020D1
:1011D00003E0002003FFFFE003FFFFE00200002028
:1011E00002000020000000000000000000000000DD
:1011F00000000000000000000000000000000000EF
:1012000000000000000000000000000000000000DE
:1012100000000000000000000000000000000000CE
:1012200000000000020000200200002003FFFFE099
:101230000380002003F0002000FC0000001F0000DD
:101240000007C0000001F00000007C0002001F80C9
:10125000020007E003FFFFE00200000002000000C0
:10126000000000000000000000000000000000007E
:10127000000000000000000000000000000000006E
:10128000000000000000000000000000000000005E
:10129000000000000000000000000000000000004E
:1012A0000000000000000000000FF800003FFE00FA
:1012B00000F00780018000C0010000400200002013
:1012C0000200002002000020020000200100004077
:1012D000018000C000F00380003FFE00000FF80016
:1012E00000000000000000000000000000000000FE
:1012F00000000000000000000000000000000000EE
:1013000000000000000000000000000000000000DD
:1013100000000000000000000000000000000000CD
:101320000000000000000000020000200200002079
:1013300003FFFFE003FFFFE00200802002008020A7
:101340000200800002008000020080000200800095
:10135000030180000183000000FE0000007C00000B
:10136000000000000000000000000000000000007D
:10137000000000000000000000000000000000006D
:10138000000000000000000000000000000000005D
:10139000000000000000000000000000000000004D
:1013A0000000000000000000000FF800007FFF00B8
:1013B00000F00380018001C001000640020004200B
:1013C0000200042002000620020003E0010000F8F1
:1013D0000180005C00E0038C003FFF0C000FFC1854
:1013E00000000000000000000000000000000000FD
:1013F00000000000000000000000000000000000ED
:1014000000000000000000000000000000000000DC
:1014100000000000000000000000000000000000CC
:101420000000000000000000020000200200002078
:1014300003FFFFE003FFFFE00201002002010020A4
:10144000020180000201E0000201FC0003033F8072
:10145000018607E001FC00E000F800200000002009
:10146000000000000000000000000000000000007C
:10147000000000000000000000000000000000006C
:10148000000000000000000000000000000000005C
:10149000000000000000000000000000000000004C
:1014A00000000000000000000000000000780600BE
:1014B00000FE01E0018600C003030040020300209B
:1014C00002018020020180200201C0200200C02011
:1014D0000100E060018070C003E03F8000001F0059
:1014E00000000000000000000000000000000000FC
:1014F00000000000000000000000000000000000EC
:1015000000000000000000000000000000000000DB
:1015100000000000000000000000000000000000CB
:1015200000000000000000000060000003800000D8
:101530000300000002000000020000200200002062
:1015400003FFFFE003FFFFE0020000200200002095
:1015500002000000020000000380000000E0000024
:10156000000000000000000000000000000000007B
:10157000000000000000000000000000000000006B
:10158000000000000000000000000000000000005B
:10159000000000000000000000000000000000004B
:1015A00000000000020000000200000003FFFF0036
:1015B00003FFFFC0020000400200006000000020A6
:1015C0000000002000000020000000200200004079
:1015D0000200008003FFFF00020000000200000084
:1015E00000000000000000000000000000000000FB
:1015F00000000000000000000000000000000000EB
:1016000000000000000000000000000000000000DA
:1016100000000000000000000000000000000000CA
:1016200000000000000000000200000002000000B6
:1016300003C0000003FC0000023FC0000003F800EC
:1016400000007F80000007E00000078000007800B5
:101650000203C000023C000003C0000002000000C2
:101660000200000000000000000000000000000078
:10167000000000000000000000000000000000006A
:10168000000000000000000000000000000000005A
:10169000000000000000000000000000000000004A
:1016A000000000000200000003C0000003FF8000F3
:1016B000023FFE0002007FE000000F000200F00089
:1016C00003EF000003FF8000020FFE0000003FE078
:1016D00000001F000207E00003F800000300000004
:1016E00002000000000000000000000000000000F8
:1016F00000000000000000000000000000000000EA
:1017000000000000000000000000000000000000D9
:1017100000000000000000000000000000000000C9
:101720000000000000000000020000200200002075
:10173000038000E003F0032002FC0C20021F3000B5
:101740000007C0000007F00002187C0002601F20A4
:10175000038003E0020000E00200002000000020FF
:101760000000000000000000000000000000000079
:101770000000000000000000000000000000000069
:101780000000000000000000000000000000000059
:101790000000000000000000000000000000000049
:1017A0000000000000000000020000000300000034
:1017B00003C0000003F80000023E0020020FC0201A
:1017C0000001FFE000007FE000038020021C0020F9
:1017D0000270000003800000020000000200000010
:1017E00000000000000000000000000000000000F9
:1017F00000000000000000000000000000000000E9
:1018000000000000000000000000000000000000D8
:1018100000000000000000000000000000000000C8
:10182000000000000000000000000020006000E058
:10183000038003E003000FA002003E200200F82016
:101840000203E020020F8020023E002002780020E8
:1018500003E00060038000E00200030000000000DD
:101860000000000000000000000000000000000078
:101870000000000000000000000000000000000068
:101880000000000000000000000000000000000058
:101890000000000000000000000000000000000048
:1018A0000000000000000000000000000000000038
:1018B0000000000000000000000000001FFFFFFC0F
:1018C00010000004100000041000000410000004C8
:1018D00010000004100000041000000400000000CC
:1018E00000000000000000000000000000000000F8
:1018F00000000000000000000000000000000000E8
:1019000000000000000000000000000000000000D7
:1019100000000000000000000000000000000000C7
:1019200000000000000000000000000000000000B7
:101930000700000003C0000000780000001E000047
:101940000003C0000000F00000001E00000007803F
:10195000000000F00000003C000000060000000055
:101960000000000000000000000000000000000077
:101970000000000000000000000000000000000067
:101980000000000000000000000000000000000057
:101990000000000000000000000000000000000047
:1019A0000000000000000000000000001000000423
:1019B00010000004100000041000000410000004D7
:1019C00010000004100000041FFFFFFC00000000D6
:1019D0000000000000000000000000000000000007
:1019E00000000000000000000000000000000000F7
:1019F00000000000000000000000000000000000E7
:101A000000000000000000000000000000000000D6
:101A100000000000000000000000000000000000C6
:101A200000000000000000000000000000000000B6
:101A30000000000002000000040000000800000098
:101A4000180000001000000018000000180000003E
:101A50000400000002000000000000000000000080
:101A60000000000000000000000000000000000076
:101A70000000000000000000000000000000000066
:101A80000000000000000000000000000000000056
:101A90000000000000000000000000000000000046
:101AA0000000000000000001000000010000000133
:101AB0000000000100000001000000010000000122
:101AC0000000000100000001000000010000000112
:101AD0000000000100000001000000010000000102
:101AE00000000001000000000000000000000000F5
:101AF00000000000000000000000000000000000E6
:101B000000000000000000000000000000000000D5
:101B100000000000000000000000000000000000C5
:101B200000000000000000000000000000000000B5
:101B3000100000001000000010000000180000005D
:101B40000800000004000000000000000000000089
:101B50000000000000000000000000000000000085
:101B60000000000000000000000000000000000075
:101B70000000000000000000000000000000000065
:101B80000000000000000000000000000000000055
:101B90000000000000000000000000000000000045
:101BA00000000000000000000000038000018FC062
:101BB00000038C6000061820000410200004102090
:101BC0000004202000042040000620400003FFC045
:101BD0000001FFE00000002000000020000000C025
:101BE00000000000000000000000000000000000F5
:101BF00000000000000000000000000000000000E5
